:100000000000032029C201000DC20100C5C101008A
:10001000C5C10100C5C10100C5C10100C5C10100C4
:10002000C5C10100C5C10100C5C101000DC201006B
:100030000DC20100C5C10100E5B601005DB90100B6
:100040000DC201000DC201000DC201000DC2010070
:100050000DC201000DC201000DC201000DC2010060
:100060000DC201000DC201000DC201000DC2010050
:100070000DC201000DC201000DC201000DC2010040
:100080000DC201000DC201000DC201000DC2010030
:100090000DC201000DC201000DC201000DC2010020
:1000A000C9810100258301000DC201000DC20100BC
:1000B0000DC201000DC201000DC2010085D4010076
:1000C0000DC2010049EA01000DC20100A5EB0100CB
:1000D0000DC20100D5EC01000DC201000DC20100EE
:1000E0000DC201000DC201000DC201000DC20100D0
:1000F0000DC201000DC201000DC201000DC20100C0
:100100000DC201000DC201000DC201000DC20100AF
:100110000DC20100B9D701000DC201000DC20100DE
:100120000DC201000DC201000DC201000DC201008F
:100130000DC201000DC201000DC201000DC201007F
:1001400031B401000DC2010005EE01000DC2010035
:100150000DC201000DC201000DC201000DC201005F
:100160000DC201000DC20100818401000DC2010019
:100170000DC201000DC201000DC201000DC201003F
:100180000DC201000DC201000DC201000DC201002F
:100190000DC201000DC2010035EF01000DC20100CA
:1001A0000DC201000DC201000DC201000DC201000F
:1001B0000DC201000DC201000DC201000DC20100FF
:1001C0000DC201000DC201000DC201000DC20100EF
:1001D000FFFFFFFFFFFFFFFFFFFFFFFFFFFFFFFF2F
:10040000FFFFFFFFFFFFFFFFFFFFFFFFDEF9FFFF23
:1004100010B5054C237833B9044B13B10448AFF33E
:1004200000800123237010BD00F0002000000000B8
:100430002C550200084B10B51BB108490848AFF312
:1004400000800848036803B910BD074B002BFBD0A0
:10045000BDE81040184700BF0000000004F0002075
:100460002C550200F4E9002000000000704700BF96
:1004700010B54FF4097104461CF09EF8204610BDDB
:1004800070B54FF06A522DED028B064643F2586369
:1004900008EE902A40F6DB72C0F202034FF61A050E
:1004A00040F6DA70C4F24902C2F20005C3F64920F0
:1004B00008EE102A336000240FE007EE904AF8EEB1
:1004C000E77A77EE807A67EEA87A67EE887A27EE89
:1004D000800A1EF079FF10EE100A21F0C7FD41ECF2
:1004E000100B1EF0BDFE00230022CCF2900351EC55
:1004F000100B21F00FFE41EC100B1EF0C5FE51EC6D
:10050000100B22F0DFF80134B4F5806FB6EE000A6C
:1005100025F8020FD1D14FF06A534FF21A0508EEB9
:10052000103AC2F20005002407EE904AF8EEE77A8E
:10053000013467EE887A17EE900A21F097FD9FED5F
:10054000140B41EC110B1FF013F8002351EC100BAE
:100550000022C3F6F07321F029FC00230022C4F22C
:10056000B00321F0D7FD22F0CDF821F07FFD41EC62
:10057000100B1EF089FE51EC100B22F0A3F8B4F51D
:10058000806F25F8020FCFD1BDEC028B304670BDD5
:100590000000000000000040704700BF10B54FF49D
:1005A000097104461CF008F8204610BD2DE9F04FF3
:1005B0004DF63456C2F200060A9D0B989DF8307035
:1005C000B6F800C043F27064C0F20204C5EB000A42
:1005D000002F18BF0C466FEA0C0B0AF1200A4DF6EB
:1005E00034194DF63438043A271FA1F1040E0FFADE
:1005F0008BFB4FEAAA1AC2F20009C2F200080026D9
:1006000027E0B4F5007F02D08CB3C943C9B239F8F2
:1006100011104CEA010101EBC00080B20BEA0004AA
:10062000E143C9B2241238F8111001F58061490084
:10063000E14010EA0C0F18BFC94357F8044F09985E
:1006400009B2013604EB8131402E03444EF8041FF9
:1006500010D052F8041F1944891301F44074554412
:10066000B4F5807FC9B2A8B2CBD1C943C9B239F8B9
:100670001110D0E7BDE8F08F2DE9F04F4DF634555D
:10068000C2F2000509982E880A9D9DF82C7043F24D
:100690007064C0F20204C0EB050E002F14BF0F46B9
:1006A00027466FEA06090EF1200E4DF634184DF676
:1006B000343C3C1F0D1F0FFA89F9FC374FEAAE1E80
:1006C000C2F20008C2F2000C2AE0BBF5007F04D0A1
:1006D000BBF1000F30D0C943C9B238F81110314313
:1006E00001EBCA0A1FFA8AFA09EA0A0B6FEA0B0140
:1006F000C9B24FEA2B2B3CF8111001F5806149007B
:100700001AEA060F21FA0BF154F804AF18BFC943D7
:1007100009B20AEB8131BC421A4445F8041F0ED0DD
:10072000911301F4407B7044BBF5807F1FFA80FA7F
:10073000C9B2CAD1C943C9B238F81110D0E7BDE86F
:10074000F08F00BF2DE9F04F4DF6345083B0C2F268
:1007500000000D9EB0F800C00C9C9DF840A00F9FBB
:100760000E980E9D019343F2706EC0F2020EC4EB20
:10077000060B6FEA0C06BAF1000F14BF8A46F24668
:1007800033B20BF1200B4DF634194DF63438AAF183
:10079000040600686D680093A1F1040E0AF1FC0ADA
:1007A0004FEAAB1B0137C2F20009C2F2000829E090
:1007B000B0F5007F02D098B3DB43DBB239F81330D9
:1007C0004CEA030303EBC101009B89B203EA010079
:1007D000C343DBB2001238F8133003F580635B00CB
:1007E000C34011EA0C0F18BFDB4356F8041F0198F1
:1007F0001BB29B031944564502444EF8041F284679
:1008000011D01D4643193B4113449B1303F4407020
:100810005C44B0F5807FDBB2A1B2C9D1DB43DBB26F
:1008200039F81330CEE70E9A1560536003B0BDE877
:10083000F08F00BF2DE9F04F44F2A07403EB4303A7
:10084000C0F2020404EBC3050646144689460FCDE8
:1008500091B00AAF0FC795E80300002387E80300B3
:10086000012704F160088DF8247007978DF8253072
:100870008DF826300AAD48E00AF1FF3101EB011195
:1008800006EB0111133121F00F0194E80140C0146F
:10089000C0F500706060BEF1000F3FD0BEF5FE7F76
:1008A0003EDA10AFBA441AF81CCCBCF1000F04D0E9
:1008B00012F1000C18BF4FF0010CC3F301123AB152
:1008C00010AF07EB020B1BF81CBCBBF1000F34D1BF
:1008D00003F0C003C02B02D11B9B0F2B41DDA3688B
:1008E000E2680190CDF808C0CDF800E03046FFF78F
:1008F000C3FE9DF81C300AF81C3CE368A26803EBB9
:100900008213E3601034A04514D055F8043B13F073
:10091000030A03F00402AFD14946B6E740F2FF1ED6
:10092000B0F5FE7FBDDB002AE7D110AB9A440AF890
:100930001C2CE2E711B0BDE8F08F013A02EB021285
:10094000E368CDF80CC006EB02120290CDF804E08B
:10095000A0680090133222F00F023046FFF726FE07
:10096000C7E71F46E268A36803971A9F0190CDF876
:1009700010C00297CDF800E03046FFF7E3FEB8E77D
:1009800000207047704700BF704700BF704700BF2E
:10099000704700BF10B504461AF000FD204610BD98
:1009A00000F0F703F52B06D0F92804D0EF2803D880
:1009B00000F0F00070470020704700BF10B50446FB
:1009C00022F07EFB01462046BDE810401DF040BEEF
:1009D00010B5044622F074FB014620461DF038FE97
:1009E00004464EF2C000C2F200001BF0ABF82044F7
:1009F00010BD00BF43F2EC70F8B51D21C0F202003B
:100A00001DF026FE41F2B853C2F20103FE21986C9C
:100A100003681B68984743F60C000F21C0F20200E0
:100A20001DF016FE41F6DC73C2F20103FE219B6C41
:100A30001A691F46501C1861117057F8106FBE429A
:100A400024BF1B611E464FF0010E4FF0000C5A6987
:100A5000B24202F1010113D0596110785A6B8F42F2
:100A60004FEA201598BF5B619C18511CBAB95A69AE
:100A700083F83050B242C3F834E002F10101EBD107
:100A800043F61C00C0F202000F211DF0E1FD4EF202
:100A9000C000C2F20000BDE8F8401BF053B80329C3
:100AA00084F830005963D2D1C3F830C0C3F834C0E1
:100AB000CDE700BF43F62C00F8B51821C0F20200C4
:100AC0001DF0C6FD41F2B853C2F20103FB21986C40
:100AD00003681B68984743F60C000F21C0F2020020
:100AE0001DF0B6FD41F6DC73C2F20103FB219B6CE5
:100AF0001A691F46501C1861117057F8106FBE42DA
:100B000024BF1B611E464FF0010E4FF0000C5A69C6
:100B1000B24202F1010113D0596110785A6B8F4231
:100B20004FEA201598BF5B619C18511CBAB95A69ED
:100B300083F83050B242C3F834E002F10101EBD146
:100B400043F61C00C0F202000F211DF081FD4EF2A1
:100B5000C000C2F20000BDE8F8401AF0F3BF03295C
:100B600084F830005963D2D1C3F830C0C3F834C020
:100B7000CDE700BF43F64800F8B51421C0F20200EB
:100B80001DF066FD41F2B853C2F20103FC21986CDE
:100B900003681B68984743F60C000F21C0F202005F
:100BA0001DF056FD41F6DC73C2F20103FC219B6C83
:100BB0001A691F46501C1861117057F8106FBE4219
:100BC00024BF1B611E464FF0010E4FF0000C5A6906
:100BD000B24202F1010113D0596110785A6B8F4271
:100BE0004FEA201598BF5B619C18511CBAB95A692D
:100BF00083F83050B242C3F834E002F10101EBD186
:100C000043F61C00C0F202000F211DF021FD4EF240
:100C1000C000C2F20000BDE8F8401AF093BF0329FB
:100C200084F830005963D2D1C3F830C0C3F834C05F
:100C3000CDE700BF43F66000F8B51521C0F2020011
:100C40001DF006FD41F2B853C2F20103FA21986C7F
:100C500003681B68984743F60C000F21C0F202009E
:100C60001DF0F6FC41F6DC73C2F20103FA219B6C25
:100C70001A691F46501C1861117057F8106FBE4258
:100C800024BF1B611E464FF0010E4FF0000C5A6945
:100C9000B24202F1010113D0596110785A6B8F42B0
:100CA0004FEA201598BF5B619C18511CBAB95A696C
:100CB00083F83050B242C3F834E002F10101EBD1C5
:100CC00043F61C00C0F202000F211DF0C1FC4EF2E1
:100CD000C000C2F20000BDE8F8401AF033BF03299B
:100CE00084F830005963D2D1C3F830C0C3F834C09F
:100CF000CDE700BF43F67800F8B51021C0F202003E
:100D000041F2E4641DF0A4FCC2F201044EF2C00002
:100D1000C2F200001AF016FF20680EF09DFD206858
:100D20000EF0A6FC20680EF0B7FC43F68C001B21E9
:100D3000C0F202001DF08CFC41F2B853C2F2010374
:100D4000FF21986C03681B68984743F60C000F213D
:100D5000C0F202001DF07CFC41F6DC73C2F201031C
:100D6000FF219B6C1A691F46501C1861117057F8BF
:100D7000106FBE4224BF1B611E464FF0010E4FF0A4
:100D8000000C5A69B24202F1010113D05961107886
:100D90005A6B8F424FEA201598BF5B619C18511C1B
:100DA000BAB95A6983F83050B242C3F834E002F15C
:100DB0000101EBD143F61C00C0F202000F211DF02F
:100DC00047FC4EF2C000C2F20000BDE8F8401AF045
:100DD000B9BE032984F830005963D2D1C3F830C0BA
:100DE000C3F834C0CDE700BF38B505464EF2C004A5
:100DF00043F6A800C2F200041E21C0F202001DF05A
:100E000027FC294600230A2220461AF0ADFE43F6AD
:100E1000C8000E21C0F202001DF01AFC41F2E0638E
:100E2000C2F201030A221978204600231AF09CFE20
:100E300043F6D8000121C0F202001DF009FC204653
:100E40001AF080FE002038BD2DE9F843044643F631
:100E5000DC001521C0F202001DF0FAFB210401F4B0
:100E6000FE0141F4734141F2007041F00201C2F20F
:100E7000010041F6DC7819F0CFF9C2F2010843F61F
:100E8000F4001421C0F202001DF0E2FBD8F8483053
:100E90001A699E46F321501C186111705EF8107F8C
:100EA000774524BF1B611F464FF0010C4FF000092E
:100EB0005A69BA4202F1010114D0596110785A6B93
:100EC0008E454FEA201698BF5B619D18511C002A81
:100ED00043D15A6983F83060BA42C3F834C002F192
:100EE0000101EAD1D8F848301A691F4604F07F049E
:100EF000511C1961147057F8106FBE4224BF1B615A
:100F00001E464FF0010E4FF0000C5A69B24202F13A
:100F1000010113D0596110785A6B8F424FEA2015A6
:100F200098BF5B619C18511C0ABB5A6983F830500A
:100F3000B242C3F834E002F10101EBD143F61C00E8
:100F4000C0F202000F211DF083FB4EF2C000C2F27E
:100F50000000BDE8F8431AF0F5BD032985F830001C
:100F60005963A5D1C3F83090C3F83490A0E70329A2
:100F700084F830005963C8D1C3F830C0C3F834C016
:100F8000C3E700BF43F60C1008B51021C0F2020001
:100F90001DF05EFB41F2B853C2F20103FA21986CD6
:100FA00003681B68984743F60C000F21C0F202004B
:100FB0001DF04EFB41F20070C2F201004FF60F210E
:100FC00019F02AF943F6F400C0F2020014211DF0D2
:100FD0003FFB4EF2C000C2F20000BDE808401AF02C
:100FE000B1BD00BF43F6201008B51321C0F20200C6
:100FF0001DF02EFB41F2B853C2F20103FB21986CA5
:1010000003681B68984743F60C000F21C0F20200EA
:101010001DF01EFB41F20070C2F201004FF60F31CD
:1010200019F0FAF843F6F400C0F2020014211DF0A2
:101030000FFB4EF2C000C2F20000BDE808401AF0FB
:1010400081BD00BF43F6341008B50F21C0F2020085
:101050001DF0FEFA41F2B853C2F20103FC21986C74
:1010600003681B68984743F60C000F21C0F202008A
:101070001DF0EEFA41F20070C2F201004FF60F418E
:1010800019F0CAF843F6F400C0F2020014211DF072
:10109000DFFA4EF2C000C2F20000BDE808401AF0CC
:1010A00051BD00BF43F6441008B51821C0F202003C
:1010B0001DF0CEFA41F2B853C2F20103FE21986C42
:1010C00003681B68984743F60C000F21C0F202002A
:1010D0001DF0BEFA41F20070C2F201004FF60F613E
:1010E00019F09AF843F6F400C0F2020014211DF042
:1010F000AFFA4EF2C000C2F20000BDE808401AF09C
:1011000021BD00BF43F66010F8B51821C0F20200FF
:101110001DF09EFA41F20070C2F201004FF60F611D
:1011200019F07AF843F6F4001421C0F202001DF021
:101130008FFA41F6DC73C2F20103FE219B6C1A693F
:101140001F46501C1861117057F8106FBE4224BF23
:101150001B611E464FF0010E4FF0000C5A6996427B
:1011600002F1010113D0596110785A6B8F424FEA96
:10117000201598BF5B619C18511CBAB95A6983F855
:1011800030509642C3F834E002F10101EBD143F64E
:101190001C00C0F202000F211DF05AFA4EF2C000EE
:1011A000C2F20000BDE8F8401AF0CCBC032984F874
:1011B00030005963D2D1C3F830C0C3F834C0CDE792
:1011C00043F67C10F8B50F21C0F202001DF040FA82
:1011D00041F20070C2F201004FF60F4119F01CF805
:1011E00043F6F4001421C0F202001DF031FA41F67A
:1011F000DC73C2F20103FC219B6C1A691F46501C70
:101200001861117057F8106FBE4224BF1B611E4653
:101210004FF0010E4FF0000C5A69964202F10101A5
:1012200013D0596110785A6B8F424FEA201598BF3E
:101230005B619C18511CBAB95A6983F830509642C8
:10124000C3F834E002F10101EBD143F61C00C0F217
:1012500002000F211DF0FCF94EF2C000C2F20000A6
:10126000BDE8F8401AF06EBC032984F830005963D9
:10127000D2D1C3F830C0C3F834C0CDE743F68C10E8
:10128000F8B51021C0F202001DF0E2F941F2007041
:10129000C2F201004FF60F2118F0BEFF43F6F40032
:1012A0001421C0F202001DF0D3F941F6DC73C2F242
:1012B0000103FA219B6C1A691F46501C18611170BA
:1012C00057F8106FBE4224BF1B611E464FF0010E3F
:1012D0004FF0000C5A69964202F1010113D0596196
:1012E00010785A6B8F424FEA201598BF5B619C18AB
:1012F000511CBAB95A6983F830509642C3F834E0A9
:1013000002F10101EBD143F61C00C0F202000F21F3
:101310001DF09EF94EF2C000C2F20000BDE8F84098
:101320001AF010BC032984F830005963D2D1C3F8F5
:1013300030C0C3F834C0CDE743F6A010F8B5132190
:10134000C0F202001DF084F941F20070C2F2010007
:101350004FF60F3118F060FF43F6F4001421C0F28D
:1013600002001DF075F941F6DC73C2F20103FB21A6
:101370009B6C1A691F46501C1861117057F8106F4A
:10138000BE4224BF1B611E464FF0010E4FF0000C01
:101390005A69964202F1010113D0596110785A6BD3
:1013A0008F424FEA201598BF5B619C18511CBAB957
:1013B0005A6983F830509642C3F834E002F10101D3
:1013C000EBD143F61C00C0F202000F211DF040F9E2
:1013D0004EF2C000C2F20000BDE8F8401AF0B2BB05
:1013E000032984F830005963D2D1C3F830C0C3F860
:1013F00034C0CDE743F67800F8B51021C0F2020002
:1014000041F2E4641DF024F9C2F201044EF2C0007E
:10141000C2F200001AF096FB20680EF01DFA206858
:101420000EF026F920680EF037F943F6B4101621B5
:10143000C0F202001DF00CF941F20070C2F201008E
:101440004FF60F7118F0E8FE43F6F4001421C0F2D5
:1014500002001DF0FDF841F6DC73C2F20103FF212A
:101460009B6C1A691F46501C1861117057F8106F59
:10147000BE4224BF1B611E464FF0010E4FF0000C10
:101480005A69964202F1010113D0596110785A6BE2
:101490008F424FEA201598BF5B619C18511CBAB966
:1014A0005A6983F830509642C3F834E002F10101E2
:1014B000EBD143F61C00C0F202000F211DF0C8F86A
:1014C0004EF2C000C2F20000BDE8F8401AF03ABB8C
:1014D000032984F830005963D2D1C3F830C0C3F86F
:1014E00034C0CDE72DE9F843044643F6CC101F2164
:1014F000C0F202001DF0ACF804F00F034FF202112D
:101500001B04C0F2100141F200701943C2F2010045
:1015100041F6DC7818F080FEC2F2010843F6F400D0
:101520001421C0F202001DF093F8D8F848301A696F
:101530009E46F121501C186111705EF8107F7745AE
:1015400024BF1B611F464FF0010C4FF000095A6980
:10155000BA4202F1010114D0596110785A6B8E45DC
:101560004FEA201698BF5B619D18511C002A41D19B
:101570005A6983F83060BA42C3F834C002F10101FD
:10158000EAD1D8F848301A691F46511C1961147005
:1015900057F8106FBE4224BF1B611E464FF0010E6C
:1015A0004FF0000C5A69B24202F1010113D05961A7
:1015B00010785A6B8F424FEA201598BF5B619C18D8
:1015C000511C0ABB5A6983F83050B242C3F834E068
:1015D00002F10101EBD143F61C00C0F202000F2121
:1015E0001DF036F84EF2C000C2F20000BDE8F8432C
:1015F0001AF0A8BA032985F830005963A7D1C3F8B7
:101600003090C3F83490A2E7032984F8300059637E
:10161000C8D1C3F830C0C3F834C0C3E743F6EC10F8
:1016200008B51621C0F202001DF012F841F2B853BD
:10163000C2F20103F621986C0368DB6C984743F60D
:101640000C000F21C0F202001DF002F841F2007000
:10165000C2F201004FF20F6118F0DEFD43F6F40014
:10166000C0F2020014211CF0F3FF4EF2C000C2F2DF
:101670000000BDE808401AF065BA00BF38B543F66F
:1016800078004EF2C00541F2E4641021C2F2010478
:10169000C2F20005C0F202001CF0DAFF28461AF080
:1016A00051FA20680EF0D8F820680DF0E1FF2068AC
:1016B0000DF0F2FF43F604201621C0F202001CF0E8
:1016C000C7FF41F2B853C2F20103FF21986C0368CF
:1016D0001B68984743F60C000F21C0F202001CF073
:1016E000B7FF41F20070C2F201004FF60F7118F01F
:1016F00093FD43F6F400C0F2020014211CF0A8FF91
:101700002846BDE838401AF01DBA00BFF8B50646B5
:1017100043F61C200C46C0F20200122115461CF0B4
:1017200097FF711EC9B20F2915D841F2B857C2F2FE
:10173000010741F0A001B86C03681B689847B86CBA
:10174000036804F07F011B689847B86C036805F0D4
:101750007F011B68984743F630200A21C0F202003F
:101760001CF076FF6B1E1B02240404F4FE0403F439
:1017700070632343310143F4504343F00D03C9B276
:1017800041F200701943C2F2010018F045FD43F622
:10179000F400C0F2020014211CF05AFF4EF2C00007
:1017A000C2F20000BDE8F8401AF0CCB943F63C2084
:1017B000F8B51621C0F202001CF04AFF41F2007099
:1017C000C2F201004FF20F6118F026FD43F6F4005B
:1017D0001421C0F202001CF03BFF41F6DC73C2F2A0
:1017E0000103F6219B6C1A691F46501C1861117089
:1017F00057F8106FBE4224BF1B611E464FF0010E0A
:101800004FF0000C5A69B24202F1010113D0596144
:1018100010785A6B8F424FEA201598BF5B619C1875
:10182000511CBAB95A6983F83050B242C3F834E057
:1018300002F10101EBD143F61C00C0F202000F21BE
:101840001CF006FF4EF2C000C2F20000BDE8F840F6
:101850001AF078B9032984F830005963D2D1C3F85B
:1018600030C0C3F834C0CDE7F8B541F2E063C2F24E
:1018700001030E461B781446054623B1984202D058
:10188000FFF7B2FA38B141F2E463C2F20103314624
:1018900018680DF0BBFD43F654201221013DC0F243
:1018A00002001CF0D5FEE9B20F2915D841F2B85755
:1018B000C2F2010741F08001B86C03681B689847C9
:1018C000B86C036806F07F011B689847B86C036822
:1018D00004F07F011B68984743F60C000F21C0F20B
:1018E00002001CF0B5FE230603F0FE43310443F46E
:1018F000004301F4FE012D0243F008030B4341F2C3
:10190000007005F470611943C2F2010018F084FC04
:1019100043F6F400C0F2020014211CF099FE4EF2CE
:10192000C000C2F20000BDE8F8401AF00BB900BFD9
:10193000F8B541F2E463C2F2010305461B6801F504
:10194000005643F668200C46013D0D21C3F8C060E7
:10195000C0F202001CF07CFEE9B20F2915D841F25A
:10196000B857C2F2010741F0E001B86C03681B6888
:101970009847B86C036806F07F011B689847B86CFD
:101980000368C6F3C6111B68984743F60C0004F3BE
:101990000D040F2104F50054C0F202001CF058FEA3
:1019A0002902230403F4FE0301F47061194341F496
:1019B0006041640404F0FE4441F00E0141F2007005
:1019C0002143C2F2010018F027FC43F6F400C0F2F4
:1019D000020014211CF03CFE4EF2C000C2F20000D6
:1019E000BDE8F8401AF0AEB81F2970B50C460546A0
:1019F00008D840F26853C2F2010318780EF03CFE9A
:101A00000AF0B6FC43F678200D21013DC0F2020039
:101A10001CF01EFEE9B20F290FD841F2B856C2F2EF
:101A2000010641F0C001B06C03681B689847B06CB8
:101A3000036804F07F011B68984743F60C000F21F0
:101A4000C0F202001CF004FE230403F4FE0329028A
:101A500043F4404343F00C0301F4706141F2007021
:101A60001943C2F2010018F0D7FB43F6F400C0F2AC
:101A7000020014211CF0ECFD4EF2C000C2F2000086
:101A8000BDE870401AF05EB8F8B541F2E063C2F20A
:101A900001030E461B781446054623B1984202D036
:101AA000FFF7A2F940B141F2E463C2F2010322461A
:101AB000186831460DF06AFA43F688201121013D7D
:101AC000C0F202001CF0C4FDE9B20F2915D841F2A2
:101AD000B857C2F2010741F09001B86C03681B6867
:101AE0009847B86C036806F07F011B689847B86C8C
:101AF000036804F07F011B68984743F60C000F2130
:101B0000C0F202001CF0A4FD230603F0FE433104E2
:101B100043F4104301F4FE012D0243F009030B438B
:101B200041F2007005F470611943C2F2010018F02F
:101B300073FB43F6F400C0F2020014211CF088FD90
:101B40004EF2C000C2F20000BDE8F84019F0FABF42
:101B5000F0B54AF23472C2F2010283B040F250632F
:101B600011680091C2F2010300991E681268019287
:101B700041F2BC65C2F2010541F2B452C2F2010267
:101B8000891B43F69C204EF2C004C2F20004019F60
:101B9000298000260C21C0F2020016701F601CF084
:101BA00057FD2B8820464EF6602191FBF3F119F08A
:101BB0006BFF43F6AC200521C0F202001CF048FD8B
:101BC0002988204619F060FF43F6B4200F21C0F2A7
:101BD00002001CF03DFD204619F0B4FF03B0F0BD3B
:101BE00008B541F2B451C2F201014AF6AB230A78BA
:101BF0000132D2B2CAF6AA23A3FB02031B0903EBEC
:101C00004303A2EBC30313F0FF0F0A7001D1FFF7E8
:101C10009FFF43F6C4201021C0F202001CF018FD03
:101C200041F2B853C2F20103F821986C03681B68B3
:101C3000984743F60C000F21C0F202001CF008FD8B
:101C400041F20070C2F201004FF60F0118F0E4FA01
:101C500043F6F400C0F2020014211CF0F9FC4EF22D
:101C6000C000C2F20000BDE8084019F06BBF00BF21
:101C7000F8B541F2B451C2F201014AF6AB230A7839
:101C80000132D2B2CAF6AA23A3FB02031B0903EB5B
:101C90004303A2EBC30313F0FF0F0A7001D1FFF758
:101CA00057FF43F6D8201021C0F202001CF0D0FCF0
:101CB00041F20070C2F201004FF60F0118F0ACFAC9
:101CC00043F6F4001421C0F202001CF0C1FC41F6FE
:101CD000DC73C2F20103F8219B6C1A691F46501C89
:101CE0001861117057F8106FBE4224BF1B611E4669
:101CF0004FF0010E4FF0000C5A69964202F10101BB
:101D000013D0596110785A6B8F424FEA201598BF53
:101D10005B619C18511CBAB95A6983F830509642DD
:101D2000C3F834E002F10101EBD143F61C00C0F22C
:101D300002000F211CF08CFC4EF2C000C2F2000029
:101D4000BDE8F84019F0FEBE032984F8300059635D
:101D5000D2D1C3F830C0C3F834C0CDE7F8B541F2F2
:101D6000B451C2F201014AF6AB230A780132D2B271
:101D7000CAF6AA23A3FB02031B0903EB4303A2EB4E
:101D8000C30313F0FF0F0A7001D1FFF7E1FE43F622
:101D9000EC201521C0F202001CF05AFC41F2B853AD
:101DA000C2F20103F821986C03681B68984743F658
:101DB0000C000F21C0F202001CF04AFC41F6DC735B
:101DC000C2F20103F8219B6C1A691F46501C18616E
:101DD000117057F8106FBE4224BF1B611E464FF0B2
:101DE000010E4FF0000C5A69B24202F1010113D00A
:101DF000596110785A6B8F424FEA201598BF5B618A
:101E00009C18511CBAB95A6983F83050B242C3F8D1
:101E100034E002F10101EBD143F61C00C0F20200F4
:101E20000F211CF015FC4EF2C000C2F20000BDE80C
:101E3000F84019F087BE032984F830005963D2D1E5
:101E4000C3F830C0C3F834C0CDE700BF43F6043058
:101E5000F8B51B21C0F202001CF0FAFB41F2B853A6
:101E6000C2F20103F621986C0368DB6C984743F6D5
:101E70000C000F21C0F202001CF0EAFB41F6DC73FB
:101E8000C2F20103F6219B6C1A691F46501C1861AF
:101E9000117057F8106FBE4224BF1B611E464FF0F1
:101EA000010E4FF0000C5A69B24202F1010113D049
:101EB000596110785A6B8F424FEA201598BF5B61C9
:101EC0009C18511CBAB95A6983F83050B242C3F811
:101ED00034E002F10101EBD143F61C00C0F2020034
:101EE0000F211CF0B5FB4EF2C000C2F20000BDE8AD
:101EF000F84019F027BE032984F830005963D2D185
:101F0000C3F830C0C3F834C0CDE700BF2DE9F843B3
:101F100041F2B8550446C2F2010543F620302421AF
:101F2000C0F202001CF094FBA86C0368F1211B684E
:101F30009847A86C036821461B6841F6DC789847EF
:101F4000C2F2010843F60C000F21C0F202001CF09F
:101F50007FFBD8F848301A699E46F121501C186161
:101F600011705EF8107F774524BF1B611F464FF04C
:101F7000010C4FF000095A69BA4202F1010114D074
:101F8000596110785A6B8E454FEA201698BF5B61F5
:101F90009D18511C002A41D15A6983F83060BA4219
:101FA000C3F834C002F10101EAD1D8F848301A6907
:101FB0001F46511C1961147057F8106FBE4224BFA0
:101FC0001B611E464FF0010E4FF0000C5A69B242E1
:101FD00002F1010113D0596110785A6B8F424FEA18
:101FE000201598BF5B619C18511C0ABB5A6983F885
:101FF0003050B242C3F834E002F10101EBD143F6B4
:102000001C00C0F202000F211CF022FB4EF2C000A7
:10201000C2F20000BDE8F84319F094BD032985F829
:1020200030005963A7D1C3F83090C3F83490A2E7C9
:10203000032984F830005963C8D1C3F830C0C3F80D
:1020400034C0C3E72DE9F84341F2B8540746C2F261
:10205000010443F648301A21C0F202001CF0F8FADD
:10206000A06C0368F3211B689847A06C036807F015
:102070007F07DB6C394641F6DC789847C2F20108ED
:1020800043F60C000F21C0F202001CF0E1FAD8F870
:1020900048301A699E46501CF321186111705EF891
:1020A000100F704524BF1B6118464FF0010C4FF014
:1020B00000095A69824202F1010114D05961147871
:1020C0005A6B8E454FEA241698BF5B619D18511CD0
:1020D000002A3FD15A6983F830608242C3F834C085
:1020E00002F10101EAD1D8F848301A699E46511C24
:1020F000196117705EF8106F764524BF1B611E468C
:1021000001274FF0000C5A69B24202F1010112D0CE
:10211000596110785A6B8E454FEA201598BF5B6164
:102120009C18511C02BB5A6983F83050B2425F635D
:1021300002F10101ECD143F61C00C0F202000F21B4
:102140001CF086FA4EF2C000C2F20000BDE8F8436F
:1021500019F0F8BC032985F830405963A9D1C3F8B8
:102160003090C3F83490A4E7032984F83000596311
:10217000C9D1C3F830C0C3F834C0C4E738B541F2A0
:10218000B8550446C2F2010543F664301521C0F289
:1021900002001CF05DFAA86C0368F3211B689847E5
:1021A000A86C036804F07F01DB6C984743F60C00D1
:1021B0000F21C0F202001CF04BFA210401F4FE01D1
:1021C00041F4734141F2007041F00201C2F201009A
:1021D00018F022F843F6F400C0F2020014211CF0BB
:1021E00037FA4EF2C000C2F20000BDE8384019F0E4
:1021F000A9BC00BF38B541F2B8550446C2F201058A
:1022000043F67C301F21C0F202001CF021FAA86CBA
:102210000368F1211B689847A86C036821461B6876
:10222000984743F60C000F21C0F2020004F00F049F
:102230001CF00EFA44F010044FF2021141F200704B
:1022400041EA0441C2F2010017F0E6FF43F6F40050
:10225000C0F2020014211CF0FBF94EF2C000C2F2E1
:102260000000BDE8384019F06DBC00BF1F292DE902
:10227000F8430F46044608D840F26853C2F20103FF
:1022800018780EF0F9F90AF073F843F69C30C0F2B2
:10229000020012211CF0DCF9601EC0B20F2800F20F
:1022A000938041F2B855C2F2010540F0C004A86C19
:1022B000036821461B689847A86C036807F07F07EE
:1022C0001B683946984743F60C000F21C0F2020004
:1022D0001CF0BEF941F6DC7CC2F2010C4FF00108A3
:1022E000DCF848301A699E46511C196114705EF87A
:1022F000101F714524BF1B6119464FF000095A6930
:102300008A4202F1010014D0586114785A6B864554
:102310004FEA241698BF5B619D18501C002A3FD1DC
:102320005A6983F830608A42C3F8348002F10100B0
:10233000EAD1DCF848301A699E46511C19611770C1
:102340005EF8106F764524BF1B611E4601274FF0D3
:10235000000C5A69964202F1010112D059611078BD
:102360005A6B8E454FEA201598BF5B619C18511C33
:1023700002BB5A6983F8305096425F6302F1010153
:10238000ECD143F61C00C0F202000F211CF060F9F2
:102390004EF2C000C2F20000BDE8F84319F0D2BB13
:1023A000032885F830405863A9D1C3F83090C3F8AA
:1023B0003490A4E7032984F830005963C9D1C3F8E5
:1023C00030C0C3F834C0C4E743F60C000F21C0F29C
:1023D00002001CF03DF9D4E71F292DE9F8430D4612
:1023E000044608D840F26853C2F2010318780EF090
:1023F00043F909F0BDFF43F6B0300D21C0F20200F1
:102400001CF026F92B04013C03F4FE03210243F4E3
:10241000404343F00C0301F4706141F20070194332
:10242000C2F2010017F0F8FE43F6F400C0F2020019
:102430001421E4B21CF00CF90F2C5BD841F6DC7EC1
:10244000C2F2010E64F03F04DEF848301A699C467F
:10245000511C196114705CF8107F674505F07F0806
:1024600024BF1B611F4601254FF000095A6997429E
:1024700002F1010113D0596110785A6B8C454FEA73
:10248000201698BF5B619C18511C002A41D15A69E3
:1024900083F8306097425D6302F10101EBD1DEF811
:1024A00048301A691F46511C196182F8008057F89C
:1024B000106FBE4224BF1B611E464FF0010E4FF04D
:1024C000000C5A69964202F1010113D0596110784B
:1024D0005A6B8F424FEA201598BF5B619C18511CC4
:1024E0000ABB5A6983F830509642C3F834E002F1CF
:1024F0000101EBD143F61C00C0F202000F211CF0D9
:10250000A7F84EF2C000C2F20000BDE8F84319F08F
:1025100019BB032984F830005963A7D1C3F8309060
:10252000C3F83490A2E7032984F830005963C8D176
:10253000C3F830C0C3F834C0C3E700BF4AF28853C1
:10254000C2F2010310B4D3F8C020136850681978A0
:102550000478507A137A044201EA03011AD0937A7C
:1025600003F0030309B143F0040343F00803991097
:10257000082B91722AD8072B22D2032B2ED011D9E7
:10258000042B13D0062B14D1D3685DF8044B023B07
:10259000D3607047937A03F003030029E7D043F038
:1025A0000403E4E7012B0BD0022B02D1D368013BDB
:1025B000D3605DF8044B70470D2BF7D00E2BF8D18C
:1025C000D3685DF8044B0133D36070470C2B05D002
:1025D000F2D8092BD8D00B2BE8D0EAE7D3685DF806
:1025E000044B0233D36070474AF28853C2F20103AE
:1025F00010B4D3F8C4201368506819780478507A5E
:10260000137A044201EA03011AD0937A03F0030318
:1026100009B143F0040343F008039910082B9172A9
:102620002AD8072B22D2032B2ED011D9042B13D05A
:10263000062B14D1D3685DF8044B023BD36070477E
:10264000937A03F003030029E7D043F00403E4E79F
:10265000012B0BD0022B02D1D368013BD3605DF874
:10266000044B70470D2BF7D00E2BF8D1D3685DF8D3
:10267000044B0133D36070470C2B05D0F2D8092BE3
:10268000D8D00B2BE8D0EAE7D3685DF8044B0233CF
:10269000D36070474AF28853C2F2010310B4D3F8F2
:1026A000C8201368506819780478507A137A044265
:1026B00001EA03011AD0937A03F0030309B143F04E
:1026C000040343F008039910082B91722AD8072BB2
:1026D00022D2032B2ED011D9042B13D0062B14D1C8
:1026E000D3685DF8044B023BD3607047937A03F0E4
:1026F00003030029E7D043F00403E4E7012B0BD0E8
:10270000022B02D1D368013BD3605DF8044B7047C4
:102710000D2BF7D00E2BF8D1D3685DF8044B0133A5
:10272000D36070470C2B05D0F2D8092BD8D00B2BD7
:10273000E8D0EAE7D3685DF8044B0233D360704712
:102740004AF28853C2F2010310B4D3F8CC201368C4
:10275000506819780478507A137A044201EA030128
:102760001AD0937A03F0030309B143F0040343F052
:1027700008039910082B91722AD8072B22D2032B19
:102780002ED011D9042B13D0062B14D1D3685DF8A9
:10279000044B023BD3607047937A03F00303002994
:1027A000E7D043F00403E4E7012B0BD0022B02D166
:1027B000D368013BD3605DF8044B70470D2BF7D015
:1027C0000E2BF8D1D3685DF8044B0133D36070470A
:1027D0000C2B05D0F2D8092BD8D00B2BE8D0EAE788
:1027E000D3685DF8044B0233D36070474AF28853D4
:1027F000C2F2010310B4D3F8D020136850681978DE
:102800000478507A137A044201EA03011AD0937AC9
:1028100003F0030309B143F0040343F008039910E4
:10282000082B91722AD8072B22D2032B2ED011D934
:10283000042B13D0062B14D1D3685DF8044B023B54
:10284000D3607047937A03F003030029E7D043F085
:102850000403E4E7012B0BD0022B02D1D368013B28
:10286000D3605DF8044B70470D2BF7D00E2BF8D1D9
:10287000D3685DF8044B0133D36070470C2B05D04F
:10288000F2D8092BD8D00B2BE8D0EAE7D3685DF853
:10289000044B0233D36070474AF28853C2F20103FB
:1028A00010B4D3F8D4201368506819780478507A9B
:1028B000137A044201EA03011AD0937A03F0030366
:1028C00009B143F0040343F008039910082B9172F7
:1028D0002AD8072B22D2032B2ED011D9042B13D0A8
:1028E000062B14D1D3685DF8044B023BD3607047CC
:1028F000937A03F003030029E7D043F00403E4E7ED
:10290000012B0BD0022B02D1D368013BD3605DF8C1
:10291000044B70470D2BF7D00E2BF8D1D3685DF820
:10292000044B0133D36070470C2B05D0F2D8092B30
:10293000D8D00B2BE8D0EAE7D3685DF8044B02331C
:10294000D36070474AF28853C2F2010310B4D3F83F
:10295000D8201368506819780478507A137A0442A2
:1029600001EA03011AD0937A03F0030309B143F09B
:10297000040343F008039910082B91722AD8072BFF
:1029800022D2032B2ED011D9042B13D0062B14D115
:10299000D3685DF8044B023BD3607047937A03F031
:1029A00003030029E7D043F00403E4E7012B0BD035
:1029B000022B02D1D368013BD3605DF8044B704712
:1029C0000D2BF7D00E2BF8D1D3685DF8044B0133F3
:1029D000D36070470C2B05D0F2D8092BD8D00B2B25
:1029E000E8D0EAE7D3685DF8044B0233D360704760
:1029F0004AF28853C2F2010310B4D3F8DC20136802
:102A0000506819780478507A137A044201EA030175
:102A10001AD0937A03F0030309B143F0040343F09F
:102A200008039910082B91722AD8072B22D2032B66
:102A30002ED011D9042B13D0062B14D1D3685DF8F6
:102A4000044B023BD3607047937A03F003030029E1
:102A5000E7D043F00403E4E7012B0BD0022B02D1B3
:102A6000D368013BD3605DF8044B70470D2BF7D062
:102A70000E2BF8D1D3685DF8044B0133D360704757
:102A80000C2B05D0F2D8092BD8D00B2BE8D0EAE7D5
:102A9000D3685DF8044B0233D36070474AF2885321
:102AA000C2F2010310B4D3F880201368506819787B
:102AB0000478507A137A044201EA03011AD0937A17
:102AC00003F0030309B143F0040343F00803991032
:102AD000082B91722AD8072B22D2032B2ED011D982
:102AE000042B13D0062B14D1D3685DF8044B023BA2
:102AF000D3607047937A03F003030029E7D043F0D3
:102B00000403E4E7012B0BD0022B02D1D368013B75
:102B1000D3605DF8044B70470D2BF7D00E2BF8D126
:102B2000D3685DF8044B0133D36070470C2B05D09C
:102B3000F2D8092BD8D00B2BE8D0EAE7D3685DF8A0
:102B4000044B0233D36070474AF28853C2F2010348
:102B500010B4D3F884201368506819780478507A38
:102B6000137A044201EA03011AD0937A03F00303B3
:102B700009B143F0040343F008039910082B917244
:102B80002AD8072B22D2032B2ED011D9042B13D0F5
:102B9000062B14D1D3685DF8044B023BD360704719
:102BA000937A03F003030029E7D043F00403E4E73A
:102BB000012B0BD0022B02D1D368013BD3605DF80F
:102BC000044B70470D2BF7D00E2BF8D1D3685DF86E
:102BD000044B0133D36070470C2B05D0F2D8092B7E
:102BE000D8D00B2BE8D0EAE7D3685DF8044B02336A
:102BF000D36070474AF28853C2F2010310B4D3F88D
:102C000088201368506819780478507A137A04423F
:102C100001EA03011AD0937A03F0030309B143F0E8
:102C2000040343F008039910082B91722AD8072B4C
:102C300022D2032B2ED011D9042B13D0062B14D162
:102C4000D3685DF8044B023BD3607047937A03F07E
:102C500003030029E7D043F00403E4E7012B0BD082
:102C6000022B02D1D368013BD3605DF8044B70475F
:102C70000D2BF7D00E2BF8D1D3685DF8044B013340
:102C8000D36070470C2B05D0F2D8092BD8D00B2B72
:102C9000E8D0EAE7D3685DF8044B0233D3607047AD
:102CA0004AF28853C2F2010310B4D3F88C2013689F
:102CB000506819780478507A137A044201EA0301C3
:102CC0001AD0937A03F0030309B143F0040343F0ED
:102CD00008039910082B91722AD8072B22D2032BB4
:102CE0002ED011D9042B13D0062B14D1D3685DF844
:102CF000044B023BD3607047937A03F0030300292F
:102D0000E7D043F00403E4E7012B0BD0022B02D100
:102D1000D368013BD3605DF8044B70470D2BF7D0AF
:102D20000E2BF8D1D3685DF8044B0133D3607047A4
:102D30000C2B05D0F2D8092BD8D00B2BE8D0EAE722
:102D4000D3685DF8044B0233D36070474AF288536E
:102D5000C2F2010310B4D3F89020136850681978B8
:102D60000478507A137A044201EA03011AD0937A64
:102D700003F0030309B143F0040343F0080399107F
:102D8000082B91722AD8072B22D2032B2ED011D9CF
:102D9000042B13D0062B14D1D3685DF8044B023BEF
:102DA000D3607047937A03F003030029E7D043F020
:102DB0000403E4E7012B0BD0022B02D1D368013BC3
:102DC000D3605DF8044B70470D2BF7D00E2BF8D174
:102DD000D3685DF8044B0133D36070470C2B05D0EA
:102DE000F2D8092BD8D00B2BE8D0EAE7D3685DF8EE
:102DF000044B0233D36070474AF28853C2F2010396
:102E000010B4D3F894201368506819780478507A75
:102E1000137A044201EA03011AD0937A03F0030300
:102E200009B143F0040343F008039910082B917291
:102E30002AD8072B22D2032B2ED011D9042B13D042
:102E4000062B14D1D3685DF8044B023BD360704766
:102E5000937A03F003030029E7D043F00403E4E787
:102E6000012B0BD0022B02D1D368013BD3605DF85C
:102E7000044B70470D2BF7D00E2BF8D1D3685DF8BB
:102E8000044B0133D36070470C2B05D0F2D8092BCB
:102E9000D8D00B2BE8D0EAE7D3685DF8044B0233B7
:102EA000D36070474AF28853C2F2010310B4D3F8DA
:102EB00098201368506819780478507A137A04427D
:102EC00001EA03011AD0937A03F0030309B143F036
:102ED000040343F008039910082B91722AD8072B9A
:102EE00022D2032B2ED011D9042B13D0062B14D1B0
:102EF000D3685DF8044B023BD3607047937A03F0CC
:102F000003030029E7D043F00403E4E7012B0BD0CF
:102F1000022B02D1D368013BD3605DF8044B7047AC
:102F20000D2BF7D00E2BF8D1D3685DF8044B01338D
:102F3000D36070470C2B05D0F2D8092BD8D00B2BBF
:102F4000E8D0EAE7D3685DF8044B0233D3607047FA
:102F50004AF28853C2F2010310B4D3F89C201368DC
:102F6000506819780478507A137A044201EA030110
:102F70001AD0937A03F0030309B143F0040343F03A
:102F800008039910082B91722AD8072B22D2032B01
:102F90002ED011D9042B13D0062B14D1D3685DF891
:102FA000044B023BD3607047937A03F0030300297C
:102FB000E7D043F00403E4E7012B0BD0022B02D14E
:102FC000D368013BD3605DF8044B70470D2BF7D0FD
:102FD0000E2BF8D1D3685DF8044B0133D3607047F2
:102FE0000C2B05D0F2D8092BD8D00B2BE8D0EAE770
:102FF000D3685DF8044B0233D36070474AF28853BC
:10300000C2F2010310B4D3F8A020136850681978F5
:103010000478507A137A044201EA03011AD0937AB1
:1030200003F0030309B143F0040343F008039910CC
:10303000082B91722AD8072B22D2032B2ED011D91C
:10304000042B13D0062B14D1D3685DF8044B023B3C
:10305000D3607047937A03F003030029E7D043F06D
:103060000403E4E7012B0BD0022B02D1D368013B10
:10307000D3605DF8044B70470D2BF7D00E2BF8D1C1
:10308000D3685DF8044B0133D36070470C2B05D037
:10309000F2D8092BD8D00B2BE8D0EAE7D3685DF83B
:1030A000044B0233D36070474AF28853C2F20103E3
:1030B00010B4D3F8A4201368506819780478507AB3
:1030C000137A044201EA03011AD0937A03F003034E
:1030D00009B143F0040343F008039910082B9172DF
:1030E0002AD8072B22D2032B2ED011D9042B13D090
:1030F000062B14D1D3685DF8044B023BD3607047B4
:10310000937A03F003030029E7D043F00403E4E7D4
:10311000012B0BD0022B02D1D368013BD3605DF8A9
:10312000044B70470D2BF7D00E2BF8D1D3685DF808
:10313000044B0133D36070470C2B05D0F2D8092B18
:10314000D8D00B2BE8D0EAE7D3685DF8044B023304
:10315000D36070474AF28853C2F2010310B4D3F827
:10316000A8201368506819780478507A137A0442BA
:1031700001EA03011AD0937A03F0030309B143F083
:10318000040343F008039910082B91722AD8072BE7
:1031900022D2032B2ED011D9042B13D0062B14D1FD
:1031A000D3685DF8044B023BD3607047937A03F019
:1031B00003030029E7D043F00403E4E7012B0BD01D
:1031C000022B02D1D368013BD3605DF8044B7047FA
:1031D0000D2BF7D00E2BF8D1D3685DF8044B0133DB
:1031E000D36070470C2B05D0F2D8092BD8D00B2B0D
:1031F000E8D0EAE7D3685DF8044B0233D360704748
:103200004AF28853C2F2010310B4D3F8AC20136819
:10321000506819780478507A137A044201EA03015D
:103220001AD0937A03F0030309B143F0040343F087
:1032300008039910082B91722AD8072B22D2032B4E
:103240002ED011D9042B13D0062B14D1D3685DF8DE
:10325000044B023BD3607047937A03F003030029C9
:10326000E7D043F00403E4E7012B0BD0022B02D19B
:10327000D368013BD3605DF8044B70470D2BF7D04A
:103280000E2BF8D1D3685DF8044B0133D36070473F
:103290000C2B05D0F2D8092BD8D00B2BE8D0EAE7BD
:1032A000D3685DF8044B0233D36070474AF2885309
:1032B000C2F2010310B4D3F8B02013685068197833
:1032C0000478507A137A044201EA03011AD0937AFF
:1032D00003F0030309B143F0040343F0080399101A
:1032E000082B91722AD8072B22D2032B2ED011D96A
:1032F000042B13D0062B14D1D3685DF8044B023B8A
:10330000D3607047937A03F003030029E7D043F0BA
:103310000403E4E7012B0BD0022B02D1D368013B5D
:10332000D3605DF8044B70470D2BF7D00E2BF8D10E
:10333000D3685DF8044B0133D36070470C2B05D084
:10334000F2D8092BD8D00B2BE8D0EAE7D3685DF888
:10335000044B0233D36070474AF28853C2F2010330
:1033600010B4D3F8B4201368506819780478507AF0
:10337000137A044201EA03011AD0937A03F003039B
:1033800009B143F0040343F008039910082B91722C
:103390002AD8072B22D2032B2ED011D9042B13D0DD
:1033A000062B14D1D3685DF8044B023BD360704701
:1033B000937A03F003030029E7D043F00403E4E722
:1033C000012B0BD0022B02D1D368013BD3605DF8F7
:1033D000044B70470D2BF7D00E2BF8D1D3685DF856
:1033E000044B0133D36070470C2B05D0F2D8092B66
:1033F000D8D00B2BE8D0EAE7D3685DF8044B023352
:10340000D36070474AF28853C2F2010310B4D3F874
:10341000B8201368506819780478507A137A0442F7
:1034200001EA03011AD0937A03F0030309B143F0D0
:10343000040343F008039910082B91722AD8072B34
:1034400022D2032B2ED011D9042B13D0062B14D14A
:10345000D3685DF8044B023BD3607047937A03F066
:1034600003030029E7D043F00403E4E7012B0BD06A
:10347000022B02D1D368013BD3605DF8044B704747
:103480000D2BF7D00E2BF8D1D3685DF8044B013328
:10349000D36070470C2B05D0F2D8092BD8D00B2B5A
:1034A000E8D0EAE7D3685DF8044B0233D360704795
:1034B0004AF28853C2F2010310B4D3F8BC20136857
:1034C000506819780478507A137A044201EA0301AB
:1034D0001AD0937A03F0030309B143F0040343F0D5
:1034E00008039910082B91722AD8072B22D2032B9C
:1034F0002ED011D9042B13D0062B14D1D3685DF82C
:10350000044B023BD3607047937A03F00303002916
:10351000E7D043F00403E4E7012B0BD0022B02D1E8
:10352000D368013BD3605DF8044B70470D2BF7D097
:103530000E2BF8D1D3685DF8044B0133D36070478C
:103540000C2B05D0F2D8092BD8D00B2BE8D0EAE70A
:10355000D3685DF8044B0233D36070474AF2885356
:10356000C2F2010310B4D3F8E02013685068197850
:103570000478507A137A044201EA03011AD0937A4C
:1035800003F0030309B143F0040343F00803991067
:10359000082B91722AD8072B22D2032B2ED011D9B7
:1035A000042B13D0062B14D1D3685DF8044B023BD7
:1035B000D3607047937A03F003030029E7D043F008
:1035C0000403E4E7012B0BD0022B02D1D368013BAB
:1035D000D3605DF8044B70470D2BF7D00E2BF8D15C
:1035E000D3685DF8044B0133D36070470C2B05D0D2
:1035F000F2D8092BD8D00B2BE8D0EAE7D3685DF8D6
:10360000044B0233D360704710B443F2907400232C
:10361000C0F202044172026104600372C36041B1EE
:10362000194600E0026942F82310427A01339A42B7
:10363000F8DC4AF28863C2F201031A680AB90CE0A6
:103640001A465369002BFBD15061002343618380EC
:10365000C38083725DF8044B70471860F5E700BFC4
:103660002DE9F84341F2B854C2F2010447F61221A1
:10367000A06C0368DB69984747F6A905032047F665
:10368000112747F6713143F6B53247F6C14384F846
:103690006400C0F20005C0F20007C0F20001C0F2F1
:1036A0000002C0F2000342F2D93065602760E16099
:1036B0006261A361C0F2000044F6E53541F2E547DE
:1036C00047F6056140F6496241F2AD732061C0F2F0
:1036D0000005C0F20007C0F20001C0F20002C0F213
:1036E000000341F67140E5612762A160A262E362D6
:1036F000C0F2000041F27D2541F2393741F2C1119B
:1037000041F2051241F2F533C0F20002C0F20003AB
:103710002063C0F20005C0F20007C0F200014EF2C3
:10372000C00643F6C03022646364C2F200066563DB
:10373000A76300254FF6FF77E163C0F2020017216F
:1037400084F84C5084F84E5084F84D50A56565655A
:1037500084F8E95084F8665084F8655084F867501E
:1037600084F86850E76527661AF072FF304618F053
:10377000E9F914F035FF41F20073C2F2010347F694
:10378000591247F6BD20C0F20002C0F2000047F611
:103790001541C3F85423C3F85003C0F2000143F6A7
:1037A000195447F6655242F26D20C3F85C13C0F21B
:1037B0000004C0F20002C0F2000044F69551C3F8C4
:1037C0006443C3F86823C3F86003C0F2000141F604
:1037D0000D7447F6896242F24500C3F87013C0F2D7
:1037E0000004C0F20002C0F2000041F64D61C3F8CF
:1037F0007443C3F85823C3F87C03C0F2000141F6B8
:103800005D5440F6354240F6B520C3F88013C0F24F
:103810000004C0F20002C0F2000040F67531C3F8A7
:103820008443C3F88823C3F88C03C0F2000140F638
:10383000F51440F6F54243F6D830C0F20002C3F862
:103840009013C0F200041D21C0F20200C3F894439B
:10385000C3F898231AF0FCFE304618F073F941F6CD
:10386000DC73C2F2010341F689209A6C02F118015F
:10387000156095615560D5619560D560156255629A
:1038800012615261D1629162C0F2000043F61534B8
:1038900041F631124FF001095860C0F20004C0F245
:1038A000000241F6E91083F84E5083F84D509D65B3
:1038B0005D65DF651F6683F8E95083F8665083F81D
:1038C000655083F8675083F868505C619A6109FA23
:1038D00009F8C0F2000041F6690C45F6E10E44F625
:1038E000593142F2F51741F20D7542F27D1441F261
:1038F0001D621861C0F2000E48EA0908C0F2000C0F
:10390000C0F20001C0F20007C0F20005C0F20004DE
:10391000C0F2000241F6E13083F84C9083F86480F5
:10392000C3F800C0C3F80CE0C0F20000D9611F6208
:103930009D609C62DA6240F6857140F6E57741F25F
:10394000450541F2A50441F27D621863C0F2000111
:10395000C0F20007C0F20005C0F20004C0F200028D
:1039600043F6F83059639F63DD631C645A64C0F208
:10397000020018211AF06CFE3046BDE8F84318F03A
:10398000E1B800BF4DF20A73C3F6234306EE103AC6
:10399000437EC17E07EE103A837CB8EEC77A07EE0D
:1039A000903A70B4F8EEE76A27EE067A83B067EED5
:1039B000267A0022FCEEE77A8273CDED017A42731B
:1039C0009DF80430027301B10373827E02B1437328
:1039D000027F02B1837390F8213090F8231007EE34
:1039E000103A4DF20A73C3F6234306EE103A037CF5
:1039F000B8EEC77A07EE903A27EE067AF8EEE76A55
:103A000067EE267AFCEEE77ACDED017A9DF8043078
:103A100021B1017B994238BF1946017390F82210F9
:103A200021B1417B994238BF1946417390F8244037
:103A300024B1817B8B4238BF0B468373437FC17FA8
:103A400007EE103A4DF20A73C3F6234306EE103A1E
:103A5000437CB8EEC77A07EE903A27EE067AF8EE86
:103A6000E76A67EE267AFCEEE77ACDED017A9DF8FB
:103A7000043021B1017B994238BF19460173817F1F
:103A800021B1417B994238BF1946417390F820100B
:103A900021B1857BAB4238BF2B46837390F825302C
:103AA00090F8275007EE103A4DF20A73C3F62343FD
:103AB00006EE103AC37BB8EEC77A07EE903A27EECF
:103AC000067AF8EEE76A67EE267AFCEEE77ACDED45
:103AD000017A9DF8043025B1057B9D4238BF1D4613
:103AE000057390F8265025B1457B9D4238BF1D4691
:103AF000457390F8285025B1867BB34238BF3346D2
:103B0000837322B919B914B90DB97F23837303B034
:103B100070BC704741F2E463C2F2010370B51B68E8
:103B2000054683F8CF1003F1C0000C46FFF72AFFCB
:103B300043F614400D21013DC0F202001AF088FD49
:103B4000E9B20F290FD841F2B856C2F2010641F08E
:103B5000D001B06C03681B689847B06C036804F030
:103B60007F011B68984743F60C000F21C0F202004A
:103B70001AF06EFD230403F4FE03290243F45043BC
:103B800043F00D0301F4706141F200701943C2F279
:103B9000010016F041FB43F6F400C0F202001421CC
:103BA0001AF056FD4EF2C000C2F20000BDE87040AF
:103BB00017F0C8BF2DE9F84341F2E463C2F20103F4
:103BC00004461B6883F8CF1003F1C0000D46FFF7D1
:103BD000D9FE43F624400D21C0F202001AF038FD50
:103BE0002B04013C03F4FE03210243F4504343F051
:103BF0000D0301F4706141F200701943C2F201003B
:103C000016F00AFB43F6F400C0F202001421E4B2FD
:103C10001AF01EFD0F2C5BD841F6DC7EC2F2010EBD
:103C200064F02F04DEF848301A699C46511C196173
:103C300014705CF8107F674505F07F0824BF1B6196
:103C40001F4601254FF000095A69974202F1010011
:103C500013D0586114785A6B84454FEA241698BFE4
:103C60005B619918501C002A41D15A6983F8306071
:103C700097425D6302F10100EBD1DEF848301A692A
:103C80001F46511C196182F8008057F8106FBE4220
:103C900024BF1B611E464FF0010E4FF0000C5A6905
:103CA000964202F1010113D0596110785A6B8F428C
:103CB0004FEA201598BF5B619C18511C0ABB5A69DA
:103CC00083F830509642C3F834E002F10101EBD1A1
:103CD00043F61C00C0F202000F211AF0B9FC4EF2AC
:103CE000C000C2F20000BDE8F84317F02BBF032864
:103CF00081F830405863A7D1C3F83090C3F83490AE
:103D0000A2E7032984F830005963C8D1C3F830C052
:103D1000C3F834C0C3E700BF2DE9F84341F2E463C0
:103D2000C2F2010304461B6883F8CF1003F1C00000
:103D30000F46FFF727FE43F63440C0F2020012217F
:103D40001AF086FC601EC0B20F2800F2938041F288
:103D5000B855C2F2010540F0D004A86C03682146B2
:103D60001B689847A86C036807F07F071B683946F3
:103D7000984743F60C000F21C0F202001AF068FCCD
:103D800041F6DC7CC2F2010C4FF00108DCF848304F
:103D90001A699E46511C196114705EF8101F714516
:103DA00024BF1B6119464FF000095A69914202F184
:103DB000010014D0586114785A6B86454FEA2416D6
:103DC00098BF5B619D18501C002A3FD15A6983F847
:103DD00030609142C3F8348002F10100EAD1DCF88E
:103DE00048301A699E46511C196117705EF8106FB1
:103DF000764524BF1B611E4601274FF0000C5A690F
:103E0000964202F1010112D0596110785A6B8E4529
:103E10004FEA201598BF5B619C18511C02BB5A6980
:103E200083F8305096425F6302F10101ECD143F612
:103E30001C00C0F202000F211AF00AFC4EF2C00072
:103E4000C2F20000BDE8F84317F07CBE032885F8F5
:103E500030405863A9D1C3F83090C3F83490A4E738
:103E6000032984F830005963C9D1C3F830C0C3F8BE
:103E700034C0C4E743F60C000F21C0F202001AF070
:103E8000E7FBD4E710B4036841681A780C78417AEC
:103E9000037A0C4202EA03021AD0837A03F0030386
:103EA0000AB143F0040343F008039A10082B82720E
:103EB0002AD8072B22D2032B2ED011D9042B13D0B2
:103EC000062B14D1C3685DF8044B023BC3607047F6
:103ED000837A03F00303002AE7D043F00403E4E706
:103EE000012B0BD0022B02D1C368013BC3605DF8EC
:103EF000044B70470D2BF7D00E2BF8D1C3685DF83B
:103F0000044B0133C36070470C2B05D0F2D8092B4A
:103F1000D8D00B2BE8D0EAE7C3685DF8044B023336
:103F2000C360704708B54AF28853C2F20103D3F860
:103F3000EC00FFF7A7FF08BD08B54AF28853C2F2AC
:103F40000103D3F8E800FFF79DFF08BD08B54AF26A
:103F50008853C2F20103D3F8E400FFF793FF08BDD2
:103F600008B54AF28853C2F20103D86FFFF78AFFFF
:103F700008BD00BF08B54AF28853C2F20103986F2A
:103F8000FFF780FF08BD00BF08B54AF28853C2F2B0
:103F90000103586FFFF776FF08BD00BF08B54AF26E
:103FA0008853C2F20103186FFFF76CFF08BD00BF12
:103FB00008B54AF28853C2F20103D86EFFF762FFD8
:103FC00008BD00BF08B54AF28853C2F20103986EDB
:103FD000FFF758FF08BD00BF08B54AF28853C2F288
:103FE0000103586EFFF74EFF08BD00BF08B54AF247
:103FF0008853C2F20103186EFFF744FF08BD00BFEB
:1040000008B54AF28853C2F20103D86DFFF73AFFB0
:1040100008BD00BF08B54AF28853C2F20103986D8B
:10402000FFF730FF08BD00BF08B54AF28853C2F25F
:104030000103586DFFF726FF08BD00BF08B54AF21F
:104040008853C2F20103186DFFF71CFF08BD00BFC3
:1040500008B54AF28853C2F20103D86CFFF712FF89
:1040600008BD00BF08B54AF28853C2F20103986C3C
:10407000FFF708FF08BD00BF08B54AF28853C2F237
:104080000103586CFFF7FEFE08BD00BF08B54AF2F9
:104090008853C2F20103186CFFF7F4FE08BD00BF9D
:1040A00008B54AF28853C2F20103D86BFFF7EAFE63
:1040B00008BD00BF08B54AF28853C2F20103986BED
:1040C000FFF7E0FE08BD00BF08B54AF28853C2F210
:1040D0000103586BFFF7D6FE08BD00BF08B54AF2D2
:1040E0008853C2F20103186BFFF7CCFE08BD00BF76
:1040F00008B54AF28853C2F20103D86AFFF7C2FE3C
:1041000008BD00BF08B54AF28853C2F20103986A9D
:10411000FFF7B8FE08BD00BF08B54AF28853C2F2E7
:104120000103586AFFF7AEFE08BD00BF08B54AF2AA
:104130008853C2F20103186AFFF7A4FE08BD00BF4E
:1041400008B54AF28853C2F20103D869FFF79AFE14
:1041500008BD00BF08B54AF28853C2F2010398694E
:10416000FFF790FE08BD00BF08B54AF28853C2F2BF
:1041700001035869FFF786FE08BD00BF08B54AF283
:104180008853C2F201031869FFF77CFE08BD00BF27
:1041900008B54AF28853C2F20103D868FFF772FEED
:1041A00008BD00BF08B54AF28853C2F201039868FF
:1041B000FFF768FE08BD00BF08B54AF28853C2F297
:1041C00001035868FFF75EFE08BD00BF08B54AF25C
:1041D0008853C2F201031868FFF754FE08BD00BF00
:1041E0001D2810B50B4600F0E983024622D92C2881
:1041F00000F064813FD8242800F0EE8340F2A880CC
:10420000282800F0748300F2D680262800F0F5817B
:1042100040F2D5824AF28854C2F2010442F651714A
:10422000C0F2000104222720C4F89C3018F0F6F9EF
:10423000012010BD0E2800F097833AD8062800F020
:10424000A1836CD90A2800F0058300F207810828B1
:1042500000F07E8140F275824AF28854C2F2010475
:1042600044F21911C0F2000104220920636218F01F
:10427000D5F9012010BD342800F0BD8336D8302890
:1042800000F0638300F2D6802E2800F0528140F2C5
:1042900001824AF28854C2F2010443F2B141C0F2F1
:1042A000000104222F20C4F8BC3018F0B7F9012017
:1042B00010BD152800F0748364D9192800F0FA8124
:1042C00000F2A580172800F08A8140F2D1824AF2DC
:1042D0008854C2F2010443F6ED71C0F200010422D9
:1042E0001820236618F09AF9012010BD382800F034
:1042F000CE8275D8362800F0398140F27F824AF2AA
:104300008854C2F2010442F6F111C0F20001042205
:104310003720C4F8DC3018F081F9012010BD0228E4
:1043200000F0018240F27881042800F04B8140F2D5
:10433000BD824AF28854C2F2010444F26911C0F20B
:10434000000104220520636118F068F9012010BD06
:10435000202800F0448240F28981222800F0238145
:1043600040F2D4824AF28854C2F2010442F6A141DA
:10437000C0F2000104222320C4F88C3018F04EF95A
:10438000012010BD112800F0B18140F25A8113289C
:1043900000F0FB8040F2B8814AF28854C2F2010476
:1043A00044F23D01C0F2000104221420236518F0FC
:1043B00035F9012010BD2A2800F0AC8040F2E081E0
:1043C0004AF28854C2F2010443F20121C0F2000112
:1043D00004222B20C4F8AC3018F020F9012010BDC5
:1043E0003A2800F08880C0F072823B2840F06D824D
:1043F0004AF28854C2F2010443F62571C0F200016A
:104400000422C4F8EC3018F009F9012010BD1B2873
:1044100063D040F28B824AF28854C2F2010443F620
:104420009D71C0F2000104221C20236718F0F6F8E9
:10443000012010BD322824D040F292814AF28854E3
:10444000C2F2010442F24171C0F2000104223320A1
:10445000C4F8CC3018F0E2F8012010BD0C281FD0B1
:1044600040F29E814AF28854C2F2010444F2C9012A
:10447000C0F2000104220D20636318F0CFF8012080
:1044800010BD4AF28854C2F2010442F29561C0F2B2
:1044900000010422C4F8C83018F0C0F8012010BD93
:1044A0004AF28854C2F2010444F2DD01C0F2000174
:1044B0000422236318F0B2F8012010BD4AF2885498
:1044C000C2F2010443F2AD21C0F200010422C4F89B
:1044D000B03018F0A3F8012010BD4AF28854C2F29F
:1044E000010443F6B171C0F200010422E36618F042
:1044F00095F8012010BD4AF28854C2F2010443F637
:104500003971C0F200010422C4F8E83018F086F8CE
:10451000012010BD4AF28854C2F2010443F2551141
:10452000C0F200010422C4F8A83018F077F8012086
:1045300010BD4AF28854C2F2010443F20541C0F2B0
:1045400000010422C4F8B83018F068F8012010BD4A
:104550004AF28854C2F2010444F22D11C0F2000163
:104560000422236218F05AF8012010BD4AF2885440
:10457000C2F2010442F64511C0F200010422C4F85F
:10458000D83018F04BF8012010BD4AF28854C2F21E
:10459000010444F25101C0F200010422E36418F066
:1045A0003DF8012010BD4AF28854C2F2010442F6DF
:1045B000F531C0F200010422C4F8883018F02EF85A
:1045C000012010BD4AF28854C2F2010444F27D1168
:1045D000C0F20001236118F021F8012010BD4AF259
:1045E0008854C2F2010444F20101C0F20001042225
:1045F000E36518F013F8012010BD4AF28854C2F2A6
:10460000010442F6A561C0F200010422C4F898300A
:1046100018F004F8012010BD002800F0FF800128E8
:1046200040F053814AF28854C2F2010444F2B911B5
:10463000C0F2000104220120636017F0EFFF0120A7
:1046400010BD0F2800F0F880102840F03E814AF29B
:104650008854C2F2010444F28D01C0F20001042228
:104660001020236417F0DAFF012010BD1E282FD080
:104670001F2840F02A814AF28854C2F2010443F60E
:104680006171C0F2000104221F20E36717F0C6FF2A
:10469000012010BD4AF28854C2F2010443F259319C
:1046A000C0F2000104222D20C4F8B43017F0B6FF88
:1046B000012010BD4AF28854C2F2010443F6D971B8
:1046C000C0F200010422636617F0A8FF012010BDAC
:1046D0004AF28854C2F2010443F67571C0F2000137
:1046E0000422A36717F09AFF012010BD4AF28854F4
:1046F000C2F2010444F27901C0F2000104226364B1
:1047000017F08CFF012010BD4AF28854C2F2010458
:1047100044F26501C0F2000104221220A36417F0E4
:104720007DFF012010BD4AF28854C2F2010444F218
:10473000A511C0F200010422A36017F06FFF012051
:1047400010BD4AF28854C2F2010444F24111C0F291
:10475000000104220720E36117F060FF012010BD73
:104760004AF28854C2F2010442F2E951C0F2000157
:1047700004223120C4F8C43017F050FF012010BDCE
:104780004AF28854C2F2010443F2A901C0F20001C6
:1047900004222920C4F8A43017F040FF012010BDE6
:1047A0004AF28854C2F2010444F2F101C0F200015D
:1047B00004220B20E36217F031FF012010BD4AF202
:1047C0008854C2F2010442F6F951C0F200010422F9
:1047D0002520C4F8943017F021FF012010BD4AF2C3
:1047E0008854C2F2010442F69D21C0F20001042265
:1047F000C4F8803017F012FF012010BD4AF288542F
:10480000C2F2010442F69901C0F2000104223520EF
:10481000C4F8D43017F002FF012010BD4AF28854CA
:10482000C2F2010444F2CD11C0F20001042223605F
:1048300017F0F4FE012010BD4AF28854C2F20104C0
:1048400044F2A101C0F200010422E36317F0E6FE86
:10485000012010BD4AF28854C2F2010444F205114D
:10486000C0F200010422A36217F0D8FE012010BD9F
:104870004AF28854C2F2010444F21501C0F2000168
:1048800004221620A36517F0C9FE012010BD4AF2CC
:104890008854C2F2010443F25D51C0F200010422C7
:1048A000C4F8E03017F0BAFE012010BD4AF2885477
:1048B000C2F2010444F29111C0F20001042203206B
:1048C000E36017F0ABFE012010BD002010BD4AF2DE
:1048D0008854C2F2010443F64D71C0F20001042273
:1048E0003920C4F8E43017F099FE012010BD4AF2D7
:1048F0008854C2F2010442F6FD71C0F200010422A4
:10490000C4F8A03017F08AFE012010BD4AF2885486
:10491000C2F2010442F64931C0F200010422212012
:10492000C4F8843017F07AFE012010BD4AF2885492
:10493000C2F2010443F6C571C0F2000104221A203C
:10494000A36617F06BFE012010BD4AF28854C2F234
:10495000010442F23D51C0F200010422C4F8C0300B
:1049600017F05CFE012010BD4AF28854C2F2010427
:1049700044F2B501C0F200010422A36317F04EFE19
:10498000012010BD4AF28854C2F2010444F25511CC
:10499000C0F200010422A36117F040FE012010BD07
:1049A0004AF28854C2F2010444F22901C0F2000123
:1049B0000422636517F032FE012010BD4AF28854CC
:1049C000C2F2010443F68971C0F200010422636758
:1049D00017F024FE012010BD4AF28854C2F20104EF
:1049E00042F64D51C0F200010422C4F8903017F095
:1049F00015FE012010BD4AF28854C2F2010442F2B1
:104A0000ED71C0F200010422C4F8D03017F006FEA8
:104A1000012010BDF8B5044615460E460846022191
:104A200018F074F82846022118F070F844F6006374
:104A3000C0F20203012253F83600227200F5007121
:104A4000216053F8351062724DF2C04301F50077D2
:104A500062F31F4300226760E260013BFDD190F8E2
:104A6000003291F8002203F00103D20744BF43F063
:104A70000203DBB2A37221463046FFF7B1FB2146A9
:104A800020742846FFF7ACFB237C18442074204692
:104A9000F8BD00BFF8B5074643F648400E46C0F2E1
:104AA00002000B2119F0D4FD4EF2C0003146C2F2D3
:104AB000000000230A2217F057F843F65440C0F2D2
:104AC0000200012119F0C4FD86B300252C4643F6EF
:104AD0004C700121C0F2020019F0BAFD01344EF20F
:104AE000C000795DE4B2C2F2000000230A2217F090
:104AF0003BF8A6422546EAD84EF2C000C2F20000BA
:104B000017F020F87B78432B19D1072E1DD043F6E0
:104B1000AC40C0F20200202119F09AFD4EF2C00014
:104B2000C2F20000BDE8F84017F00CB84EF2C00029
:104B3000C2F2000017F006F87B78432BE7D043F66B
:104B40005840C0F202001B21E6E743F67440C0F271
:104B500002003621E0E700BF2DE9F04141F2B855EF
:104B60000F468046C2F20105FFF794FF43F6D0409E
:104B70001021C0F2020019F06BFDA86C0368F0214F
:104B8000DB6C984757B1444608EB0706A86C14F84D
:104B9000011B03681B689847A642F7D1A86C0368FD
:104BA000F721DB6C984743F60C000F21C0F202009E
:104BB00019F04EFD41F200703A464146C2F2010042
:104BC000002315F067FB43F6F400C0F20200142145
:104BD00019F03EFD4EF2C000C2F20000BDE8F04107
:104BE00016F0B0BF2DE9F04705460C46FFF752FF1F
:104BF00043F6E4401021C0F2020019F029FD41F211
:104C00000070224600232946C2F2010041F6DC78FA
:104C100015F040FBC2F2010843F6F4001421C0F283
:104C2000020019F015FDD8F848301A691F46501CCB
:104C3000F0211861117057F8102FBA4226BF1B617E
:104C40009E4696464FF0010C4FF000095A69724596
:104C500002F1010114D0596110785A6B8F424FEA6A
:104C6000201A98BF5B619E18511C002A7DD15A6999
:104C700083F830A07245C3F834C002F10101EAD1D3
:104C80007CB3AE4605EB040901274FF0000CD8F8C1
:104C900048301EF8011B1A691E46501C186111701D
:104CA00056F8105FB54224BF1B611D465A69AA42DF
:104CB00002F1010113D0596110785A6B8E424FEA0C
:104CC000201A98BF5B619C18511C002A58D15A6960
:104CD00083F830A0AA425F6302F10101EBD1CE4517
:104CE000D5D1D8F848301A691E46F721501C1861F2
:104CF000117056F8107FB74201D31B611F464FF069
:104D0000010E4FF0000C5A69BA4202F1010113D0B2
:104D1000596110785A6B8E424FEA201598BF5B613B
:104D20009C18511CBAB95A6983F83050BA42C3F87A
:104D300034E002F10101EBD143F61C00C0F20200A5
:104D40000F2119F085FC4EF2C000C2F20000BDE850
:104D5000F04716F0F7BE032984F830005963D2D12A
:104D6000C3F830C0C3F834C0CDE7032986F830005B
:104D700059637FF46BAFC3F83090C3F8349065E7A4
:104D8000032984F83000596390D1C3F830C0C3F8C8
:104D900034C08BE72DE9F04741F2B8570D4606467F
:104DA000C2F20107FFF776FE43F6F8401521C0F284
:104DB000020019F04DFCB86C0368F021DB6C9847D9
:104DC00055B1344606EB0508B86C14F8011B0368AE
:104DD0001B6898474445F7D1B86C0368F721DB6C32
:104DE00041F6DC789847C2F2010843F60C000F2127
:104DF000C0F2020019F02CFCD8F848301A691F469E
:104E0000501CF0211861117057F8102FBA42C0F0F1
:104E1000A0801B619E464FF0010C4FF000095A69BB
:104E2000724502F1010114D0596110785A6B8F421A
:104E30004FEA201A98BF5B619C18511C002A7DD153
:104E40005A6983F830A07245C3F834C002F10101F9
:104E5000EAD17DB3B64606EB050901274FF0000CF9
:104E6000D8F848301EF8011B1A691E46501C1861FC
:104E7000117056F8105FB54224BF1B611D465A6978
:104E8000AA4202F1010113D0596110785A6B8E4287
:104E90004FEA201A98BF5B619C18511C002A5AD116
:104EA0005A6983F830A0AA425F6302F10101EBD195
:104EB000F145D5D1D8F848301A691E46F721501C63
:104EC0001861117056F8107FB74201D31B611F465D
:104ED0004FF0010E4FF0000C5A69BA4202F1010185
:104EE00013D0596110785A6B8E424FEA201598BF43
:104EF0005B619C18511CBAB95A6983F83050BA42A8
:104F0000C3F834E002F10101EBD143F61C00C0F21A
:104F100002000F2119F09CFB4EF2C000C2F200000B
:104F2000BDE8F04716F00EBE032984F8300059633F
:104F3000D2D1C3F830C0C3F834C0CDE7032984F818
:104F4000300059637FF46BAFC3F83090C3F83490EE
:104F500065E796465FE7032984F8300059638ED1F0
:104F6000C3F830C0C3F834C089E700BFFFFFFFFFBC
:104F700070B52DED068B4DF644524DF6385343F681
:104F8000105082B0F0EE408AC2F20002C2F200037A
:104F90001421C0F2020082ED000AC3ED000AB0EE57
:104FA000608A19F055FB18EE900A1DF05FF84EF27A
:104FB000C004C2F2000443F6285641EC100BC0F2C4
:104FC000020620460A2116F00FFE0121304619F094
:104FD0003FFB022017F00AF843F62C5501900A22F5
:104FE000C0F2020501990023204616F0BDFD2846B7
:104FF000012119F02DFB019B07EE903A0023C4F22A
:105000007F3307EE103AF8EE677A9FED5B9BC7EEB1
:10501000876A16EE900A1DF029F841EC100B204625
:105020000A2116F0E1FD43F630500621C0F20200DD
:1050300019F00EFB0121304619F00AFB032016F08F
:10504000D5FF0A22019001460023204616F08CFD70
:105050002846012119F0FCFA019B07EE903A002343
:10506000C4F2FE2307EE103AF8EE677AC7EE876ABD
:1050700016EE900A1CF0FAFF41EC100B20460A21B4
:1050800016F0B2FD43F638500221C0F2020019F0CA
:10509000DFFA40F6DB73C4F2490307EE903A28EEDC
:1050A000278AF6EE007A28EE278AB0EE480A1AF030
:1050B0008BF968EE807A17EE900A1CF0D7FFB0EEFD
:1050C000491AF0EE691A41EC100B41EC1A0B1AF078
:1050D0004FFA2046032116F087FD0121284619F0DA
:1050E000B7FAB0EE480A1AF027F968EE807A17EEA0
:1050F000900A1CF0BBFFB0EE491AF0EE691A41ECC1
:10510000100B41EC180B1AF033FA0321204616F06D
:105110006BFD204616F016FDB0EE491AF0EE691A46
:10512000B0EE4A0AF0EE6A0A1AF022FAB0EE491A14
:10513000F0EE691A55EC104BB0EE480AF0EE680A32
:105140001AF016FA51EC100B1DF0DCFA294601900A
:1051500020461DF0D7FA019B00EE100A00EE903AAF
:1051600040F25C50C2F2010002B0BDEC068BBDE81B
:1051700070400DF013BB00BF0000002085EBB13F75
:105180002DE9F041044643F63C502DED028B0D46CF
:10519000C0F20200032119F05BFA4EF2C0000023B6
:1051A0000A222146C2F2000016F0DEFC43F640500F
:1051B0000121C0F2020019F04BFA4EF2C00029465C
:1051C00000230A22C2F2000016F0CEFC4EF2C0000C
:1051D000C2F2000016F0B6FC672C00F0058251D92F
:1051E000782C00F08E8100F2D180692C00F0FF80D5
:1051F000C0F083826A2C00F045826B2C5AD10023C8
:1052000001EE903A05EB45050023C4F2482305EB77
:10521000051501EE103AC5F3C71307EE903A41F6B3
:10522000D872C2F20102B8EE670AF0EE610AB7EE78
:10523000002A137004F094FA4FF47E43C4F2FF6323
:1052400007EE903AB4EEE70AF1EE10FA00F393821B
:105250004FF47E43CCF2FF6307EE903AB4EEE70AD8
:10526000F1EE10FA40F12F830023C8F20103BDECE8
:10527000028B41F21452C2F20102BDE8F041D36147
:1052800007F076B8072C00F0918117D8012C00F0B8
:10529000A380C0F07D81022C00F06F81042C09D125
:1052A00041F2E463C2F20103186880F8D150C030C3
:1052B000FEF768FBBDEC028BBDE8F081202C00F00E
:1052C000858040F2E880402C00F02681662CF1D1E8
:1052D00005EB45054DF63C5205EB0515EB11C2F209
:1052E0000002322B137000F04A8248F21F529B02D8
:1052F000C5F2EB1282FB0312DB17C3EB221307EE9E
:10530000903A0023C4F21633F8EEE77A00EE103A32
:1053100041F6D853C2F2010387EE800A00214FF410
:10532000803259629A611AF0BFFA0023C4F2A023B6
:1053300007EE903AB2EE047AE0EE077AB3EE047A22
:10534000F4EEC77AF1EE10FA00F151824DF61E63C9
:10535000C4F2896307EE103AF4EEC77AF1EE10FA60
:1053600040F31C824FF40C424FF43E44C4F63C32EE
:10537000C5F26C04BDEC028B41F68873C2F20103E6
:105380009C61DA61BDE8F04106F0F2BF7B2C12D0DF
:1053900040F29D807E2C00F0A8807F2C8AD1BDEC4D
:1053A000028B41F2E463C2F2010300211868BDE8F8
:1053B000F0410AF049B9BDEC028B41F2E463C2F25C
:1053C0000103BDE8F04118680AF046BA40F268539C
:1053D000C2F201031D706DE741F2E463C2F2010302
:1053E000186880F8D250C030FEF7CCFA62E700238C
:1053F00001EE903A0023C4F2964302EE103A05EB18
:1054000045050023C4F2482305EB051501EE103ACB
:10541000C5F3C71307EE903A40F24552C2F20102BB
:10542000B8EE670AF0EE610A137004F099F9B5EE70
:10543000C00AF1EE10FA00F1CC8147F67903C4F20C
:10544000302307EE103AF6EE007AE0EE077A49F6DE
:105450008073C0F20103FCEEE77A17EE902A9A42BD
:1054600040F238821A464FF4507040F23073C2F264
:105470000103197ECC0700F1B181DC8B1A62A042D6
:1054800041F0010188BFD8831976BDEC028BBDE8DD
:10549000F04106F06DBF0A2C7FF40CAF4DF644527C
:1054A000BDEC028B07EE905AC2F20002FBEEEC7AE2
:1054B00012684DF63853C2F2000300EE102AF0EEE7
:1054C000670ABDE8F041C3ED007AFFF751BD792CC2
:1054D0007FF4F0AEBDEC028B41F2E463C2F2010353
:1054E000BDE8F04118680AF0D7B8BDEC028B41F274
:1054F000E463C2F2010301211868BDE8F0410AF03B
:10550000A3B8BDEC028B41F2E463C2F20103BDE833
:10551000F04118680AF0ACB841F2E466C2F2010644
:105520003F2D94BF0021012130680AF095F83068C2
:105530000AF09AF8054600287FF4BCAE306837467A
:105540000AF02EFAEBB203EB430498424FEA8404CC
:105550007FF6B0AE306803190135DA78002AEFD053
:1055600093F80280B8F1000FEAD198680BF08CFC38
:105570003868044484F80380E2E741F2E463C2F24D
:105580000103186880F8D050C030FEF7FBF991E6AF
:10559000632D3FF68FAE40F26853C2F201031D70D7
:1055A000BDEC028BBDE8F04106F0E2BE07EE905A7A
:1055B0000023C4F2FE23B8EE677A07EE903A87EE36
:1055C000270A4DF63852BDEC028BC2F200024DF6AE
:1055D00044531268C2F20003BDE8F04100EE902A85
:1055E00083ED000AFFF7C4BC43F23332C3F63372D3
:1055F00005EBC50508EE102AC5F34715002207EE96
:10560000905AC4F20C2241F61963C2F2010301EE72
:10561000102A0022B8EE670A00EE902AF0EE481A2F
:10562000B1EE042A1D7004F09BF81AF03DF943F620
:105630005813C3F6345307EE103A42F6F603C3F696
:105640001C7307EE903AE0EE077AF4EEC87AF1EEBA
:1056500010FA00F18780B1EE047AF4EEC77AF1EE29
:1056600010FA40F31E814CF6D042C0F6CC42BDEC9D
:10567000028B41F68873C2F20103BDE8F0415A6221
:1056800006F076BE05EBC5050022C5F3471501EE11
:10569000902A07EE905A41F618630022C2F20103E5
:1056A000C4F20C22B8EE670A01EE102AF0EE610A8D
:1056B000B7EE002A1D7004F053F84FF47E43C4F295
:1056C000FF6307EE903AB4EEE70AF1EE10FA4EDC13
:1056D0004FF47E43CCF2FF6307EE903AB4EEE70A54
:1056E000F1EE10FA40F1E8800023C8F2010341F620
:1056F000D852C2F20102D361C7E6C5EBC505C5F3B6
:10570000471507EE905A4DF640530022C2F20003AF
:1057100001EE902AB8EE670A00EE902AB1EE0C2A4C
:10572000B3EE0B1A1D7004F01BF8B5EEC00AF1EED3
:1057300010FA51D44FF62E73C4F2DF0307EE903AFD
:10574000B4EEE70AF1EE10FA5ADD46F6FF73BDEC4F
:10575000028B41F68872C2F20102BDE8F041136289
:1057600006F006BE4FF43742C5F66D327FE70023E0
:10577000C7F6FF73BBE70023C7F6FF7377E541F673
:10578000D853C2F201034FF48031002259629A616A
:1057900045F27C43C4F2116307EE903A45F246634A
:1057A000C3F6150300EE103A4FF09E4308EE103A90
:1057B00027EE800A60EE087AFDEEE77A17EE904A4F
:1057C00019F002FE20EE080AFDEEC07A17EE902ACC
:1057D000D0E50120002248E60023B8E71C6AA24277
:1057E00015D9D98B1A62884288BFD8834DE645F215
:1057F0007A5245F27B54C0F21702C0F21704B9E5A1
:10580000F0EE407AFEEECA7A17EE903A9FE702F188
:105810007F00C009013000281A62024638BF00220A
:10582000880706D5586A7F30C0090130824238BFE8
:1058300002464F0706D5986A7F30C0090130824280
:1058400038BF02460E0706D5D86A7F30C00901303E
:10585000824238BF0246CD0606D5186B7F30C0099C
:105860000130824238BF02468C0606D5586B7F3025
:10587000C0090130824238BF0246480606D5986BFF
:105880007F30C0090130824238BF0246C90906D0C4
:10589000D96B7F31C90901318A4238BF0A46DA83A0
:1058A000F3E5F7EE006A86EEA77AF0EE477AFEEEB1
:1058B000C17A17EE902ADAE6F0EE407AFEEEC87A68
:1058C00017EE903A13E7F0EE407AFEEEC87A17EE44
:1058D000903ACCE402F17F00C0090130C5E500BF79
:1058E000F8B541F2E063C2F201030E461B7814469C
:1058F000054623B1984202D0FBF776FA18B121464B
:105900003046FFF73DFC43F644500D21013DC0F207
:10591000020018F09DFEE9B20F2915D841F2B857E0
:10592000C2F2010741F0B001B86C03681B689847E8
:10593000B86C036806F07F011B689847B86C036871
:1059400004F07F011B68984743F60C000F21C0F25A
:10595000020018F07DFE230603F0FE43310443F4F9
:10596000304301F4FE012D0243F00B030B4341F2DF
:10597000007005F470611943C2F2010014F04CFC90
:1059800043F6F400C0F20200142118F061FE4EF25A
:10599000C000C2F20000BDE8F84016F0D3B800BF66
:1059A000F0B540F6DB7091B016F020FB064640F6ED
:1059B000DC7016F01BFB030440F6DD7043EA06665C
:1059C00016F014FB074640F6DE7016F00FFB43F2AC
:1059D000AC74C0F2020406430FCC6D460FC50FCC69
:1059E0000FC50FCC0FC594E80F0085E80F0000200D
:1059F00016F0FCFAC24310A902F00F0201EB82027A
:105A0000034652F8405C85F07045ED4385EA231368
:105A100003F00F0301EB8303012053F8403C83EABA
:105A2000151516F0E3FAED4380EA050210A902F01D
:105A30000F0201EB8202034652F8402C82EA151550
:105A400085EA231303F00F0301EB8303022053F8CD
:105A5000403C83EA151516F0C9FAED4380EA0502C9
:105A600010A902F00F0201EB8202034652F8402C0B
:105A700082EA151585EA231303F00F0301EB830374
:105A8000032053F8403C83EA151516F0AFFAED43B6
:105A900080EA050210A902F00F0201EB8202034620
:105AA00052F8402C82EA151585EA231303F00F0300
:105AB00001EB8303042053F8403C83EA151516F0EC
:105AC00095FAED4380EA050210A902F00F0201EBFE
:105AD0008202034652F8402C82EA151585EA231308
:105AE00003F00F0301EB830343F6545053F8403C9B
:105AF0001321C0F2020083EA151546EA072418F0C4
:105B0000A7FD4EF2C000002310222146C2F2000081
:105B100016F02AF843F668500521C0F2020018F08A
:105B200097FDED434EF2C0002946C2F2000000236B
:105B3000102216F019F8A5424BD1002016F056FAA3
:105B400040F26853C2F201031870012016F04EFAB9
:105B500041F61063C2F201031870022016F046FAF3
:105B6000002307EE900AC4F27F3307EE103AF8EEF6
:105B7000676A4DF64453C6EE877AC2F200030320EB
:105B8000C3ED007A16F032FA002307EE900AC4F251
:105B9000FE2307EE103AF8EE676A4DF63853C6EE6C
:105BA000877AC2F200030420C3ED007A16F01EFAD1
:105BB00041F2E0631028C2F201038ABF002218708C
:105BC0001A704EF2C000C2F2000015F0BBFF11B017
:105BD000F0BD43F670502321C0F2020018F038FDEA
:105BE0004AF23473C2F2010340F244541A6800923C
:105BF000C2F2010441F6D47223780099C2F2010284
:105C000043F69450116043F01F031A21C0F20200C2
:105C1000237018F01DFD4EF2C000217800230A22E7
:105C2000C2F2000015F0A0FF4EF2C000C2F2000068
:105C300015F088FFC5E700BF30B543F2AC74C0F281
:105C400002040FCC91B06D460FC50FCC0FC50FCC21
:105C50000FC594E80F0085E80F00002016F0C6F984
:105C6000C24310A902F00F0201EB8202034652F870
:105C7000404C84F07044E44384EA231303F00F03A0
:105C800001EB8303012053F8403C83EA141416F01F
:105C9000ADF9E44380EA040210A902F00F0201EB1F
:105CA0008202034652F8402C82EA141484EA231339
:105CB00003F00F0301EB8303022053F8403C83EA17
:105CC000141416F093F9E44380EA040210A902F0D8
:105CD0000F0201EB8202034652F8402C82EA1414B0
:105CE00084EA231303F00F0301EB8303032053F82B
:105CF000403C83EA141416F079F9E44380EA040284
:105D000010A902F00F0201EB8202034652F8402C68
:105D100082EA141484EA231303F00F0301EB8303D4
:105D2000042053F8403C83EA141416F05FF9E4436E
:105D300080EA040210A902F00F0201EB820203467E
:105D400052F8402C82EA141484EA231303F00F0360
:105D500001EB830340F6DB7053F8403C83EA1414F4
:105D600016F044F9E443250E854204D0294640F656
:105D7000DB7016F055F940F6DC7016F037F9C4F315
:105D80000745854204D0294640F6DC7016F048F9F4
:105D900040F6DD7016F02AF9C4F30725854204D0D9
:105DA000294640F6DD7016F03BF940F6DE7016F03D
:105DB0001DF9E4B2844207D0214640F6DE7011B0EE
:105DC000BDE8304016F02CB911B030BD10B540F22E
:105DD0004454C2F2010482B023781843207058B1B1
:105DE0004AF23472C2F2010241F6D473126801928F
:105DF000C2F20103019A1A6043F694501A21C0F2CC
:105E0000020018F025FC4EF2C000217800230A227F
:105E1000C2F2000015F0A8FE4EF2C000C2F200006F
:105E200015F090FE02B010BD30B540F24454C2F2FD
:105E300001044DF63E552378C2F200053222D80700
:105E400083B02A8010D499072ED45A074CD418074F
:105E500000F19480D90676D41A0600F1B7800BB908
:105E60008023237003B030BD40F26853C2F20103B7
:105E700000201D7816F0BAF8854203D0294600208C
:105E800016F0CEF843F6B0501621C0F2020018F01A
:105E9000DFFB4EF2C000C2F2000015F053FE237883
:105EA00003F0FE032370DAE741F61063C2F2010348
:105EB00001201D7816F09AF8854203D0294601206A
:105EC00016F0AEF843F6C8501721C0F2020018F0E1
:105ED000BFFB4EF2C000C2F2000015F033FE237883
:105EE00003F0FD032370BAE74DF64453C2F20003FA
:105EF00002201B6807EE903A0023C4F27F3307EEBE
:105F0000103A67EE877AFCEEE77ACDED017A16F06B
:105F10006DF89DF80450854203D02946022016F002
:105F20007FF843F6E0501821C0F2020018F090FB11
:105F30004EF2C000C2F2000015F004FE237803F018
:105F4000FB0323708BE741F2E063C2F201030420FC
:105F50001D7816F04BF8854203D02946042016F030
:105F60005FF8FFF769FE43F61860C0F20200FAF727
:105F70002FFD237803F0EF03237070E74DF63853BD
:105F8000C2F2000303201B6807EE903A0023C4F21C
:105F9000FE2307EE103A67EE877AFCEEE77ACDED46
:105FA000017A16F023F89DF80450854203D0294663
:105FB000032016F035F843F6FC50C0F20200FAF761
:105FC00007FD237803F0F703237048E7FFF734FE5B
:105FD00043F63860C0F20200FAF7FAFC237841F287
:105FE000883203F07F0323702A803BE72DE9F843D2
:105FF0004AF20E79C2F2010943F654602DED028B8C
:106000000521C0F2020018F023FBB9F8003007EEBA
:10601000103A43F23333C4F2233308EE903AB8EE29
:10602000C77A43F23333C4F2A33308EE103A37EEA3
:10603000287A4EF2C004C7EE087AC2F200044AF28F
:106040000877C2F201074AF20C78C2F201084AF25C
:106050008C66C2F2010640F22C05C2F2010517EE71
:10606000900A1CF003F841EC100B0221204615F0B9
:10607000BBFD43F65C600D21C0F2020018F0E8FAA7
:106080003B8807EE903AF8EEE77A77EEA87A87EE4B
:10609000887A17EE100A1BF0E9FF41EC100B022181
:1060A000204615F0A1FD43F66C600821C0F2020005
:1060B00018F0CEFAB8F80010204615F0E5FC43F6CB
:1060C00078600C21C0F2020018F0C2FA3188204634
:1060D00015F0DAFC43F688601421C0F2020018F0D3
:1060E000B7FA2988204615F0CFFC43F6A0600921B5
:1060F000C0F2020018F0ACFA41F28853C2F2010378
:106100000A2219682046002315F02EFD43F6AC60E4
:106110000D21C0F2020018F09BFA40F22003C2F2F7
:1061200001030A2219682046002315F01DFD43F6DD
:10613000BC600921C0F2020018F08AFA41F6C0538F
:10614000C2F201030A2219682046002315F00CFD53
:1061500043F6C8600C21C0F2020018F079FA8021E1
:10616000204615F091FC204615F0ECFCBDEC028BAE
:10617000B9F80030B8F800203B80002332802B8033
:10618000BDE8F88370B584B0002441F2E465029460
:106190000194CDF80B40C2F20105062643F6D86003
:1061A0000221C0F2020018F053FA4EF2C00031464C
:1061B000C2F2000015F068FC44F238000221C0F27F
:1061C000020018F045FA4EF2C000C2F2000015F0CD
:1061D000B9FC43F6DC605621C0F2020018F038FA30
:1061E0004EF2C000C2F2000015F0ACFC2B68234454
:1061F0004EF2C00093F8F0100A220023C2F2000011
:1062000015F0B2FC43F64C700121C0F2020018F008
:106210001FFA2B6823444EF2C00093F8F1100A22B3
:106220000023C2F2000015F09FFC43F64C700121E0
:10623000C0F2020018F00CFA2B6823444EF2C000A2
:1062400093F8F2100A220023C2F2000015F08CFC31
:1062500043F64C700121C0F2020018F0F9F92B68E6
:1062600023444EF2C00093F8F3100A220023C2F236
:10627000000015F079FC43F64C700121C0F20200D9
:1062800018F0E6F92B6823444EF2C00093F8F4109E
:106290000A220023C2F2000015F066FC43F64C709F
:1062A0000121C0F2020018F0D3F92B6823444EF20A
:1062B000C00093F8F5100A220023C2F2000015F086
:1062C00053FC43F64C700121C0F2020018F0C0F9F3
:1062D0002B6823444EF2C00093F8F6100A220023E4
:1062E000C2F2000015F040FC43F64C700121C0F2F0
:1062F000020018F0ADF92B6823444EF2C00093F869
:10630000F7100A220023C2F2000015F02DFC43F61C
:1063100034700821C0F2020018F09AF92B68234467
:106320004EF2C00093F8F8100A220023C2F20000D7
:1063300015F01AFC43F640700D21C0F2020018F06F
:1063400087F92B6823444EF2C00093F8F9100A2213
:106350000023C2F2000015F007FC43F640700D2147
:10636000C0F2020018F074F92B6823444EF2C0000A
:106370000A2293F8FA10C2F20000002315F0F4FB91
:106380004EF2C000C2F2000015F0DCFB43F6507084
:106390005C21C0F2020018F05BF94EF2C000C2F2BC
:1063A000000015F0CFFB43F6B0700621C0F20200EA
:1063B00018F04EF92B6823444EF2C00093F8FB10FE
:1063C0000A220023C2F2000015F0CEFB43F644700F
:1063D0000921C0F2020018F03BF92B6823444EF269
:1063E000C00093F8FC100A220023C2F2000015F04E
:1063F000BBFB43F644700921C0F2020018F028F9F3
:106400002B6823444EF2C00093F8FD100A220023AB
:10641000C2F2000015F0A8FB43F634700821C0F268
:10642000020018F015F92B6823444EF2C00093F8CF
:10643000FE100A220023C2F2000015F095FB43F67D
:1064400048700521C0F2020018F002F92B682344BD
:106450004EF2C00093F8FF100A220023C2F200009F
:1064600015F082FB43F6B0700621C0F2020018F06E
:10647000EFF82B6823444EF2C00093F800110A2273
:106480000023C2F2000015F06FFB43F6B070062146
:10649000C0F2020018F0DCF82B6823444EF2C00072
:1064A00093F801110A220023C2F2000015F05CFBF0
:1064B00043F638700421C0F2020018F0C9F82B68C6
:1064C00023444EF2C00093F802110A220023C2F2C4
:1064D000000015F049FB43F648700521C0F20200A8
:1064E00018F0B6F82B6823444EF2C00093F803115D
:1064F0000A220023C2F2000015F036FB43F6487072
:106500000521C0F2020018F0A3F82B6823444EF2D4
:10651000C00093F804110A220023C2F2000015F013
:1065200023FB4EF2C0001534C2F2000015F00AFB46
:106530007E2C06F1FF367FF431AE43F6B8702D2184
:10654000C0F2020018F084F84EF2C000C2F200005F
:1065500015F0F8FA43F64C70C0F20200012118F071
:1065600077F82B6823444EF2C00093F8F0100A220B
:106570000023C2F2000015F0F7FA43F6B4700134BC
:10658000C0F20200022141F2E46618F061F8862CA4
:10659000C2F20106E5D14EF2C000C2F2000015F0D1
:1065A000D1FA43F6E8700521C0F2020018F050F865
:1065B00033684EF2C00093F876110A220023C2F22B
:1065C000000015F0D1FA4EF2C000C2F2000015F042
:1065D000B9FA43F6F0700421C0F2020018F038F85E
:1065E00033684EF2C00093F877110A220023C2F2FA
:1065F000000015F0B9FA4EF2C000C2F2000015F02A
:10660000A1FA43F6F8700521C0F2020018F020F854
:1066100033684EF2C00093F878110A220023C2F2C8
:10662000000015F0A1FA4EF2C000C2F2000015F011
:1066300089FA44F200000921C0F2020018F008F8BB
:1066400033684EF2C00093F879110A220023C2F297
:10665000000015F089FA4EF2C000C2F2000015F0F9
:1066600071FA44F20C000921C0F2020017F0F0FFA9
:1066700033684EF2C00093F87A110A220023C2F266
:10668000000015F071FA4EF2C000C2F2000015F0E1
:1066900059FA44F218000921C0F2020017F0D8FF9D
:1066A00033684EF2C00093F87B110A220023C2F235
:1066B000000015F059FA4EF2C000C2F2000015F0C9
:1066C00041FA44F224000921C0F2020017F0C0FF91
:1066D00033684EF2C00093F87C110A220023C2F204
:1066E000000015F041FA4EF2C000C2F2000015F0B1
:1066F00029FA44F230000A21C0F2020017F0A8FF84
:1067000033684EF2C00093F87D110A220023C2F2D2
:10671000000015F029FA4EF2C000C2F2000015F098
:1067200011FA44F23C000D21C0F2020017F090FF74
:1067300033684EF2C00093F87E110A220023C2F2A1
:10674000000015F011FA4EF2C000C2F2000015F080
:10675000F9F944F24C000921C0F2020017F078FF69
:1067600033684EF2C00093F87F110A220023C2F270
:10677000000015F0F9F94EF2C000C2F2000015F069
:10678000E1F944F258000921C0F2020017F060FF5D
:1067900033684EF2C00093F880110A220023C2F23F
:1067A000000015F0E1F94EF2C000C2F2000015F051
:1067B000C9F944F264000621C0F2020017F048FF54
:1067C00031680A2201F2811101A81CF0E7FC43F6AE
:1067D00028500121C0F2020017F03AFF01A81CF076
:1067E0006FFC014601A817F033FF43F65440012126
:1067F000C0F2020017F02CFF4EF2C000C2F20000FF
:1068000015F0A0F99B244EF2C00000230A22214675
:10681000C2F2000015F0A8F944F238000221C0F2DB
:10682000020017F015FF2B6823444EF2C00093F8C6
:10683000F0100A220023C2F2000015F095F94EF282
:10684000C0000134C2F2000015F07CF9AD2CDAD1A1
:106850004EF2C000C2F2000015F074F904B070BD31
:106860002DE9F0432DED028B41F6C47087B0C2F2E2
:10687000010014F0EFFB41F6C470C2F2010014F005
:106880007FFA41F6C470C2F2010014F071FA41F6C9
:10689000C470C2F2010014F0FDF841F6C470C2F2F7
:1068A000010014F075FA41F6C470C2F2010014F050
:1068B00027FA41F6C470C2F2010014F051FA44F212
:1068C0006C03C0F2020393E8070000244FF0203568
:1068D0006B46029503940494CDF80B508DF8144048
:1068E00003C341F6C4701A8021462246C2F2010059
:1068F00014F012FA68461CF0E3FB024641F6C4703D
:106900006946C2F2010015F0ABF84EF2C000234612
:106910000A222146C2F2000015F026F943F62C5057
:106920000121C0F2020017F093FE4EF2C000234690
:106930000A222146C2F2000015F016F944F278004E
:106940000321C0F2020017F083FE68461CF0B8FB7A
:106950000146684617F07CFE43F654400121C0F220
:10696000020017F075FE4EF2C000C2F2000015F0F2
:10697000E9F844F27C03C0F2020393E803000090BC
:1069800041F6C470019522468DF80410C2F2010050
:106990000B21029503940494CDF80B508DF814400C
:1069A00014F0BAF968461CF08BFB024641F6C4703D
:1069B0006946C2F2010015F053F84EF2C0002346BA
:1069C0000A222146C2F2000015F0CEF843F62C5000
:1069D0000121C0F2020017F03BFE4EF2C000234638
:1069E0000A220B21C2F2000015F0BEF844F2780032
:1069F0000321C0F2020017F02BFE68461CF060FB7A
:106A00000146684617F024FE43F654400121C0F2C7
:106A1000020017F01DFE4EF2C000C2F2000015F099
:106A200091F844F28403C0F202030FCB8DE80F000B
:106A300041F6C47021460122C2F2010004948DF88F
:106A4000144014F069F968461CF03AFB024641F61E
:106A5000C4706946C2F2010015F002F84EF2C0009F
:106A600023460A220121C2F2000015F07DF843F608
:106A70002C500121C0F2020017F0EAFD4EF2C000D6
:106A80000A2223462146C2F2000015F06DF844F2B6
:106A900078000321C0F2020017F0DAFD68461CF00E
:106AA0000FFB0146684617F0D3FD43F65440012121
:106AB000C0F2020017F0CCFD4EF2C000C2F200009E
:106AC00015F040F80221042016F020F802211E20C3
:106AD00016F01CF8DC2016F07DF844F29800342102
:106AE000C0F2020017F0B4FD4EF2C000C2F2000086
:106AF00015F028F844F2D0002E21C0F2020017F061
:106B0000A7FD4EF2C000C2F2000015F01BF844F2DF
:106B100000102721C0F2020017F09AFD4EF2C000CB
:106B2000C2F2000015F00EF844F228100D21C0F258
:106B3000020017F08DFD4EF2C000C2F2000015F009
:106B400001F8FEF72DFFFCF78BFD4EF28813CEF215
:106B50000003012740F2002040F25C55C2F201051B
:106B60001F604FF4E171C1F6FF7014F085FA2846FA
:106B70000BF068FF28460BF035FCEA88242122F050
:106B8000100228460BF0FEFAEA88242122F48072D3
:106B900028460BF0F7FA28460BF0A4FBF7EE000AA4
:106BA000B0EE600A28460BF017FD1F2128460BF0B7
:106BB0008FFC28460BF0FEFE4CF6CD4EC3F64C5E25
:106BC00001EE10EA4DF20A7EC3F6234E00EE90EA83
:106BD00046F2666EC3F6667E00EE10EA3A463B4623
:106BE000394628460CF008F928460BF0F9FA44F229
:106BF00038101B21C0F2020017F02AFD4EF2C0002F
:106C0000C2F2000014F09EFF4DF63853C2F20003AA
:106C10004DF644581B68C2F2000800EE903AD8F8CE
:106C2000003000EE103AFEF7A3F94DF66850C2F2BC
:106C300000000B210DF034FC4DF66850C2F200004C
:106C40000D210DF095FC49F27410C2F20100FE21F5
:106C50000DF0CCFD002840F0088144F25410C0F241
:106C60000200F9F7B5FE44F26C13C0F2020393E898
:106C7000030041F6C45241F67C73C2F20102C2F233
:106C8000010382E8030083E8030041F61065C2F2C5
:106C90000105D8F8003007EE103A0023C4F2C823EB
:106CA00006EE903A0023C4F22C2307EE903A27EE2A
:106CB000267A002327EE277A06EE103AC7EE267AC8
:106CC00077EE867AFDEEE77A17EE903A9B0072B681
:106CD00041F24C54C2F20104E36062B6237C012B02
:106CE00040F2A38372B6E36862B640F22402002B3E
:106CF000C2F20102B8BF03339B1013602B7872B647
:106D00009B00236262B694F82430012B40F2F68394
:106D100072B6236A62B640F22402002BB8BF033376
:106D2000C2F2010240F26C509B10C2F201005360AB
:106D300013F052FE40F27C50C2F2010013F04CFE00
:106D40004AF20E744AF20C71C2F20104C2F201015D
:106D50004AF208724AF28C63C2F20102C2F20103E3
:106D600044F2901025880C8815801821C0F202008A
:106D70001C8017F06DFC002015F038F901464EF22A
:106D8000C00000230A22C2F2000014F0EDFE43F618
:106D90002C500121C0F2020017F05AFC012015F01E
:106DA00025F901464EF2C00000230A22C2F200007B
:106DB00014F0DAFE43F654400121C0F2020017F04D
:106DC00047FC4EF2C000C2F2000014F0BBFEFFF719
:106DD000D9F944F2AC101421C0F2020017F038FCCB
:106DE0004EF2C0008021C2F2000014F04DFE44F2C9
:106DF000C4101121C0F2020017F02AFC4EF2C000AC
:106E000040F65A31C2F2000014F03EFE44F2D810AF
:106E10000321C0F2020017F01BFC4EF2C000C2F2C8
:106E2000000014F08FFEFFF7E1F841F6C470C2F2E3
:106E3000010013F065FF02F0B5FC4EF20813CEF22C
:106E40000003012244F2DC101A600B21C0F20200A0
:106E500017F0FEFB4EF2C000C2F2000014F072FE0A
:106E600007B0BDEC028BBDE8F08344F274100E2134
:106E7000C0F2020017F0ECFB4EF2C000C2F20000BC
:106E800014F060FE40F2685941F2A463C2F20103BB
:106E9000C2F201091F7009F05BFA99F8003041F65F
:106EA0001162C2F2010203EB430140F2300503EB31
:106EB0008103C2F2010541F6C4511070C2F2010112
:106EC000E81809F0D3F899F8000009F0EDF844F259
:106ED0008410C0F20200F9F771FD99F8003003EB5D
:106EE000430003EB80002844F9F768FD43F62C507B
:106EF000C0F20200F9F762FD41F6C450C2F201008F
:106F0000F9F75CFD43F65440C0F2020041F61C65FF
:106F10006E46F9F75DFDC2F201052FE044F28C10D8
:106F20000321C0F2020017F093FB4EF2C0000023D1
:106F30000A222146C2F2000014F016FE43F6285041
:106F40000121C0F2020017F083FB28461CF0B8F8BC
:106F50000146284617F07CFB43F654400121C0F25D
:106F6000020017F075FB4EF2C0000134C2F20000BF
:106F700014F0E8FD202C05F10B0509D0092CCDD823
:106F800043F64C700121C0F2020017F061FBC5E727
:106F90004AF2CE0344F29C1743F6C45544F27454AB
:106FA00041F27840C0F22A733246C2F20100002159
:106FB000C0F65567CCF63115C1F2793400930293CF
:106FC0000197039504940CF0E7FB4DF63C52C2F296
:106FD000000248F21F5113780022C4F21632C5F2A3
:106FE000EB119B0200EE102A81FB03231B0907EE25
:106FF000903AF8EEE77A87EE800A18F055FC002305
:10700000C4F2A02307EE903AB2EE047AE0EE077ADB
:10701000B3EE047AF4EEC77AF1EE10FA14D44DF61A
:107020001E63C4F2896307EE103AF4EEC77AF1EEFC
:1070300010FA40F3B9814FF40C424FF43E44C4F6C9
:107040003C32C5F26C0407E045F27A5245F27B54BB
:10705000C0F21702C0F2170441F61963C2F201032D
:1070600041F688751B7800EE103A43F23333C3F6CD
:10707000337308EE103A0023C4F20C23C2F2010568
:1070800001EE103A002300EE903AF0EE481AB1EE0D
:10709000042AEA61B8EE400AAC6102F061FB18F024
:1070A00003FC43F65813C3F6345307EE103A42F686
:1070B000F603C3F61C7307EE903AE0EE077AF4EE9F
:1070C000C87AF1EE10FA00F19A81B1EE047AF4EE8A
:1070D000C77AF1EE10FA00F3B581F7EE006A86EE9A
:1070E000A77AF0EE477AFEEEC17A17EE902A4DF6B7
:1070F0004053C2F2000300211B786A6200EE103A8E
:1071000001EE901AB8EE400A00EE901AB1EE0C2A89
:10711000B3EE0B1A02F024FBB5EEC00AF1EE10FA42
:1071200000F17E814FF62E73C4F2DF0307EE903A32
:10713000B4EEE70AF1EE10FA00F36F81F0EE407A58
:10714000FEEECA7A17EE903A41F61864C2F20104D4
:10715000002201EE902A22782B6200EE102A0022F3
:10716000C4F2964202EE102A0022C4F2482201EE36
:10717000102AB8EE400AF0EE610A02F0F1FAB5EE1C
:10718000C00AF1EE10FA00F14D8147F67903C4F21E
:10719000302307EE103AF6EE007AE0EE077A49F671
:1071A0008073C0F20103FCEEE77A17EE902A9A4250
:1071B00040F29F811A464FF4507040F23073C2F291
:1071C0000103197ECE0700F11F81DD8B1A62A842F0
:1071D00041F0010188BFD8831976237800EE103A78
:1071E000002301EE903A41F6D8540023C4F20C2358
:1071F000C2F2010401EE103AB8EE400A4FF48033B7
:10720000F0EE610AB7EE002AA36102F0A9FA4FF48A
:107210007E43C4F2FF6307EE903AB4EEE70AF1EE64
:1072200010FA00F3E8804FF47E43CCF2FF6307EEE0
:10723000903AB4EEE70AF1EE10FA00F15681F0EE62
:10724000407AFEEEC87A17EE903A41F6D875C2F24F
:107250000105002201EE902A2A78E36100EE102A4F
:107260000022C4F248224FF4803301EE102AB8EE17
:10727000400A0022F0EE610AB7EE002A6362A261C2
:1072800002F06EFA4FF47E43F7EE007AC4F2FF6329
:1072900037EEC00A07EE903AB4EEE70AF1EE10FAC4
:1072A00000F3A5804FF47E43CCF2FF6307EE903AE3
:1072B000B4EEE70AF1EE10FA00F11381F0EE407A35
:1072C000FEEEC87A17EE903A2A7800EE102A0022D5
:1072D00001EE902A41F214540022C4F24822C2F274
:1072E000010401EE102AB8EE400AF0EE610AB7EE92
:1072F000002AA36102F034FA4FF47E43C4F2FF6324
:1073000007EE903AB4EEE70AF1EE10FA6BDC4FF4B8
:107310007E43CCF2FF6307EE903AB4EEE70AF1EE5B
:1073200010FA00F18B80F0EE407AFEEEC87A17EE8C
:10733000903A2A78E36100EE102A002201EE902AAA
:107340000022C4F2482201EE102AB8EE400AF0EE04
:10735000610AB7EE002A02F003FA4FF47E43C4F24A
:10736000FF6307EE903AB4EEE70AF1EE10FA36DC6E
:107370004FF47E43CCF2FF6307EE903AB4EEE70A97
:10738000F1EE10FA56D4F0EE407AFEEEC87A17EE1F
:10739000903A41F61065C2F2010599F8000029788B
:1073A000236209F069F974E445F24663C3F61503F4
:1073B00000EE103A4FF09E4308EE103A27EE800A96
:1073C00060EE087AFDEEE77A17EE904A17F0FCFFC0
:1073D00020EE080AFDEEC07A17EE902A3CE6002364
:1073E000C7F6FF73D5E70023C7F6FF73A1E70023B5
:1073F000C7F6FF7368E70023C7F6FF7325E74FF46E
:107400003742C5F66D3272E61D6AAA421FD9D98B82
:107410001A62884288BFD883DFE646F6FF7393E698
:10742000002391E601200022C7E672B62046FCF751
:1074300029FD58E40023C8F20103AAE70023C8F29B
:10744000010376E74CF6D042C0F6CC424FE602F19B
:107450007F00C009013000281A62024638BF0022AE
:107460008D0706D5586A7F30C0090130824238BF87
:107470000246480706D5986A7F30C009013082422B
:1074800038BF02460F0706D5D86A7F30C0090130E1
:10749000824238BF0246CE0606D5186B7F30C0093F
:1074A0000130824238BF02468D0606D5586B7F30C8
:1074B000C0090130824238BF0246480606D5986BA3
:1074C0007F30C0090130824238BF0246C90906D068
:1074D000D96B7F31C90901318A4238BF0A46DA8344
:1074E0007BE60023C8F20103EEE60023C8F20103A5
:1074F000ABE602F17F00C00901305EE672B641F2F0
:107500006050C2F20100FCF7BDFC02E42DE9F04F2F
:1075100083B093F001038946019300F0B080836C3F
:1075200019691F464D1CF0241D610C7057F8106F2F
:10753000BE4224BF1B611E464FF0010E4FF0000CEF
:107540005969B14201F1010416D05C610D78596BA3
:10755000A7424FEA251A98BF5B6103EB01084C1C58
:10756000002940F08180596983F830A0B142C3F806
:1075700034E001F10104E8D1B9F1000F33D04FF04C
:10758000000802F1FF3AC3460121836C1AF8014F4B
:107590001A691F46551C1D61147057F8106FBE42C2
:1075A00024BF1B611E465A69B24202F1010414D085
:1075B0005C6115785A6BA7424FEA251C98BF5B6146
:1075C00003EB020E541C002A3AD15A6983F830C0EA
:1075D000B242596302F10104EAD108F10108C14540
:1075E000D3D8019B4BB3836C1A691F46F721501CFB
:1075F0001861117057F8106FBE4224BF1B611E4600
:107600004FF0010E4FF0000C5A69B24202F1010135
:1076100013D0596110785A6B8F424FEA201598BFEA
:107620005B619C18511CAAB95A6983F83050B24268
:10763000C3F834E002F10101EBD103B0BDE8F08FF3
:10764000032C8EF830505C63ADD1C3F830B0C3F872
:1076500034B0A8E7032984F830005963D4D1C3F8C3
:1076600030C0C3F834C0CFE7032C88F830505C63D7
:107670007FF466AFC3F830C0C3F834C060E70029B8
:107680007FF47DAFD9E700BF2DE9F0479DF820409A
:10769000013CE4B20F2C03D84EB2002E0D4601DBA4
:1076A000BDE8F087E0290FD9F729F9D90835EDB2FF
:1076B000012303FA05F515F0DD0FF1D0806C0368A6
:1076C000BDE8F0471B6818478146806C1F46036879
:1076D00046EA0401C9B21B6890469847D9F84800A9
:1076E000036808F07F011B6805F0EF059847C02D7F
:1076F000D6D0D9F84800036807F07F011B68BDE8C1
:10770000F0471847F0B506464FF0010E56F8107FC7
:107710004FF0000C43699F4203F1010213D0426114
:107720001978436BB2424FEA211528BF4061C41853
:107730005A1C4BB9436980F830509F42C0F834E07E
:1077400003F10102EBD1F0BD032A84F8301042634B
:10775000E0D1C0F830C0C0F834C0DBE72DE9F84F05
:107760009DF82850013DEDB20F2D02D84EB2002EEB
:1077700001DBBDE8F88FE0296DD8846C27693543BB
:10778000A6467E1C26613D705EF8107F774502F0AC
:107790007F0824BF246127464FF0010C4FF00009F9
:1077A0006269974202F1010515D065611678626B36
:1077B000AE454FEA261B98BF646104EB020A551CD4
:1077C000002A5DD1626984F830B09742C4F834C0B1
:1077D00002F10105E9D1826C14699446651C1561BA
:1077E00084F800805CF8104F644526BF126196460D
:1077F000A6464FF001084FF000095469744504F1A2
:10780000010514D055612678546BAC454FEA261A11
:1078100098BF52611719651C002C3BD1546982F83E
:1078200030A07445C2F8348004F10105EAD101F0BA
:10783000EF01C0299DD0806C016902464C1C42F8C2
:10784000104F03F07F030B700369934200D3006174
:10785000FFF758FF8DE7F7298BD901F10803DAB25A
:107860000123934013F0DD0F83D0806C026903463F
:10787000541C43F8104F117002699A42E8D3E6E7AE
:10788000032D8AF8306065638AD1C4F83090C4F85B
:10789000349085E7032D87F830605563ADD1C2F889
:1078A0003090C2F83490A8E770B541F2E063C2F2BC
:1078B000010382B01B780C461546064623B1984258
:1078C00002D0F9F791FA40B141F2E463C2F2010348
:1078D0002A461868214607F059FB44F2E8101121A6
:1078E000C0F2020016F0B4FE2B0603F0FE432104A2
:1078F000721E43F4104343F0090301F4FE01120227
:10790000194302F4706241F200701143C2F20100A7
:1079100012F082FC43F6F4001421C0F2020016F0CB
:1079200097FE41F6DC702B4622460096C2F201001B
:107930009021FFF713FF43F61C000F21C0F2020055
:1079400016F086FE4EF2C000C2F2000002B0BDE8A2
:10795000704014F0F7B800BFF0B541F2E063C2F236
:10796000010383B01B780D461646044623B19842A6
:1079700002D0F9F739FA40B141F2E463C2F20103EF
:1079800032461868294607F001FB44F2FC10162124
:10799000C0F2020016F05CFE611EC9B20F2915D8B4
:1079A00041F2B857C2F2010741F09001B86C036888
:1079B0001B689847B86C036805F07F011B689847FF
:1079C000B86C036806F07F011B68984743F60C000B
:1079D0000F21C0F2020016F03BFE41F6DC70334688
:1079E0002A460094C2F201009021FFF7B7FE43F649
:1079F0001C000F21C0F2020016F02AFE4EF2C00059
:107A0000C2F2000003B0BDE8F04014F09BB800BF24
:107A100070B541F2E063C2F2010382B01B780C46FC
:107A20001646054623B1984202D0F9F7DDF938B180
:107A300041F2E463C2F201032146186807F0E6FC54
:107A400044F214201221C0F2020016F001FE3306A7
:107A500003F0FE4321046A1E43F4004343F008038D
:107A600001F4FE011202194302F4706241F2007047
:107A70001143C2F2010012F0CFFB43F6F4001421CF
:107A8000C0F2020016F0E4FD41F6DC7033462246F7
:107A90000095C2F201008021FFF760FE43F61C0052
:107AA0000F21C0F2020016F0D3FD4EF2C000C2F268
:107AB000000002B0BDE8704014F044B8F0B541F2E7
:107AC000E063C2F2010383B01B780D4616460446FC
:107AD00023B1984202D0F9F787F938B141F2E46353
:107AE000C2F201032946186807F090FC44F22820EE
:107AF0001721C0F2020016F0ABFD611EC9B20F29BA
:107B000015D841F2B857C2F2010741F08001B86CB4
:107B100003681B689847B86C036805F07F011B6811
:107B20009847B86C036806F07F011B68984743F6D6
:107B30000C000F21C0F2020016F08AFD41F6DC7045
:107B400033462A460094C2F201008021FFF706FE68
:107B500043F61C000F21C0F2020016F079FD4EF230
:107B6000C000C2F2000003B0BDE8F04013F0EABF6D
:107B700070B541F2E063C2F2010382B01B780C469B
:107B80001546064623B1984202D0F9F72DF918B1EF
:107B900029462046FDF7F4FA44F240200D21C0F2B8
:107BA000020016F055FD2B0603F0FE432104721E61
:107BB00043F4304343F00B0301F4FE011202194376
:107BC00002F4706241F200701143C2F2010012F03F
:107BD00023FB43F6F4001421C0F2020016F038FD36
:107BE00041F6DC702B4622460096C2F20100B0211D
:107BF000FFF7B4FD43F61C000F21C0F2020016F09F
:107C000027FD4EF2C000C2F2000002B0BDE8704095
:107C100013F098BFF0B541F2E063C2F2010383B004
:107C20001B780D461646044623B1984202D0F9F758
:107C3000DBF818B131462846FDF7A2FA44F250208D
:107C40001221C0F2020016F003FD611EC9B20F2915
:107C500015D841F2B857C2F2010741F0B001B86C33
:107C600003681B689847B86C036805F07F011B68C0
:107C70009847B86C036806F07F011B68984743F685
:107C80000C000F21C0F2020016F0E2FC41F6DC709D
:107C900033462A460094C2F20100B021FFF75EFD90
:107CA00043F61C000F21C0F2020016F0D1FC4EF288
:107CB000C000C2F2000003B0BDE8F04013F042BFC4
:107CC00070B541F2E463C2F2010301F500561B688E
:107CD00005460C4644F2642082B0C3F8C0600D2112
:107CE000C0F2020004F30D0416F0B2FC04F50054D7
:107CF0006A1E1202210401F4FE0302F470611943AA
:107D0000640441F4604104F0FE4441F00E0141F28C
:107D100000702143C2F2010012F07EFA43F6F40033
:107D20001421C0F2020016F093FC41F6DC70C6F399
:107D3000C61306F07F020095C2F20100E021FFF7B2
:107D40000DFD43F61C000F21C0F2020016F080FC6E
:107D50004EF2C000C2F2000002B0BDE8704013F065
:107D6000F1BE00BFF0B541F2E463C2F2010301F5D8
:107D700000541B68054644F27420C3F8C040122129
:107D800083B0C0F2020016F063FC691EC9B20F296D
:107D900004F07F06C4F3C61413D841F2B857C2F2F8
:107DA000010741F0E001B86C03681B689847B86CA4
:107DB000036831461B689847B86C036821461B6806
:107DC000984743F60C000F21C0F2020016F040FC69
:107DD00041F6DC70234632460095C2F20100E021F4
:107DE000FFF7BCFC43F61C000F21C0F2020016F0A6
:107DF0002FFC4EF2C000C2F2000003B0BDE8F0401C
:107E000013F0A0BE70B5064644F2882082B0154635
:107E10000C46C0F20200122116F01AFC6B1E22045E
:107E20001B0203F4706102F4FE030B4343F450435E
:107E3000310143F00D03C9B241F200701943C2F29F
:107E4000010012F0E9F943F6F4001421C0F2020037
:107E500016F0FEFB41F6DC702B4622460096C2F27D
:107E60000100A021FFF77AFC43F61C000F21C0F2AD
:107E7000020016F0EDFB4EF2C000C2F2000002B0AC
:107E8000BDE8704013F05EBEF0B5044644F29C209D
:107E900083B00D46C0F202001721164616F0D8FB3B
:107EA000611EC9B20F2915D841F2B857C2F20107B5
:107EB00041F0A001B86C03681B689847B86C036870
:107EC00005F07F011B689847B86C036806F07F01D6
:107ED0001B68984743F630200A21C0F2020016F0D2
:107EE000B7FB41F6DC7033462A460094C2F201002B
:107EF000A021FFF733FC43F61C000F21C0F2020063
:107F000016F0A6FB4EF2C000C2F2000003B0BDE8BE
:107F1000F04013F017BE00BFF8B50446806C03684C
:107F20001B69984708B90020F8BDA06C03685B691D
:107F30009847C3B203F0FB01F929F4D0A26D7AB9D6
:107F400094F84D2084F84F30150666D440B20028CE
:107F5000C0F24781002084F84D00A0656065F8BD3F
:107F6000010633D494F84F10F02904EB020124D019
:107F700081F84F30616D4B1E9A4224D394F84F2004
:107F8000F02AE7D0130600F1C280002094F85030A8
:107F900084F86600032984F8650084F8673000F0EF
:107FA000CD80012384F86800A065606584F8E9301D
:107FB000002384F84D300120F8BD81F86930636DED
:107FC000013B9A42C6D20132A265ACE7A3F1F701A8
:107FD0000829C7D8012505FA01F010F4DD7F40F02B
:107FE000CD800029BED194F86930F02BB2D1561C57
:107FF0002244F720370A82F8690084F8676084F821
:10800000687084F8651084F84D10284684F866304E
:1080100084F8E950A1656165F8BD02F10C05EEB286
:10802000012E93D902F0FB0EBEF1F90F8ED0EF2A8C
:1080300036D802F0F007802F33D140B2002886DB1B
:10804000012184F84F2084F85030A165EDB2012D54
:1080500080D9BEF1F90F3FF47DAFEF2A00F29B808B
:1080600002F0F003F12B4ED000F29780B02B43D0FA
:108070003BD9D02B47D043D9E02B3DD0F02B7FF418
:1080800069AF0021802084F84D1084F86930606564
:108090007F21A36D8B4211D20133A3650020F8BD6F
:1080A000174607F0DF06902EC7D007F0BF06A02EB8
:1080B000C3D007F0EF07C02FBFD047E71046F8F74F
:1080C0006FFC02F00F020023013294F8501084F884
:1080D000660084F86520012084F8671084F8683011
:1080E000A365636584F8E900F8BD902B04D0A02B4C
:1080F00002D0802B7FF42EAF032363650221C8E7F3
:10810000C02B7FF427AF022363650121C1E7F42A66
:108110003FF43BAF1046F8F743FC802884F8660034
:1081200064D102F00F03013394F8505084F8675083
:10813000032984F8653018BF002501D194F8515007
:1081400084F8685000230121B028A365636584F892
:10815000E91007D00AD8902804D0A02802D080289F
:108160007FF426AF84F84D200120F8BDD028F9D047
:10817000E028F7D0C0287FF41BAFF3E7002284F893
:10818000672084F8682084F8652084F8663084F8D5
:10819000E9502846F8BD134664E7F82B06D018D8F6
:1081A000F32BB0D0A8D3F62B7FF4D4AE1046F8F75B
:1081B000F7FB0022012384F8652084F8672084F807
:1081C000682084F86600A265626584F8E930184684
:1081D000F8BDFA2BFFF4BEAEFC2BE7D9FE2BE5D29F
:1081E000B8E61A468E4603F10C052FE7902898D082
:1081F000B02896D0A02894D0D02892D0E02890D053
:10820000C0288ED000238FE790F86630F12B7CD009
:108210000ED9FA2B2BD01FD8F32B38D0C0F0818089
:10822000F62B7AD0F82B40F08B80036BF3B1184714
:10823000B02B6ED031D9D02B21D03ED9E02B42D0FB
:10824000F02B7ED1C3698BB1B0F86710802900F1A3
:10825000690028BF80211847FC2B0CD051D3FE2B7E
:108260004BD0FF2B6BD1436C002BE0D17047436B9D
:10827000002BDCD1FAE7C36B002BD8D1F6E74369BA
:10828000002BF3D090F8671090F865001847836AC8
:10829000002BEBD090F867001847902B29D0A02B2B
:1082A00023D0802BE2D10368002BDFD090F8682028
:1082B00090F8671090F865001847C02B42D1036909
:1082C000002BDFD1D2E78269002ACFD090F8681066
:1082D00090F8673090F86500C90101F47E5103F011
:1082E0007F031943A1F5005110478368002BDDD1AE
:1082F000BCE74368002BD9D1B8E7036C002B96D1BB
:10830000B4E7836B002B92D1B0E7036A002BC1D195
:10831000ACE7C368002BC9D1A8E7C36A002B86D19C
:10832000A4E7426A002AA1D090F8683090F867006C
:10833000DB0103F47E5300F07F00184310477047C1
:1083400070477047704700BF90F86430DA0725D552
:1083500013F0FE0F22D070B590F8665085F08002C1
:10836000602A82B004461AD9F62D6ED067D8F12D56
:108370007ED04FD9F22D2DD0F32D1AD1806C94F8E8
:108380006760036829461B689847A06C0368DB6C2C
:1083900006F07F0102B0BDE870401847704790F8C2
:1083A00065608E4207D031B15B08012B08D0032BEA
:1083B00027D002B070BD5B08012B01D0022BF8D191
:1083C00094F8683094F86720009629462046FFF715
:1083D0005BF9EEE7806C94F86730026894F86860A7
:1083E0001268294643EAC6159047A06C036805F059
:1083F0007F019B6C9847A06C0368C5F3C6119B6C0A
:10840000C8E794F8683094F8672000962946FFF78B
:108410003BF9CEE7F02DCCD1B0F86760802E28BFB5
:10842000802600F16905002EC3D02E44A06C15F8FB
:10843000011B03681B689847AE42F7D1B9E7FC2DD2
:1084400026D8FA2D01D2F82DB3D105F10803DBB2FD
:10845000072BAED8012202FA03F313F0DD0FA8D0E8
:10846000A06C03681B68294602B0BDE8704018473D
:10847000806C94F8672094F86830066812012946E9
:1084800003F00F0302F0700532681D439047E7E7E1
:10849000FE2D8ED3D9E700BFF8B50546846C16F0E3
:1084A00033F8C0F30723C0F30742010E10F0FF00BA
:1084B0005BD004F1280604F1180712E0A02829D0A7
:1084C00024DDC0283ED0D0283CD0B02822D016F0E1
:1084D0001BF8C0F30723C0F30742010E10F0FF00A2
:1084E00043D00001E02815D0E8DDFC2839DCFA286B
:1084F00003DAF62801D0F828E9D1A26A511CA1625A
:108500001370A36AB342E2D3A762E0E7802801D0E8
:108510009028DCD1A06A00F1010EC4F828E00370B5
:10852000A36AB34228BF3B46581CA0621A70A36AD4
:108530009E4298BF3B465A1CA2621970A36A9E4293
:10854000C5D8E1E7A16A481CA0620B70A36AB342D8
:1085500028BF3B46591CA1621A70A36A9E42B6D836
:10856000D2E7FE380128B2D8C7E7E16AA36A994288
:1085700051D052D318341B1B03F110020B1BD31A1A
:10858000002B48D0AB6CDA6A511CD96203F1280089
:108590008142127824BF03F11801D96202F0FB0373
:1085A000F92B38D0AB6D002B39D0140600F1A68022
:1085B00095F84F10F02905EB030124D081F84F20E6
:1085C000696D4A1E934224D395F84F20F02A30D08B
:1085D000100600F1BC80002095F8503085F8660048
:1085E000032985F8650085F8673000F0C88001230D
:1085F00085F86800A865686585F8E930002385F886
:108600004D300120F8BD81F869206A6D013A93422E
:108610000FD20133AB650020F8BD5B1AB0E795F8C7
:108620004D0085F84F20060609D453B2002BC0F246
:108630003781002085F84D00A8656865F8BD00F118
:108640000C04E3B2012BF0D900F0FB03F92BECD0C2
:10865000EF2800F2AC8000F0F001802940F0A88003
:10866000130600F1C780012385F84F0085F85020DC
:10867000AB65E4B2012CDCD900F0FB03F92BD8D0B8
:10868000EF2800F2D48000F0F003F12B00F0AE8070
:1086900000F2CF80B02B00F0A28040F29980D02B66
:1086A00000F0A48040F29F80E02B00F09880F02B37
:1086B000BFD10022802185F84D2085F86930696599
:1086C0007F22AB6D9342A4D300F00F030133EF2858
:1086D00095F8502085F865304FF0000394BF00F006
:1086E000F001014685F86720012085F8683085F89B
:1086F0006610AB656B6585F8E900F8BD02F109010C
:10870000C9B208293FF654AF012404FA01F010F46D
:10871000DD7F7FD100297FF44BAF95F86920F02AE7
:1087200087D15E1C2B44F720370A83F8690085F84F
:10873000676085F8687085F8651085F84D102046EB
:1087400085F8662085F8E940A9656965F8BDF42AD1
:108750003FF441AF1046F8F723F9802885F866000A
:1087600040F08A8002F00F03013395F8504085F8FD
:108770006740032985F8653018BF002401D195F8BA
:10878000514085F8684000230121B028AB656B6536
:1087900085F8E91007D035D8902804D0A02802D059
:1087A00080287FF42BAF85F84D200120F8BD0146CD
:1087B00001F0DF03902B3FF453AF01F0BF03A02B78
:1087C0003FF44EAF01F0EF01C0293FF449AF2CE771
:1087D000902B04D0A02B02D0802B7FF42AAF032350
:1087E0006B6502226DE7C02B7FF423AF02236B651C
:1087F000012266E702F10C03DBB2012B7FF619AF11
:1088000010463DE7D028CED0E028CCD0C0287FF459
:10881000F5AEC8E7002385F8673085F8683085F83D
:10882000653085F8662085F8E9402046F8BD0346A6
:108830002BE7F82B06D017D8F32BD7D0CFD3F62BB6
:108840007FF4F7AEF8F7ACF80022012385F8652035
:1088500085F8672085F8682085F86600AA656A654E
:1088600085F8E9301846F8BDFA2BFFF4E2AEFC2B90
:10887000E8D9FE2BE6D2DCE690283FF473AFB028AF
:108880003FF470AFA0283FF46DAFD0283FF46AAF3B
:10889000E0283FF467AFC0283FF464AF002364E7EB
:1088A000104602F10C04E4E690F86630F12B7CD01F
:1088B0000ED9FA2B2BD01FD8F32B38D0C0F08180E3
:1088C000F62B7AD0F82B40F08B80036BF3B118476E
:1088D000B02B6ED031D9D02B21D03ED9E02B42D055
:1088E000F02B7ED1C3698BB1B0F86710802900F1FD
:1088F000690028BF80211847FC2B0CD051D3FE2BD8
:108900004BD0FF2B6BD1436C002BE0D17047436BF6
:10891000002BDCD1FAE7C36B002BD8D1F6E7436913
:10892000002BF3D090F8671090F865001847836A21
:10893000002BEBD090F867001847902B29D0A02B84
:1089400023D0802BE2D10368002BDFD090F8682081
:1089500090F8671090F865001847C02B42D1036962
:10896000002BDFD1D2E78269002ACFD090F86810BF
:1089700090F8673090F86500C90101F47E5103F06A
:108980007F031943A1F5005110478368002BDDD107
:10899000BCE74368002BD9D1B8E7036C002B96D114
:1089A000B4E7836B002B92D1B0E7036A002BC1D1EF
:1089B000ACE7C368002BC9D1A8E7C36A002B86D1F6
:1089C000A4E7426A002AA1D090F8683090F86700C6
:1089D000DB0103F47E5300F07F001843104770471B
:1089E00070477047704700BF90F86430DA0778D559
:1089F00013F0FE0F75D02DE9F04390F8665085F026
:108A00008002602A83B004466CD9F62D00F0E9801C
:108A100000F2DF80F12D00F0F68040F2CD80F22DE3
:108A200000F08280F32D59D1836C90F867E01A69C9
:108A30009C46511C196115705CF8107F674524BF76
:108A40001B611F464FF001084FF000095A69BA42F6
:108A500002F1010115D0596110785A6B8C454FEA2B
:108A6000201698BF5B619D18511C002A40F08E8033
:108A70005A6983F83060BA42C3F8348002F10101C8
:108A8000E9D1A36C1A690EF07F0E1F46511C1961C3
:108A900082F800E057F8106FBE4224BF1B611E46EB
:108AA0004FF0010E4FF0000C5A69B24202F1010181
:108AB00014D0596110785A6B8F424FEA201598BF35
:108AC0005B619C18511C002A6BD15A6983F83050A5
:108AD000B242C3F834E002F10101EAD103B0BDE8CB
:108AE000F083704790F865608E420ED069B15B08E4
:108AF000012B0FD0032BF1D194F8683094F8672044
:108B000000962946FEF72AFEE8E75B08012B01D014
:108B1000022BE3D194F8683094F867200096294638
:108B20002046FEF71BFED9E7806C94F867100269B7
:108B300094F868600346571C43F8107F157002696B
:108B40009A4228BF006141EAC615FEF7DBFDA06C22
:108B500002690346511C43F8101F05F07F01117094
:108B600002699A4228BF0061FEF7CCFDA06C026941
:108B70000346511CC5F3C61543F8101F1570026952
:108B80009A4228BF0061FEF7BDFDA7E7032985F8DB
:108B9000300059637FF45AAFC3F83090C3F8349073
:108BA00054E7032984F8300059637FF47DAFC3F89C
:108BB00030C0C3F834C077E7F02D8FD1B0F867101C
:108BC000802900F1690228BF80210123FEF79EFC65
:108BD00084E7FC2D00F28C80FA2D02D2F82D7FF470
:108BE0007DAF05F10803DBB2072B3FF677AF01221B
:108BF00002FA03F313F0DD0F3FF470AFA06C0269CB
:108C00000346511CB8E7836C90F86720196990F807
:108C100068E09C46481C18610D705CF8107F1201DA
:108C2000674502F070020EF00F0E42EA0E0E24BFEE
:108C30001B611F464FF001084FF000095A69BA4204
:108C400002F1010114D0596110785A6B8C454FEA3A
:108C5000201698BF5B619D18511C002A34D15A69B7
:108C600083F83060BA42C3F8348002F10101EAD1DE
:108C7000A36C1A691F46511C196182F800E057F86D
:108C8000106FBE4224BF1B611E464FF0010E4FF015
:108C9000000C5A69B24202F101013FF41FAF596161
:108CA00010785A6B8F424FEA201598BF5B619C1871
:108CB000511C9AB95A6983F83050B242C3F834E073
:108CC00002F10101EBD109E7032985F8300059636E
:108CD000B4D1C3F83090C3F83490AFE7032984F8D7
:108CE00030005963D5D1C3F830C0C3F834C0D0E7E1
:108CF000FE2DFFF4F3AE74E738B541F2B854C2F27A
:108D0000010494F84C50102D12D941F6DC74C2F2D3
:108D1000010494F84C50102D2CD910F095FC41F220
:108D20000070C2F201000021BDE8384011F06EBBB6
:108D30002046FFF7F1F80028E7D094F86630902B32
:108D40003DD083F08003602B3CD941F2B850C2F291
:108D50000100FFF759FA41F6DC7441F2B850C2F253
:108D600001042946C2F20100FFF7EEFA94F84C50D4
:108D7000102DD2D82046FFF78FFB0028CDD094F8D5
:108D80006630902B11D083F08003602B10D941F610
:108D9000DC70C2F20100FFF787FD41F6DC70294666
:108DA000C2F20100FFF720FEB7E794F86830A3B1E4
:108DB00094F865309D42EAD0002DE8D0EDE794F8B4
:108DC000683033B194F865309D42BED0002DBCD0E0
:108DD000C1E7802384F86630F4E7802384F86630A6
:108DE000E6E700BF30B540F2B05085B0C2F20100F6
:108DF0000BF024FA002847D140F24453C2F2010399
:108E00004AF234741B78C2F201047BB141F6D47388
:108E100022680092C2F201034DF63E51C2F20001F7
:108E2000009A18680988121A914221D9FFF764FF45
:108E300041F6146322680292C2F20103029A196891
:108E4000521A632A1BD840F2906322680392C2F23E
:108E50000103039A196841F28730521A824205D9F8
:108E600001F59C5108311960FDF7C0F805B030BD1F
:108E700022680192019A1A60FCF7D6FFD6E76431A6
:108E8000196003F075FADEE741F27444C2F201049E
:108E900013F078FE2368C01AB0F5356FACD913F023
:108EA00071FE206040F2B050C2F201000BF0D6F922
:108EB000044613F067FE41F2E463C2F20103054683
:108EC00022461868802105F09DFF13F05BFE40F6F6
:108ED0005A33401B984251D840F22C0413F052FEF2
:108EE000C2F20104401B238883424FD372B640F282
:108EF0008C53C2F201031A7F02F0FF010AB1002273
:108F00001A7762B699B372B647F6FF744FF4004011
:108F1000B3F91E10B3F92020DC83188462B600294F
:108F200082EAE273A3EBE273B8BF49428B42B8BF57
:108F30000B4607EE903A4FF47E43C4F2FF6306EE11
:108F4000103AF8EEE77A47F2A403C7EE866AC3F652
:108F50007D7307EE103AF4EEC76AF1EE10FA06DD03
:108F600041F6C053C2F201031A6801321A6040F29E
:108F7000B050C2F201000BF083F93DE741F2885393
:108F8000C2F201031A6801321A60A5E713F0FAFD74
:108F9000401B2080AAE700BF2DE9F04F41F2B855F1
:108FA000C2F201058BB012F0CFFF95F864300024B7
:108FB00001264DF6F06743F001034FF6FF7866F3A4
:108FC0004703214685F8654085F8664085F8674087
:108FD00085F8684085F8E940C2F2000705F16900AC
:108FE000802285F86430AF6485F84C4085F84D40A8
:108FF00085F84E406C65AC65C5F85C80C5F860804E
:1090000019F018FF4DF6301240F68911C0F2000138
:109010002846C2F200022C606C60AC60EC602C61EF
:109020006C61AC61EC612C626C62AC62EC622C63D2
:109030006C63AC63EC632C646C6416F07BF841F2F7
:109040000073C2F2010340F2F86744F64452C2F2E0
:109050000107C0F202025C6018469C6041F6DC75B4
:10906000C2F201051A6011F091F807F118034DF6EC
:10907000301240F68D11BC613C607C60BC60FC60CD
:10908000BB62FB62FC613C627C623846C2F2000259
:10909000C0F200013F617F6116F04CF895F8643032
:1090A00085F86540334366F34703214685F86640FB
:1090B00085F8674085F8684085F8E94005F1690062
:1090C000802285F86430AF6485F84C4085F84D40C7
:1090D00085F84E406C65AC65C5F85C80C5F860806D
:1090E00041F6C47719F0A6FE4DF6301240F6911104
:1090F0002846C2F20002C0F20001C2F201072C6051
:109100006C60AC60EC602C616C61AC61EC612C62F9
:109110006C62AC62EC622C636C63AC63EC632C64D9
:109120006C6416F007F8022310222721384611F04C
:10913000A3FC41F24C5043F29C73C0F202030222A2
:109140000321C2F201003B60FBF764FC41F2605076
:109150001D221C21C2F20100FBF75CFC4AF23473B1
:1091600040F26C50C2F2010314220421C2F2010049
:109170001D46019311F018FC40F27C5014221E2170
:10918000C2F2010011F010FC2B68059341F6146344
:10919000C2F2010340F2B058C2F20108059A1A6007
:1091A0002146224640F28C5A4046FAF72DFAC2F286
:1091B000010A44F6D433C0F202030AF11802314620
:1091C000504688F89C40C8F8984088F89D40C8F8F8
:1091D000003041F68879FAF717FA44F67033C2F294
:1091E0000109C0F2020347F6FF7140F23075C2F286
:1091F0000105CAF8003009F134024FF40043AAF81F
:109200001E1048460221AAF82030FAF7FDF94FF661
:109210008011C5F6852123464FF43242C9F8284013
:10922000C9F82C40C9F830402C72EC6044F6B034D8
:10923000C0F28E42C0F2020447F2E820C9F82410BE
:1092400043F29071C0F28E40C9F80040C9F818206E
:109250004FF4805405F55462C0F20201C9F81C00B5
:10926000C9F820406E722A61296018462C4600E039
:10927000226942F82300697A013340F23072994240
:10928000C2F20102F4DC4AF28863C2F201030293E3
:10929000196809B95FE219464B69002BFBD14D6192
:1092A000002441F6D85744F6983340F27070C2F269
:1092B00001072146C0F202036C61AC80EC80AC7205
:1092C0004FF45062C2F201002C766C83AC83EC83C5
:1092D0002B6019F0AFFD41F2784307F12802042119
:1092E00038460093FAF790F944F6BC33C0F2020313
:1092F0003B60039341F21456009BC2F201064FF407
:10930000803BC2F2010306F128020421304600939B
:10931000C7F818B0C7F81CB0C7F820B0C7F824B019
:10932000FAF772F9009BC6F818B01A469832184638
:109330000121039B3360C6F81CB0C6F820B0C6F804
:1093400024B0FAF761F9009844F6A433C0F202039E
:1093500040F2546BC2F2010B40F8183B21468022C8
:1093600019F068FD58468BE800058BF808408BF82B
:109370000940CBF80C408BF8104040F2686A11F0BD
:10938000D9FF4DF6301240F69511C2F2010AC2F231
:109390000002C0F20001584615F0CCFE009BCAF84E
:1093A00004305046CAF800808AF808408AF809401C
:1093B000CAF80C408AF8104011F0BCFF4DF630128C
:1093C00040F69511C2F20002C0F20001504640F290
:1093D0007C6B15F0AFFEC2F2010B009B8BF80840CE
:1093E00058468BE808028BF80940CBF80C408BF804
:1093F000104041F2745A11F09DFF4DF6301240F6C4
:109400009511C2F2010AC2F20002C0F200015846F0
:1094100015F090FE5046CAF80090CAF804508AF839
:1094200008408AF80940CAF80C408AF8104040F217
:10943000946B11F07FFF4DF6301240F69511C2F299
:10944000010BC2F20002C0F20001504615F072FE9C
:109450005846CBF800908BF808408BF80940CBF8C1
:109460000C408BF81040CBF8047040F2A86A11F061
:1094700061FF4DF6301240F69511C2F2010AC2F2B8
:109480000002C0F20001584615F054FE5046CAF8DA
:1094900000908AF808408AF80940CAF80C408AF817
:1094A0001040CAF8046040F2BC6911F043FF4DF669
:1094B000301240F69511C2F20109C2F20002C0F268
:1094C0000001504615F036FE0123484689F8093060
:1094D000009389E8A00089F80840C9F80C4089F891
:1094E000104040F2D06A11F025FF4DF6301240F6E0
:1094F0009511C2F2010AC2F20002C0F20001484610
:1095000015F018FE4FF0020B50468AE860008AF80A
:109510000840CAF80C408AF810408AF809B040F2B6
:10952000E46911F007FF4DF6301240F69511C2F2D2
:109530000109C2F20002C0F20001504615F0FAFD26
:109540004846C9F8045089F8084089F80940C9F824
:109550000C4089F81040C9F8007041F2A86511F07C
:10956000E9FE4DF6301240F69511C2F20105C0F247
:109570000001C2F20002484615F0DCFD0322284635
:10958000C5F800802C72EC602C746A726F6040F237
:10959000485811F0CFFE4DF6301240F69511C2F248
:1095A0000108C2F20002C0F20001284615F0C2FD17
:1095B000009B88F80930404688F80840C8F80C40FD
:1095C00088F81040C8F80070C8F8046011F0B2FEC6
:1095D0004DF6301240F69511C2F20002C0F20001C1
:1095E00041F2C065404615F0A5FDC2F2010543F207
:1095F000907105F11802C0F2020123462C72EC6052
:10960000204685F809B029602A612C4600E02269CD
:1096100042F82300697A013341F2C0629942C2F2F2
:109620000102F4DC029B19684AF28863C2F201036A
:1096300009B992E019464B69002BFBD14D6100241A
:1096400041F2C06041F28C5844F6C833C2F20108BE
:10965000C0F202036C61AC80EC80AC72C2F201001B
:109660002B600AF06BFC4046C8F80060C8F8045054
:1096700088F8084088F80940C8F80C4088F810407D
:1096800041F2A05711F056FE4DF6301240F69511FA
:10969000C2F20107C2F20002C0F20001404615F01A
:1096A00049FD012338467B723E607D603C72FC6060
:1096B0003C7411F03FFE4DF6301240F69511C0F2A9
:1096C00000013846C2F2000215F034FD40F25C534E
:1096D000C2F2010344F67C32C0F202021A604FF477
:1096E000E4700A221A7212F065FF4AF644410646F7
:1096F00005F014F9019F3B680693069D3B680793AC
:10970000079C3B68089341F2E460C2F2010041F615
:10971000D47140F2506241F6D453C2F20101C2F258
:109720000102C2F20103066008980D60146018601F
:1097300013F028FA019F3B68099341F2744240F20A
:109740009063C2F20102C2F201030999106019602C
:109750000BB0BDE8F08F1A60A2E51A606FE700BF9A
:1097600030EE600A32EE612A31EE601A20EE022AF3
:1097700082EE010A30EE210A704700BF00B583B0C7
:1097800012F0E2FB4AF23472C2F2010242F2C80362
:1097900012680192C2F20103019A1A6003B05DF8E7
:1097A00004FB00BF2DE9F04340F21C06C2F20106A3
:1097B0008DB03378002B40F0968540F26855C2F2A8
:1097C000010569460A22287819F038F8044619F08C
:1097D00077FCC0B20228024628BF0222C2F1020072
:1097E00006AB21461844002443F230030694079444
:1097F000ADF81830089409940A948DF82C4019F0AB
:10980000CDFC41F6C47022462146C2F2010011F09F
:1098100083FA06A819F054FC024641F6C47006A962
:10982000C2F2010012F01CF94EF2C00023460A22D7
:109830002146C2F2000012F097F943F62C500121A4
:10984000C0F2020014F004FF4EF2C00023460A22C8
:109850002146C2F2000012F087F944F27800032199
:10986000C0F2020014F0F4FE06A819F029FC01462B
:1098700006A814F0EDFE43F654400121C0F20200A8
:1098800014F0E6FE4EF2C000C2F2000012F05AF9E7
:1098900041F6C47022460221C2F201004FF02008B6
:1098A00006940794089409940A948DF82C408DF836
:1098B000188011F031FA06A819F002FC024641F6B0
:1098C000C47006A9C2F2010012F0CAF84EF2C0003C
:1098D00023460A222146C2F2000012F045F943F65F
:1098E0002C500121C0F2020014F0B2FE4EF2C00072
:1098F00023460A220221C2F2000012F035F944F296
:1099000078000321C0F2020014F0A2FE06A819F0AC
:10991000D7FB014606A814F09BFE43F654400121F4
:10992000C0F2020014F094FE4EF2C000C2F2000039
:1099300012F008F92B7840F2300003EB43024DF6A9
:10994000485703EB8203C2F2010041F6C451C2F250
:1099500000071844C2F2010106F088FB3D7841F689
:10996000C47015F0FD05C2F2010000F0D28222465B
:10997000022106940794089409940A948DF82C40C7
:109980008DF8188011F0C8F906A819F099FB024665
:1099900041F6C47006A9C2F2010012F061F84EF25D
:1099A000C00023460A222146C2F2000012F0DCF871
:1099B00043F62C500121C0F2020014F049FE4EF291
:1099C000C00023460A220221C2F2000012F0CCF8A5
:1099D00044F278000321C0F2020014F039FE06A818
:1099E00019F06EFB014606A814F032FE43F654400F
:1099F0000121C0F2020014F02BFE4EF2C000C2F2B0
:109A0000000012F09FF841F6C450C2F2010019F0B4
:109A100057FBC2B2082A41F6C45128BF08224FF0B2
:109A20002033C2F2010106A8069307940894CDF8EA
:109A30001B3009940A948DF82C4019F0AFFB41F6C5
:109A4000C47022460321C2F2010011F065F906A894
:109A500019F036FB024641F6C47006A9C2F20100B5
:109A600011F0FEFF4EF2C00023460A222146C2F248
:109A7000000012F079F843F62C500121C0F20200E8
:109A800014F0E6FD4EF2C00023460A220321C2F282
:109A9000000012F069F844F278000321C0F20200DD
:109AA00014F0D6FD06A819F00BFB014606A814F029
:109AB000CFFD43F654400121C0F2020014F0C8FD6E
:109AC0004EF2C000C2F2000012F03CF841F6C47041
:109AD00022460B21C2F201000694079408940994CF
:109AE0000A948DF82C408DF8188011F015F906A80D
:109AF00019F0E6FA024641F6C47006A9C2F2010066
:109B000011F0AEFF4EF2C00023460A222146C2F2F7
:109B1000000012F029F843F62C50C0F20200012197
:109B200014F096FD23464EF2C0000A220B21C2F229
:109B3000000012F019F844F278000321C0F202008C
:109B400014F086FD06A819F0BBFA014606A814F029
:109B50007FFD43F654400121C0F2020041F6106936
:109B600014F076FDC2F201094EF2C000C2F200000C
:109B700011F0E8FF99F8000069460A22013018F058
:109B80005DFE044619F09CFAC0B20228024628BFC6
:109B90000222C2F1020006AB21461844002443F21F
:109BA000300306940794ADF81830089409940A9489
:109BB0008DF82C4019F0F2FA41F6C47021460122CA
:109BC000C2F2010011F0A8F806A819F079FA0246CD
:109BD00041F6C47006A9C2F2010011F041FF4EF235
:109BE000C00023460A220121C2F2000011F0BCFF8E
:109BF00043F62C500121C0F2020014F029FD4EF270
:109C0000C00023460A222146C2F2000011F0ACFF38
:109C100044F278000321C0F2020014F019FD06A8F6
:109C200019F04EFA014606A814F012FD43F654400E
:109C30000121C0F2020014F00BFD4EF2C000C2F28E
:109C4000000011F07FFF41F6C47001220221C2F230
:109C50000100202506940794089409940A948DF82D
:109C60002C408DF8185011F057F806A819F028FA72
:109C7000024641F6C47006A9C2F2010011F0F0FEDE
:109C80004EF2C00023460A220121C2F2000011F068
:109C90006BFF43F62C500121C0F2020014F0D8FCF7
:109CA0004EF2C00023460A220221C2F2000011F047
:109CB0005BFF44F278000321C0F2020014F0C8FCFC
:109CC00006A819F0FDF9014606A814F0C1FC43F6F8
:109CD00054400121C0F2020014F0BAFC4EF2C00060
:109CE000C2F2000011F02EFF97F8008008F0FD0886
:109CF00041F6C470B8F1010FC2F2010000F0E88132
:109D00000122022106940794089409940A948DF87C
:109D10002C408DF8185010F0FFFF06A819F0D0F96C
:109D2000024641F6C47006A9C2F2010011F098FE85
:109D30004EF2C00023460A220121C2F2000011F0B7
:109D400013FF43F62C500121C0F2020014F080FCF6
:109D50004EF2C00023460A220221C2F2000011F096
:109D600003FF44F278000321C0F2020014F070FCFB
:109D700006A819F0A5F9014606A814F069FC43F6F7
:109D800054400121C0F2020014F062FC4EF2C00007
:109D9000C2F2000011F0D6FE99F8002041F61C63D3
:109DA00002EB820702EB4707C2F201031F44384669
:109DB00019F086F9C2B20A2A28BF0A224FF02033CE
:109DC000394606A806930793089409940A948DF8D7
:109DD0002C408DF8205019F0E1F941F6C4700122B1
:109DE0000321C2F2010010F097FF06A819F068F9EC
:109DF000024641F6C47006A9C2F2010011F030FE1D
:109E00004EF2C00023460A220121C2F2000011F0E6
:109E1000ABFE43F62C500121C0F2020014F018FCF6
:109E20004EF2C00023460A220321C2F2000011F0C4
:109E30009BFE44F278000321C0F2020014F008FCFB
:109E400006A819F03DF9014606A814F001FC43F6F6
:109E500054400121C0F2020014F0FAFB4EF2C0009F
:109E6000C2F2000011F06EFE41F6C47001220E2114
:109E7000C2F2010006940794089409940A948DF89C
:109E80002C408DF8185010F047FF06A819F018F96B
:109E9000024641F6C47006A9C2F2010011F0E0FDCD
:109EA0004EF2C00023460A220121C2F2000011F046
:109EB0005BFE43F62C500121C0F2020014F0C8FBF7
:109EC0004EF2C00023460A220E21C2F2000011F019
:109ED0004BFE44F278000321C0F2020014F0B8FBFC
:109EE00006A819F0EDF8014606A814F0B1FB43F6F8
:109EF00054400121C0F2020014F0AAFB4EF2C0004F
:109F0000C2F2000011F01EFE002333700DB0BDE858
:109F1000F0835B232A460221069507958DF81830B9
:109F2000089509950A958DF82C5010F0F5FE06A8B5
:109F300019F0C6F8024641F6C47006A9C2F2010043
:109F400011F08EFD4EF2C0002B460A222946C2F2C5
:109F5000000011F009FE43F62C500121C0F202006E
:109F600014F076FB4EF2C0002B460A220221C2F208
:109F7000000011F0F9FD44F278000321C0F2020064
:109F800014F066FB06A819F09BF8014606A814F029
:109F90005FFB43F654400121C0F2020014F058FB6D
:109FA0004EF2C000C2F2000011F0CCFD41F6C450E8
:109FB000C2F2010019F084F8C2B2082A41F6C45175
:109FC00028BF08224FF02033C2F2010106A80693F1
:109FD00007950895CDF81B3009950A958DF82C50FA
:109FE00019F0DCF841F6C4702A460321C2F20100E0
:109FF00010F092FE06A819F063F8024641F6C4700C
:10A0000006A9C2F2010011F02BFD4EF2C0002B4652
:10A010000A222946C2F2000011F0A6FD43F62C5098
:10A020000121C0F2020014F013FB4EF2C0002B46D7
:10A030000A220321C2F2000011F096FD44F27800DA
:10A040000321C0F2020014F003FB06A819F038F84F
:10A05000014606A814F0FCFA43F654400121C0F270
:10A06000020014F0F5FA4EF2C000C2F2000011F046
:10A0700069FD41F6C4705D232A460B21C2F201003E
:10A08000069507958DF81830089509950A958DF86D
:10A090002C5010F041FE06A819F012F8024641F6C5
:10A0A000C47006A9C2F2010011F0DAFC4EF2C00041
:10A0B0002B460A222946C2F2000011F055FD43F654
:10A0C0002C50C0F20200012114F0C2FA2B462AE5FE
:10A0D0005B2342460221069407948DF818300894B9
:10A0E00009940A948DF82C4010F016FE06A818F07A
:10A0F000E7FF024641F6C47006A9C2F2010011F062
:10A10000AFFC4EF2C00023460A224146C2F20000D4
:10A1100011F02AFD43F62C504146C0F2020014F023
:10A1200097FA4EF2C00023460A220221C2F2000032
:10A1300011F01AFD44F278000321C0F2020014F07D
:10A1400087FA06A818F0BCFF014606A814F080FAAA
:10A1500043F654404146C0F2020014F079FA4EF240
:10A16000C000C2F2000011F0EDFC99F8002041F6A9
:10A170001C6302EB820702EB4707C2F201031F4494
:10A18000384618F09DFFC2B20A2A28BF0A224FF0B3
:10A190002033394606A806930793089409940A9435
:10A1A0008DF82C408DF8205018F0F8FF41F6C4705F
:10A1B00042460321C2F2010010F0AEFD06A818F0DD
:10A1C0007FFF024641F6C47006A9C2F2010011F0F9
:10A1D00047FC4EF2C00023460A224146C2F200006C
:10A1E00011F0C2FC43F62C504146C0F2020014F0BC
:10A1F0002FFA4EF2C00023460A220321C2F20000C9
:10A2000011F0B2FC44F278000321C0F2020014F015
:10A210001FFA06A818F054FF014606A814F018FA11
:10A2200043F654404146C0F2020014F011FA4EF2D7
:10A23000C000C2F2000011F085FC41F6C4705D233D
:10A2400042460E21C2F20100069407948DF81830A0
:10A25000089409940A948DF82C4010F05DFD06A82E
:10A2600018F02EFF024641F6C47006A9C2F20100A2
:10A2700011F0F6FB4EF2C00023460A224146C2F21C
:10A28000000011F071FC43F62C504146C0F2020070
:10A2900014F0DEF94EF2C00023460A220E21C2F26B
:10A2A000000011F061FC44F278000321C0F20200CA
:10A2B00014F0CEF906A818F003FF014606A814F022
:10A2C000C7F943F654404146C0F2020014F0C0F909
:10A2D0004EF2C000C2F2000011F034FC00233370D3
:10A2E0000DB0BDE8F08341F6C470C2F2010010F079
:10A2F00007FDFFF762BA00BF2DE9F0412DED028B9B
:10A300004AF23473C2F2010340F21C0790B0C2F269
:10A3100001071B6803933A78039942F2C803C2F21B
:10A320000103012A196000F0C38141F6C470C2F232
:10A33000010010F0E5FC44F2B423C0F2020393E8FC
:10A3400003000AAC00254FF02033A3606360E56092
:10A350002561C4F80B3025750A9041F6C4702A4671
:10A36000ADF82C10C2F20100294610F0D5FC2046B1
:10A3700018F0A6FE024641F6C4702146C2F2010062
:10A3800011F06EFB4EF2C0002B460A222946C2F2A3
:10A39000000011F0E9FB43F62C500121C0F202004D
:10A3A00014F056F94EF2C0002B460A222946C2F29A
:10A3B000000011F0D9FB44F278000321C0F2020042
:10A3C00014F046F9204618F07BFE0146204614F0B2
:10A3D0003FF943F65440C0F20200012114F038F96D
:10A3E0004EF2C000C2F2000011F0ACFB4DF6445832
:10A3F000C2F20008D8ED007A9FEDE08ADFEDE08A36
:10A4000067EE887A0A22FDEEE77A04A917EE900A31
:10A4100018F014FA054618F053FEC0B2032802469D
:10A4200028BF0322C2F1030043F23003C0F230031D
:10A430002946204400250A956560A560E5602561F0
:10A440002575ADF82830A37018F0A8FE41F6C47049
:10A450002A460D21C2F2010010F05EFC204618F0E1
:10A460002FFE024641F6C4702146C2F2010011F0EF
:10A47000F7FA4EF2C0002B460A222946C2F200002B
:10A4800011F072FB43F62C500121C0F2020014F0CF
:10A49000DFF84EF2C0002B460A220D21C2F2000066
:10A4A00011F062FB44F278000321C0F2020014F0C4
:10A4B000CFF8204618F004FE0146204614F0C8F8F4
:10A4C00043F654400121C0F2020014F0C1F84EF2EC
:10A4D000C000C2F2000011F035FBD8ED007AF4EEB6
:10A4E000687AF1EE10FA00F0E5809FEDA67AF4EEBE
:10A4F000C77AF1EE10FA00F1328167EE887AB3EE96
:10A50000007A27EE877AC7EE087A77EEA87AF5EE1A
:10A51000C07AF1EE10FA67DD41F6C47000262A23F6
:10A5200029460122C2F2010026606660A660E6604C
:10A53000266126758DF8283010F0EEFB204618F0C5
:10A54000BFFD024641F6C4702146C2F2010011F07F
:10A5500087FA4EF2C00033460A220121C2F20000FF
:10A5600011F002FB43F62C500121C0F2020014F05E
:10A570006FF84EF2C00033460A222946C2F20000AC
:10A5800011F0F2FA44F278000321C0F2020014F054
:10A590005FF8204618F094FD0146204614F058F864
:10A5A00043F654400121C0F2020014F051F84EF27B
:10A5B000C000C2F2000011F0C5FAD8ED007A67EED3
:10A5C000887AB3EE007A67EE877A013587EE887A6B
:10A5D000EDB207EE905AF8EEE76A77EE287AF4EEDD
:10A5E000E76AF1EE10FA97D4FCEEE77ACDED017A46
:10A5F0009DF804600F2E54D841F6C4700025202326
:10A6000031460122C2F2010025606560A560E56067
:10A61000256125758DF8283010F07EFB204618F056
:10A620004FFD024641F6C4702146C2F2010011F00E
:10A6300017FA4EF2C0002B460A220121C2F2000096
:10A6400011F092FA43F62C500121C0F2020013F0EF
:10A65000FFFF4EF2C0002B460A223146C2F2000034
:10A6600011F082FA44F278000321C0F2020013F0E4
:10A67000EFFF204618F024FD0146204613F0E8FFC6
:10A6800043F654400121C0F2020013F0E1FF01360D
:10A690004EF2C000C2F20000F6B211F053FA102ED2
:10A6A000AAD101233B7010B0BDEC028BBDE8F08154
:10A6B0000AAC9BE64FF0203341F6C470E56025619B
:10A6C0002575C2F201000A93202601222946A360C3
:10A6D0006360C4F80B308DF8286010F01DFB204635
:10A6E00018F0EEFC024641F6C4702146C2F20100A9
:10A6F00011F0B6F94EF2C0002B460A220121C2F237
:10A70000000011F031FA43F62C500121C0F2020092
:10A7100013F09EFF4EF2C0002B460A222946C2F2D9
:10A72000000011F021FA44F278000321C0F2020087
:10A7300013F08EFF204618F0C3FC0146204613F0AC
:10A7400087FF43F654400121C0F2020013F080FF5E
:10A750004EF2C000C2F2000011F0F4F9A1E74FF090
:10A76000203341F6C470C2F201002A260122294694
:10A77000E56025612575A3602360A9E70000C84254
:10A78000000000000AD7233EF0B54AF23473C2F24B
:10A79000010340F21C068FB0C2F201061B68019350
:10A7A0003278019942F2C803C2F20103022A196009
:10A7B00000F0D18041F6C470C2F2010010F0A0FA9E
:10A7C00044F2BC23C0F2020393E8070008AC002562
:10A7D0004FF02033E560C4F80B3084E8070041F601
:10A7E000C4702A462946C2F201002561257510F081
:10A7F00093FA204618F064FC024641F6C4702146E4
:10A80000C2F2010011F02CF94EF2C0002B4629468D
:10A810000A22C2F2000011F0A7F943F62C500121E0
:10A82000C0F2020013F014FF4EF2C0002B460A22C1
:10A830002946C2F2000011F097F944F27800032192
:10A84000C0F2020013F004FF204618F039FC014664
:10A85000204613F0FDFE43F654400121C0F20200F1
:10A8600041F2E06713F0F4FEC2F201074EF2C000BD
:10A87000C2F2000011F066F93D78002D73D00A2273
:10A8800002A9284617F0DAFF054618F019FCC0B2F5
:10A890000228024628BF0222C2F1020043F230031E
:10A8A00029462044002508956560A560E56025617E
:10A8B0002575ADF8203018F071FC41F6C4702946BA
:10A8C0000122C2F2010010F027FA204618F0F8FB2E
:10A8D000024641F6C4702146C2F2010011F0C0F8F0
:10A8E0004EF2C0002B460A220121C2F2000011F0F4
:10A8F0003BF943F62C500121C0F2020013F0A8FEF0
:10A900004EF2C0002B460A222946C2F2000011F086
:10A910002BF944F278000321C0F2020013F098FEF4
:10A92000204618F0CDFB0146204613F091FE43F679
:10A9300054400121C0F2020013F08AFE4EF2C00022
:10A94000C2F2000011F0FEF83F78012F60D0022320
:10A9500033700FB0F0BD41F2E067C2F2010708ACFE
:10A960003D78002D8BD144F64F5341F6C470C4F6A8
:10A970004E1329460122C2F201006560A560E56020
:10A9800025612575089310F0C7F9204618F098FB4B
:10A99000024641F6C4702146C2F2010011F060F88F
:10A9A0004EF2C0002B460A220121C2F2000011F033
:10A9B000DBF843F62C500121C0F2020013F048FEF0
:10A9C0004EF2C0002B460A222946C2F2000011F0C6
:10A9D000CBF844F278000321C0F2020013F038FEF5
:10A9E000204618F06DFB0146204613F031FE43F679
:10A9F00054400121C0F2020013F02AFE4EF2C000C2
:10AA0000C2F2000011F09EF8022333700FB0F0BDC7
:10AA100041F6C47042F220033A460221C2F201001C
:10AA200008956560A560E56025612575ADF8203065
:10AA300010F072F9204618F043FB024641F6C4704C
:10AA40002146C2F2010011F00BF84EF2C0002B4675
:10AA50000A223946C2F2000011F086F843F62C5063
:10AA60003946C0F2020013F0F3FD4EF2C0002B464F
:10AA70000A220221C2F2000011F076F844F27800B6
:10AA80000321C0F2020013F0E3FD204618F018FB8A
:10AA90000146204613F0DCFD43F654403946C0F22F
:10AAA000020013F0D5FD4EF2C000C2F2000011F01A
:10AAB00049F8022333700FB0F0BD00BF2DE9F0411B
:10AAC00040F21C06C2F201068CB03378042B00F071
:10AAD000F88441F6C470C2F2010010F011F944F29A
:10AAE000CC23C0F2020393E8030006AC00256560A6
:10AAF000A560E56025612575069041F6C4702A467B
:10AB00008DF81C10C2F20100294610F005F920460C
:10AB100018F0D6FA024641F6C4702146C2F201008E
:10AB200010F09EFF4EF2C0002B460A222946C2F2C8
:10AB3000000011F019F843F62C500121C0F2020078
:10AB400013F086FD4EF2C0002B460A222946C2F2BF
:10AB5000000011F009F844F278000321C0F202006D
:10AB600013F076FD204618F0ABFA0146204613F0AC
:10AB70006FFD43F654400121C0F2020013F068FD5E
:10AB80004EF2C000C2F2000010F0DCFF41F6C470CB
:10AB900043F654232A460621C2F201000695656059
:10ABA000A560E56025612575ADF8183010F0B4F8A2
:10ABB000204618F085FA024641F6C4702146C2F2DA
:10ABC000010010F04DFF4EF2C0002B460A2229462C
:10ABD000C2F2000010F0C8FF43F62C500121C0F271
:10ABE000020013F035FD4EF2C0002B460A2206216A
:10ABF000C2F2000010F0B8FF44F278000321C0F266
:10AC0000020013F025FD204618F05AFA01462046AE
:10AC100013F01EFD43F654400121C0F2020013F070
:10AC200017FD4EF2C000C2F2000010F08BFF41F69B
:10AC3000C47047F26D332A460E21C2F20100069518
:10AC40006560A560E56025612575ADF8183010F0E8
:10AC500063F8204618F034FA024641F6C4702146E3
:10AC6000C2F2010010F0FCFE4EF2C0002B460A2298
:10AC70002946C2F2000010F077FF43F62C50012164
:10AC8000C0F2020013F0E4FC4EF2C0002B460A2290
:10AC90000E21C2F2000010F067FF44F27800032199
:10ACA000C0F2020013F0D4FC204618F009FA014665
:10ACB000204613F0CDFC43F654400121C0F20200BF
:10ACC00013F0C6FC4EF2C000C2F2000010F03AFFD2
:10ACD00044F2D423C0F2020341F6C4701B68069507
:10ACE0001F0C29460122C2F201006560A560E560E3
:10ACF00025612575ADF818308DF81A7010F00CF834
:10AD0000204618F0DDF9024641F6C4702146C2F231
:10AD1000010010F0A5FE4EF2C0002B460A220121D0
:10AD2000C2F2000010F020FF43F62C500121C0F2C7
:10AD3000020013F08DFC4EF2C0002B460A22294679
:10AD4000C2F2000010F010FF44F278000321C0F2BC
:10AD5000020013F07DFC204618F0B2F901462046AF
:10AD600013F076FC43F654400121C0F2020013F0C8
:10AD70006FFC4EF2C000C2F2000010F0E3FE46F697
:10AD8000567341F6C470C3F66C2301220821C2F247
:10AD900001006560A560E5602561257506930FF0EB
:10ADA000BBFF204618F08CF9024641F6C4702146DC
:10ADB000C2F2010010F054FE4EF2C0002B460A22EF
:10ADC0000121C2F2000010F0CFFE43F62C50012109
:10ADD000C0F2020013F03CFC4EF2C0002B460A22E7
:10ADE0000821C2F2000010F0BFFE44F278000321F7
:10ADF000C0F2020013F02CFC204618F061F9014665
:10AE0000204613F025FC43F65440C0F20200012115
:10AE100013F01EFC4EF2C000C2F2000010F092FED1
:10AE200040F24552C2F201024FF49663107848F2A4
:10AE30001F57C5F2EB1703FB00F387FB0320DB175B
:10AE4000C3EB201069460A2217F0F8FC054618F0FB
:10AE500037F9C0B20428024628BF0422C2F1040018
:10AE60004FF030332946204400256560A560E56039
:10AE700025612575069318F091F941F6C4702A46AC
:10AE80000921C2F201000FF047FF204618F018F91F
:10AE9000024641F6C4702146C2F2010010F0E0FD06
:10AEA0004EF2C0002B460A222946C2F2000010F0E2
:10AEB0005BFE43F62C500121C0F2020013F0C8FBE8
:10AEC0004EF2C0000A222B460921C2F2000010F007
:10AED0004BFE44F278000321C0F2020013F0B8FBED
:10AEE000204618F0EDF80146204613F0B1FB43F67A
:10AEF00054400121C0F2020013F0AAFB4EF2C00040
:10AF0000C2F2000010F01EFE41F61863C2F2010307
:10AF10004AF2EB001B7803EB430303EB4313CEF63B
:10AF20000E2080FB03201844DB17C3EB601069463A
:10AF30000A2217F083FC804618F0C2F8C0B202283B
:10AF4000024628BF0222C2F102004146204443F2D9
:10AF5000300806956560A560E56025612575ADF84A
:10AF6000188018F01BF941F6C47001220421C2F2C6
:10AF700001000FF0D1FE204618F0A2F8024641F67B
:10AF8000C4702146C2F2010010F06AFD4EF2C0000A
:10AF90002B460A220121C2F2000010F0E5FD43F623
:10AFA0002C500121C0F2020013F052FB4EF2C000FF
:10AFB0000A222B460421C2F2000010F0D5FD44F213
:10AFC00078000321C0F2020013F042FB204618F083
:10AFD00077F80146204613F03BFB43F6544001212D
:10AFE000C0F2020013F034FB4EF2C000C2F20000C7
:10AFF00010F0A8FD41F6D873C2F2010369461B7830
:10B0000003EB430303EB431387FB0320DB17C3EB83
:10B0100020100A2217F012FC074618F051F8C0B2AF
:10B020000228024628BF0222C2F10200394620440B
:10B0300006956560A560E56025612575ADF8188009
:10B0400018F0ACF841F6C47001220D21C2F20100E3
:10B050000FF062FE204618F033F8024641F6C47045
:10B060002146C2F2010010F0FBFC4EF2C0002B465C
:10B070000A220121C2F2000010F076FD43F62C50A6
:10B080000121C0F2020013F0E3FA4EF2C0002B4699
:10B090000A220D21C2F2000010F066FD44F2780091
:10B0A0000321C0F2020013F0D3FA204618F008F88A
:10B0B0000146204613F0CCFA43F654400121C0F279
:10B0C00002004DF6485713F0C3FAC2F200074EF2E1
:10B0D000C000C2F2000010F035FD3B7841F6C470AC
:10B0E000072BC2F2010000F04A822A4608214FF0E5
:10B0F000200806956560A560E560256125758DF8D9
:10B1000018800FF009FE204617F0DAFF024641F6DC
:10B11000C4702146C2F2010010F0A2FC4EF2C00041
:10B120002B460A222946C2F2000010F01DFD43F60C
:10B130002C500121C0F2020013F08AFA4EF2C00036
:10B140000A222B460821C2F2000010F00DFD44F245
:10B1500078000321C0F2020013F07AFA204617F0BB
:10B16000AFFF0146204613F073FA43F65440012125
:10B17000C0F2020013F06CFA4EF2C000C2F20000FE
:10B1800010F0E0FC41F6C4700695C2F20100656063
:10B19000A560E560256125752A460D218DF818808A
:10B1A0000FF0BAFD204617F08BFF024641F6C4703F
:10B1B0002146C2F2010010F053FC4EF2C0002B46B3
:10B1C0000A222946C2F2000010F0CEFC43F62C50B1
:10B1D0000121C0F2020013F03BFA4EF2C0002B46F0
:10B1E0000A220D21C2F2000010F0BEFC44F27800E9
:10B1F0000321C0F2020013F02BFA204617F060FF83
:10B200000146204613F024FA43F654400121C0F2CF
:10B21000020013F01DFA4EF2C000C2F2000010F05E
:10B2200091FC3B7841F6C470082B4FF00005C2F248
:10B23000010000F04881012203214FF0200806950B
:10B240006560A560E560256125758DF818800FF0B3
:10B2500063FD204617F034FF024641F6C4702146D4
:10B26000C2F2010010F0FCFB4EF2C0002B460A2295
:10B270000121C2F2000010F077FC43F62C500121AE
:10B28000C0F2020013F0E4F94EF2C0000A222B468D
:10B290000321C2F2000010F067FC44F278000321A1
:10B2A000C0F2020013F0D4F9204617F009FF01465E
:10B2B000204613F0CDF943F654400121C0F20200BC
:10B2C00013F0C6F94EF2C000C2F2000010F03AFCD2
:10B2D00041F6C4700695C2F201006560A560E560A4
:10B2E00025612575012206218DF818800FF014FDC7
:10B2F000204617F0E5FE024641F6C4702146C2F230
:10B30000010010F0ADFB4EF2C0002B460A220121D5
:10B31000C2F2000010F028FC43F62C500121C0F2CC
:10B32000020013F095F94EF2C0002B460A220621C6
:10B33000C2F2000010F018FC44F278000321C0F2C1
:10B34000020013F085F9204617F0BAFE01462046A8
:10B3500013F07EF943F654400121C0F2020013F0CD
:10B3600077F94EF2C000C2F2000010F0EBFB3B7820
:10B3700041F6C470092B4FF00005C2F2010000F045
:10B380005A8101220C21202706956560A560E560A1
:10B39000256125758DF818700FF0BEFC204617F05A
:10B3A0008FFE024641F6C4702146C2F2010010F041
:10B3B00057FB4EF2C0002B460A220121C2F20000C8
:10B3C00010F0D2FB43F62C500121C0F2020013F022
:10B3D0003FF94EF2C0000A222B460C21C2F20000B7
:10B3E00010F0C2FB44F278000321C0F2020013F017
:10B3F0002FF9204617F064FE0146204613F028F985
:10B4000043F654400121C0F2020013F021F94EF23C
:10B41000C000C2F2000010F095FB41F6C470069522
:10B42000C2F201006560A560E56025612575012215
:10B430000F218DF818700FF06FFC204617F040FEBA
:10B44000024641F6C4702146C2F2010010F008FB2A
:10B450004EF2C0002B460A220121C2F2000010F079
:10B4600083FB43F62C500121C0F2020013F0F0F8E8
:10B470004EF2C0002B460A220F21C2F2000010F04B
:10B4800073FB44F278000321C0F2020013F0E0F8ED
:10B49000204617F015FE0146204613F0D9F843F672
:10B4A00054400121C0F2020013F0D2F84EF2C00065
:10B4B000C2F2000010F046FB042333700CB0BDE86C
:10B4C000F08106ACACE45B230122032106956560A4
:10B4D000A560E560256125758DF818300FF01CFC1E
:10B4E000204617F0EDFD024641F6C4702146C2F237
:10B4F000010010F0B5FA4EF2C0002B460A220121DD
:10B50000C2F2000010F030FB43F62C500121C0F2D3
:10B51000020013F09DF84EF2C0002B460A220321D0
:10B52000C2F2000010F020FB44F278000321C0F2C8
:10B53000020013F08DF8204617F0C2FD01462046A8
:10B5400013F086F843F654400121C0F2020013F0D4
:10B550007FF84EF2C000C2F2000010F0F3FA41F69C
:10B56000C4705D230695C2F201006560A560E560C8
:10B5700025612575012206218DF81830B6E65B237A
:10B580002A46082106956560A560E5602561257558
:10B590008DF818300FF0C0FB204617F091FD0246E1
:10B5A00041F6C4702146C2F2010010F059FA4EF281
:10B5B000C0002B460A222946C2F2000010F0D4FA3D
:10B5C00043F62C500121C0F2020013F041F84EF274
:10B5D000C0002B460A220821C2F2000010F0C4FA73
:10B5E00044F278000321C0F2020013F031F8204643
:10B5F00017F066FD0146204613F02AF843F6544042
:10B600000121C0F2020013F023F84EF2C000C2F292
:10B61000000010F097FA41F6C4705D230695C2F25F
:10B6200001006560A560E560256125752A460D214C
:10B630008DF81830B4E55B2301220C210695656076
:10B64000A560E560256125758DF818300FF064FB65
:10B65000204617F035FD024641F6C4702146C2F27D
:10B66000010010F0FDF94EF2C0002B460A22012124
:10B67000C2F2000010F078FA43F62C500121C0F21B
:10B68000020012F0E5FF4EF2C0002B460A220C2108
:10B69000C2F2000010F068FA44F278000321C0F210
:10B6A000020012F0D5FF204617F00AFD01462046A1
:10B6B00012F0CEFF43F654400121C0F2020012F016
:10B6C000C7FF4EF2C000C2F2000010F03BFA41F694
:10B6D000C4705D230695C2F201006560A560E56057
:10B6E0002561257501220F218DF81830A3E600BFD2
:10B6F0002DE9F04140F21C06C2F201068EB033780B
:10B70000032B00F0C48441F6C470C2F201000FF0B4
:10B71000F7FA44F2D823C0F2020393E8030008AC1E
:10B7200000254FF02033A3606360E5602561C4F815
:10B730000B302575089041F6C4702A46ADF82410E8
:10B74000C2F2010029460FF0E7FA204617F0B8FCD4
:10B75000024641F6C4702146C2F2010010F080F9A1
:10B760004EF2C0002B460A222946C2F2000010F019
:10B77000FBF943F62C500121C0F2020012F068FFE1
:10B780004EF2C0002B460A222946C2F2000010F0F9
:10B79000EBF944F278000321C0F2020012F058FFE6
:10B7A000204617F08DFC0146204612F051FF43F66B
:10B7B00054400121C0F2020012F04AFF4EF2C000D4
:10B7C000C2F2000010F0BEF941F6C47043F6462301
:10B7D0002A460721C2F2010008956560A560E56070
:10B7E00025612575ADF820300FF096FA204617F048
:10B7F00067FC024641F6C4702146C2F2010010F017
:10B800002FF94EF2C0002B460A222946C2F2000050
:10B8100010F0AAF943F62C500121C0F2020012F0F8
:10B8200017FF4EF2C0002B460A220721C2F2000089
:10B8300010F09AF944F278000321C0F2020012F0ED
:10B8400007FF204617F03CFC0146204612F000FF9F
:10B8500043F654400121C0F2020012F0F9FE4EF20C
:10B86000C000C2F2000010F06DF946F2525341F6EA
:10B87000C470C3F6732329460122C2F20100656039
:10B88000A560E5602561257508930FF045FA20460F
:10B8900017F016FC024641F6C4702146C2F20100C0
:10B8A00010F0DEF84EF2C0002B460A220121C2F24F
:10B8B000000010F059F943F62C500121C0F20200AB
:10B8C00012F0C6FE4EF2C0002B460A222946C2F2F2
:10B8D000000010F049F944F278000321C0F20200A0
:10B8E00012F0B6FE204617F0EBFB0146204612F0A0
:10B8F000AFFE43F654400121C0F2020012F0A8FE50
:10B900004EF2C000C2F2000010F01CF946F24F33B4
:10B9100041F6C470C3F6742301220821C2F201006B
:10B920006560A560E5602561257508930FF0F4F961
:10B93000204617F0C5FB024641F6C4702146C2F20C
:10B94000010010F08DF84EF2C0002B460A220121B2
:10B95000C2F2000010F008F943F62C500121C0F2A9
:10B96000020012F075FE4EF2C0002B460A2208219A
:10B97000C2F2000010F0F8F844F278000321C0F29F
:10B98000020012F065FE204617F09AFB01462046A1
:10B9900012F05EFE43F654400121C0F2020012F0A4
:10B9A00057FE4EF2C000C2F2000010F0CBF84DF688
:10B9B0003C53C2F200031B78322B00F0718348F233
:10B9C0001F52C5F2EB129B0282FB03231B0907EEF9
:10B9D000903AB8EEE70ADFEDE37A80EE270A13F03B
:10B9E00063FF02AF39460A220025DFEDDF7AB2EEAF
:10B9F000047AE0EE077AFCEEE77ACDED017ABDF845
:10BA0000040016F01BFF804617F05AFBC0B2042852
:10BA1000024628BF0422C2F104004FF030334146F1
:10BA200020446560A560E56025612575089317F0E1
:10BA3000B5FB41F6C4702A460A21C2F201000FF09C
:10BA40006BF9204617F03CFB024641F6C4702146D4
:10BA5000C2F2010010F004F84EF2C0002B460A2298
:10BA60002946C2F2000010F07FF843F62C50012165
:10BA7000C0F2020012F0ECFD0A224EF2C0001146A4
:10BA80002B46C2F2000010F06FF844F27800032158
:10BA9000C0F2020012F0DCFD204617F011FB014657
:10BAA000204612F0D5FD43F65440C0F202000121B9
:10BAB00012F0CEFD4EF2C000C2F2000010F042F8CB
:10BAC00041F61963C2F201034AF2EB001B7803EB63
:10BAD000430303EB4313CEF60E2080FB03201844F0
:10BAE000DB17C3EB601039460A2216F0A7FE0546A5
:10BAF00017F0E6FAC0B20228024628BF0222C2F1BD
:10BB00000200294643F2300800252044089565606C
:10BB1000A560E56025612575ADF8208017F03EFB36
:10BB200041F6C47001220521C2F201000FF0F4F8C1
:10BB3000204617F0C5FA024641F6C4702146C2F20B
:10BB400001000FF08DFF4EF2C0002B460A220121AA
:10BB5000C2F2000010F008F843F62C500121C0F2A8
:10BB6000020012F075FD4EF2C0000A222B4605219C
:10BB7000C2F200000FF0F8FF44F278000321C0F297
:10BB8000020012F065FD204617F09AFA01462046A1
:10BB900012F05EFD43F654400121C0F2020012F0A3
:10BBA00057FD4EF2C000C2F200000FF0CBFF4DF681
:10BBB0004053C2F2000341F2F7201B7803EB8303EA
:10BBC0001B01C4F6DA3080FB0320DB17C3EBE00077
:10BBD00039460A2216F032FE074617F071FAC0B253
:10BBE0000228024628BF0222C2F102003946204440
:10BBF00008956560A560E56025612575ADF8208034
:10BC000017F0CCFA41F6C47001220D21C2F20100F6
:10BC10000FF082F8204617F053FA024641F6C4703E
:10BC20002146C2F201000FF01BFF4EF2C0002B466E
:10BC30000A220121C2F200000FF096FF43F62C50B9
:10BC40000121C0F2020012F003FD4EF2C0002B46AB
:10BC50000A220D21C2F200000FF086FF44F27800A4
:10BC60000321C0F2020012F0F3FC204617F028FA7C
:10BC70000146204612F0ECFC43F654400121C0F28C
:10BC800002004DF6485712F0E3FCC2F200074EF2F4
:10BC9000C000C2F200000FF055FF3B7841F6C470BF
:10BCA000042BC2F2010000F0AB822A4609214FF0BA
:10BCB000200808956560A560E560256125758DF80B
:10BCC00020800FF029F8204617F0FAF9024641F6D5
:10BCD000C4702146C2F201000FF0C2FE4EF2C00055
:10BCE0002B460A222946C2F200000FF03DFF43F620
:10BCF0002C500121C0F2020012F0AAFC4EF2C0004A
:10BD00000A222B460921C2F200000FF02DFF44F257
:10BD100078000321C0F2020012F09AFC204617F0CE
:10BD2000CFF90146204612F093FC43F6544001211E
:10BD3000C0F2020012F08CFC4EF2C000C2F2000011
:10BD40000FF000FF41F6C4700895C2F20100656073
:10BD5000A560E560256125752A460E218DF82080B5
:10BD600004E000BF000016430000A1420EF0D4FF23
:10BD7000204617F0A5F9024641F6C4702146C2F2EA
:10BD800001000FF06DFE4EF2C0002B460A2229463C
:10BD9000C2F200000FF0E8FE43F62C500121C0F281
:10BDA000020012F055FC4EF2C0002B460A220E2172
:10BDB000C2F200000FF0D8FE44F278000321C0F276
:10BDC000020012F045FC204617F07AF901462046A1
:10BDD00012F03EFC43F654400121C0F2020012F082
:10BDE00037FC4EF2C000C2F200000FF0ABFE3B7811
:10BDF00041F6C470052B4FF00005C2F2010000F0BF
:10BE0000A381012204214FF0200808956560A560F8
:10BE1000E560256125758DF820800EF07DFF2046B8
:10BE200017F04EF9024641F6C4702146C2F20100F5
:10BE30000FF016FE4EF2C0002B460A220121C2F27C
:10BE400000000FF091FE43F62C500121C0F20200D9
:10BE500012F0FEFB4EF2C0000A222B460421C2F271
:10BE600000000FF081FE44F278000321C0F20200CE
:10BE700012F0EEFB204617F023F90146204612F09F
:10BE8000E7FB43F654400121C0F2020012F0E0FB50
:10BE90004EF2C000C2F200000FF054FE41F6C47032
:10BEA0000895C2F201006560A560E5602561257511
:10BEB000012207218DF820800EF02EFF204617F07A
:10BEC000FFF8024641F6C4702146C2F201000FF0AD
:10BED000C7FD4EF2C0002B460A220121C2F200002B
:10BEE0000FF042FE43F62C500121C0F2020012F086
:10BEF000AFFB4EF2C0002B460A220721C2F200001F
:10BF00000FF032FE44F278000321C0F2020012F07A
:10BF10009FFB204617F0D4F80146204612F098FB0C
:10BF200043F654400121C0F2020012F091FB4EF2A0
:10BF3000C000C2F200000FF005FE3B7841F6C4706D
:10BF4000062B4FF00005C2F2010000F0B58101227E
:10BF50000C21202708956560A560E56025612575A1
:10BF60008DF820700EF0D8FE204617F0A9F8024692
:10BF700041F6C4702146C2F201000FF071FD4EF28D
:10BF8000C0002B460A220121C2F200000FF0ECFD96
:10BF900043F62C500121C0F2020012F059FB4EF280
:10BFA000C0000A222B460C21C2F200000FF0DCFD7B
:10BFB00044F278000321C0F2020012F049FB20464F
:10BFC00017F07EF80146204612F042FB43F654403B
:10BFD0000121C0F2020012F03BFB4EF2C000C2F29F
:10BFE00000000FF0AFFD41F6C4700895C2F20100E9
:10BFF0006560A560E5602561257501220F218DF83A
:10C0000020700EF089FE204617F05AF8024641F6DD
:10C01000C4702146C2F201000FF022FD4EF2C000B2
:10C020002B460A220121C2F200000FF09DFD43F6CB
:10C030002C500121C0F2020012F00AFB4EF2C000A7
:10C040002B460A220F21C2F200000FF08DFD44F2B0
:10C0500078000321C0F2020012F0FAFA204617F02D
:10C060002FF80146204612F0F3FA43F6544001211E
:10C07000C0F2020012F0ECFA4EF2C000C2F2000070
:10C080000FF060FD032333700EB0BDE8F0814DF674
:10C090003C53C2F2000308AC1B78322B7FF48FAC08
:10C0A000002544F24F6341F6C470C2F246032A46AB
:10C0B0000A21C2F201006560A560E5602561257571
:10C0C00008930EF029FE204616F0FAFF024641F6CC
:10C0D000C4702146C2F201000FF0C2FC4EF2C00053
:10C0E0002B460A222946C2F200000FF03DFD43F61E
:10C0F0002C500121C0F2020012F0AAFA0A224EF2DC
:10C10000C00011462B46C2F200000FF02DFD44F294
:10C1100078000321C0F2020012F09AFA204616F0CD
:10C12000CFFF0146204612F093FA43F65440012116
:10C13000C0F2020012F08CFA4EF2C000C2F200000F
:10C140000FF000FD02AFBBE45B2301220421089540
:10C150006560A560E560256125758DF820300EF0DD
:10C16000DBFD204616F0ACFF024641F6C4702146C6
:10C17000C2F201000FF074FC4EF2C0002B460A22FE
:10C180000121C2F200000FF0EFFC43F62C50012118
:10C19000C0F2020012F05CFA4EF2C0002B460A22F6
:10C1A0000421C2F200000FF0DFFC44F2780003210A
:10C1B000C0F2020012F04CFA204616F081FF014650
:10C1C000204612F045FA43F654400121C0F2020025
:10C1D00012F03EFA4EF2C000C2F200000FF0B2FCC4
:10C1E00041F6C4705D230895C2F201006560A56048
:10C1F000E56025612575012207218DF820305BE679
:10C200005B232A46092108956560A560E5602561E4
:10C2100025758DF820300EF07FFD204616F050FF7A
:10C22000024641F6C4702146C2F201000FF018FC2C
:10C230004EF2C0002B460A222946C2F200000FF03F
:10C2400093FC43F62C500121C0F2020012F000FAD8
:10C250004EF2C0002B460A220921C2F200000FF064
:10C2600083FC44F278000321C0F2020012F0F0F9DE
:10C27000204616F025FF0146204612F0E9F943F664
:10C2800054400121C0F2020012F0E2F94EF2C00067
:10C29000C2F200000FF056FC41F6C4705D23089511
:10C2A000C2F201006560A560E560256125752A463A
:10C2B0000E218DF8203059E55B2301220C210895D1
:10C2C0006560A560E560256125758DF820300EF06C
:10C2D00023FD204616F0F4FE024641F6C4702146C6
:10C2E000C2F201000FF0BCFB4EF2C0002B460A2246
:10C2F0000121C2F200000FF037FC43F62C5001215F
:10C30000C0F2020012F0A4F94EF2C0002B460A223D
:10C310000C21C2F200000FF027FC44F27800032148
:10C32000C0F2020012F094F9204616F0C9FE014650
:10C33000204612F08DF943F654400121C0F202006C
:10C3400012F086F94EF2C000C2F200000FF0FAFBC4
:10C3500041F6C4705D230895C2F201006560A560D6
:10C36000E5602561257501220F218DF8203048E612
:10C370002DE9F04F2DED048B4AF23477C2F201071C
:10C3800087B042F2C8023B680293C2F20102029BEC
:10C39000116840F6B7325B1A934207D940F21C038A
:10C3A000C2F201031B78002B40F0278141F6D473C1
:10C3B0003A680392C2F2010341F287321968039B83
:10C3C0005B1A934208D94DF64854C2F20004237810
:10C3D000023B012B40F248814DF64853C2F2000364
:10C3E00041F24C54019340F26C53C2F2010440F20A
:10C3F00024064BF6836AC2F201039FEDC38A9FEDC8
:10C40000C39ADFEDC38A009304F10C08C2F201065F
:10C41000C2F6A07A0025009B03EB051B58460EF0E0
:10C42000DBFA58465FFA85F90EF01CFB38B13B6821
:10C43000049341F6D453C2F20103049A1A60584699
:10C440000EF006FBA0B341F6D4533A680592C2F24F
:10C4500001031A68059B9B1AB3F5FA7F00F210815D
:10C4600040F21C03C2F20103B9F1010F1B7800F086
:10C47000B980012B00F06983C0F02682022B00F006
:10C480003E83AB4644F20C300721C0F2020012F0AA
:10C49000DFF84EF2C0005946C2F2000000230A2223
:10C4A0000FF062FB4EF2C000C2F200000FF04AFB38
:10C4B000237C012B40F22E8172B6E36862B6002B1A
:10C4C00056F8042BB8BF0333B2EBA30F4BD040F2A6
:10C4D0001C03C2F20103B9F1010F1B7850D1032BE9
:10C4E00000F08881042B00F07A82002B00F0938109
:10C4F00044F2C8300821C0F2020012F0A9F84EF24E
:10C50000C00000230A222946C2F200000FF02CFBD3
:10C5100044F23800C0F20200022112F099F8237CA4
:10C52000012B40F2018272B6E16862B60029B8BF01
:10C5300003314EF2C0008910C2F200000FF0A4FADD
:10C540004EF2C000C2F200000FF0FCFA237C012B77
:10C5500040F2128272B6E36862B6002BB8BF0333B2
:10C560009B1046F8043C0135022D04F1140408F137
:10C5700014087FF450AF07B0BDEC048BBDE8F08F1A
:10C58000012B40F2F180022BB2D1237C012B41F22E
:10C59000438072B6E36862B6032B40F3D684237CF3
:10C5A000012B41F2658072B6E36862B63F2B03DD72
:10C5B00072B64023E36062B6237C012B40F2A88769
:10C5C00072B6E36862B641F2E062002BC2F2010289
:10C5D000B8BF03339B1010201370F9F7F7FBFEF779
:10C5E000D3F885E7002B00F05D81033B012B4FF072
:10C5F000040240F22E82CB4644E7033B012B7FF638
:10C60000D5AE4DF64453C2F2000393ED007ADFED50
:10C610003E6ADFED3E7A9FED3E6A27EE267A27EEF0
:10C62000277AC7EE267A77EE867AFDEEE77A17EE5E
:10C63000903A9B0072B641F24C52C2F20102D360B2
:10C6400062B6137C012B40F2308272B6D36862B6B8
:10C6500040F22402002BC2F20102B8BF03339B1048
:10C660001360FDF79FF8A1E6FDF79CF82378022BF5
:10C6700000F0CE80032B7FF4AFAE01232370ABE636
:10C6800044F2E0202921C0F2020011F0E1FF4EF255
:10C69000C00000230A222946C2F200000FF064FA0B
:10C6A0004EF2C000C2F200000FF04CFAB9F1010FD7
:10C6B000AB467FF4E7AE40F21C03C2F201031B78E5
:10C6C000032B00F06E84042B00F04F84002B7FF4CA
:10C6D000D9AE4DF63C530199C2F2000304221B78F7
:10C6E0000A7072B69B00E36062B6237C012B41F2B4
:10C6F0005E8372B6E36862B6002BB8BF03339B104B
:10C700003360FEF7F5FFBDE60000C84200002C4292
:10C710000000000072B694E80C0010781978637A73
:10C72000227A194202EA00025CD0A37A03F00303E2
:10C730000AB143F0040343F008039A10082BA272D5
:10C7400000F24281072B80F01F82032B00F0208231
:10C7500040F2E080042B00F0E380062B7FF4ADAEC6
:10C76000E368023BE360A9E6237C012B40F2FC86F0
:10C7700072B6E36862B6032B40F3E283237C012B9D
:10C7800040F2B08772B6E36862B6AB2B03DD72B6D7
:10C79000AC23E36062B6237C012B40F2118772B6B2
:10C7A000E36862B64DF63852002BB8BF0333C2F2CD
:10C7B0000002D2ED000A9A10642303FB02F38AFB05
:10C7C0000312DB17C3EBE20307EE903AB8EEE70A79
:10C7D00080EE080AF8F7CCFB0420F9F7F7FAFDF72A
:10C7E0008BFD85E6A37A03F00303002AA5D043F06E
:10C7F0000403A2E7019B1B78052B00F09784062B0E
:10C8000000F01884042B00F0E182FEF771FF6FE660
:10C8100000232370E0E5019B1B78012B00F052867A
:10C82000C0F00882022B00F00882032B37D1237C52
:10C83000012B41F2288272B6E36862B6032B40F303
:10C84000AB87237C012B41F2418372B6E36862B669
:10C8500040F2685B7F2BC2F2010B08DD9BF80030D1
:10C86000622B41F2688272B67C23E36062B6237C5D
:10C87000012B41F2348272B6E36862B641F610626F
:10C88000002BB8BF0333C2F20102C3F387019BF848
:10C890000000117003F0F0FE0220F9F797FAFCF7A0
:10C8A00081FF25E6019B1B78012B00F0CE85C0F0AF
:10C8B0002E83022B00F02B83032B00F0C685FCF7A0
:10C8C00071FF4FF0010BDDE54DF64453C2F200035A
:10C8D00093ED007A27EE087A27EE097AC7EE087AF8
:10C8E00077EEA87AFDEEE77A17EE903A9B0072B6E3
:10C8F000E36062B6237C012B41F2BE8072B6E3682E
:10C9000062B6002BB8BF03339B103360AB46FDF714
:10C91000F3FCB7E5012B00F03781022B7FF4CDAD9E
:10C92000E368013BE360C9E572B6236861681A7881
:10C930000878617A237A084202EA03025DD0A37A7A
:10C9400003F003030AB143F0040343F008039A1011
:10C95000082BA27261D8072B80F04281032B00F0D4
:10C96000FF8240F21F81042B61D0062B7FF4DCADE7
:10C97000E1680239E160D8E572B6236861681A7827
:10C980000878617A237A084202EA03023DD0A37A4A
:10C9900003F003030AB143F0040343F008039A10C1
:10C9A000082BA27247D8072B80F01081032B00F0D0
:10C9B000D28240F2F180042B47D0062B7FF4CBAD1E
:10C9C000E368023BE360C7E50C2B00F0E18000F276
:10C9D000D580092B3FF4C4AE0B2BA1D06DE5019B94
:10C9E0001B78082B00F0BB84092B00F01F84072B59
:10C9F00000F06781FEF762F87AE5A37A03F003039B
:10CA0000002AA4D043F00403A1E7A37A03F00303B0
:10CA1000002AC4D043F00403C1E70C2B00F0A0822D
:10CA200000F2D880092BA3D00B2B7FF47DADE168F9
:10CA30000139E16079E50C2B00F08D8200F2C080B5
:10CA4000092BBDD00B2B7FF486ADE368013BE3607F
:10CA500082E5019B1B78062B00F0D28640F2C48051
:10CA6000082B00F03485C0F0BF86092B40F04C85C0
:10CA700040F24553C2F2010301991B7807220A7064
:10CA800072B69B00E36062B6237C012B41F2EE8319
:10CA900072B6E36862B6002BB8BF03339B103360F5
:10CAA0004FF0010BFEF70AF8ECE472B61368506819
:10CAB00019780478507A137A044201EA030177D096
:10CAC000937A03F0030309B143F0040343F008032E
:10CAD0009910082B917200F28082072B80F0578604
:10CAE000032B00F0498640F26B86042B00F0808215
:10CAF000062B7FF4ABADD368023BD360A7E54DF6C0
:10CB00004453C2F2000393ED007A27EE087A27EE31
:10CB1000097AC7EE087A77EEA87AFDEEE77A17EE83
:10CB2000903A9B0072B6E36062B6237C012B40F220
:10CB3000768772B6E36862B6002BB8BF03339B10EA
:10CB40003360AB46FCF72EFE9CE441F2E063C2F298
:10CB500001031B7872B69B00E36062B6237C012B55
:10CB600040F2308772B6E36862B6002BB8BF033379
:10CB70009B103360AB46FDF707FE83E40D2B3FF4BB
:10CB8000CFAE0E2B7FF499ACE3680133E36095E4FC
:10CB9000E3680233E36091E4012B17D0022B3FF4EA
:10CBA00054AFD8E4012B1BD0022B3FF440AFBBE4C1
:10CBB000937A03F0030300298AD043F0040387E744
:10CBC0000D2B3FF442AF0E2B7FF4C5ACE36801336D
:10CBD000E360C1E40D2B3FF42AAF0E2B7FF4A4AC2D
:10CBE000E1680131E160A0E4042B00F0F085052B41
:10CBF00040F08A844DF640534DF64851C2F200038E
:10CC0000C2F2000106221B780A7072B69B00E36034
:10CC100062B6237C012B41F2248172B6E36862B6CE
:10CC2000002BB8BF03339B1033604FF0010BFEF7AE
:10CC30005FFD27E4019A02231370237C012B40F24D
:10CC4000CA8772B6E36862B6032B40F3B38541F638
:10CC50001162237CC2F20102012B117841F207819B
:10CC600072B6E36862B6002BB8BF0333B1EBA30F13
:10CC700005DC1378013B9B0072B6E36062B6237C4F
:10CC8000012B40F2D48772B6E36862B6002BB8BFBE
:10CC9000033340F2685BC3F38703C2F2010B18460B
:10CCA0008BF8003003F000FA41F61063C2F2010382
:10CCB0009BF80000197803F0DFFC0120F9F786F8F3
:10CCC000EDE5237C012B41F2E08172B6E36862B6A8
:10CCD000032B40F34086237C012B41F2218372B663
:10CCE000E36862B6CB2B03DD72B6C823E36062B69D
:10CCF000237C012B41F2DE8172B6E36862B6002B21
:10CD0000B8BF0333C3F3870307EE903AB8EE677AF0
:10CD1000DFEDBA7ADFEDC46A67EE277A40F2455953
:10CD200087EEA67AC2F2010989F8003077EE287AF8
:10CD3000F5EEC07AF1EE10FA00F10886DFEDB06A88
:10CD4000B6EE007AA7EEA67A49F68073C0F2010328
:10CD5000FCEEC77A17EE90EA9E4540F236879E4673
:10CD60004FF4507040F23073C2F201031A7ED107C3
:10CD700000F1F284D98BC3F820E0814242F0010235
:10CD800038BFD8831A7644F278301721C0F20200F7
:10CD900011F05EFC99F800104FF4966348F21F52B0
:10CDA00003FB01F3C5F2EB1282FB03124EF2C0004B
:10CDB000D917C1EB2211C2F200000EF065FE4EF24F
:10CDC000C000C2F200000EF0BDFE13E6237C012B72
:10CDD00041F2C68172B6E36862B6032B40F3DA858E
:10CDE000237C012B41F2868272B6E36862B6CB2BBC
:10CDF00003DD72B6C823E36062B6237C012B41F2E7
:10CE0000FD8072B6E36862B6002BB8BF03334DF6FF
:10CE10003C59C3F38703C2F20009322B89F8003072
:10CE200000F06B8548F21F52C5F2EB129B0282FBA9
:10CE300003231B0907EE903A9FED720AF8EEE77A9A
:10CE400041F6D853C2F2010387EE800A00214FF465
:10CE5000803259629A6112F027FDDFED6B7AB2EEF3
:10CE6000047AE0EE077AB3EE047AF4EEC77AF1EED4
:10CE700010FA00F1D1849FED657AF4EEC77AF1EEF5
:10CE800010FA41F333854FF40C424FF43E4BC4F695
:10CE90003C32C5F26C0B41F68873C2F2010344F2D6
:10CEA0001430C3F818B01D21DA61C0F2020011F08D
:10CEB000CFFB99F800309FED530A48F21F52C5F29C
:10CEC000EB129B0282FB03231B0907EE903AF8EE5C
:10CED000E77A87EE800A12F0E7FCDFED4B7AB2EEDC
:10CEE000047AE0EE077A17EE900A15F0BFF841ECED
:10CEF000100B4EF2C0000A21C2F200000EF074FEC8
:10CF00004EF2C000C2F200000EF01CFE7DE441F6BD
:10CF100010630199C2F2010301221B780A7072B6F4
:10CF20009B00E36062B6237C934240F29F8272B61C
:10CF3000E36862B6002BB8BF03339B103360BEE4D6
:10CF400072B60023E36062B625E472B60023E360A4
:10CF500062B6FFF731BBE3680233E360FFF7FCBA68
:10CF6000E1680231E160FFF7E0BA41F61063019A2F
:10CF7000C2F2010382F800901B7872B69B00E36056
:10CF800062B6237C012B40F2E58672B6E36862B696
:10CF9000002BB8BF03339B103360FCF703FCFFF793
:10CFA00071BA40F245530199C2F2010307221B787E
:10CFB0000A7072B69B00E36062B6237C012B40F2DC
:10CFC000238772B6E36862B6002BB8BF03339B10A9
:10CFD0003360FDF773FDFFF755BA0C2B00F0CC83DF
:10CFE00000F2CF83092B3FF486AD0B2B7FF42EABE1
:10CFF000D368013BD360FFF72ABB00BF0000964413
:10D0000079783042000016430000A0421EDE8946B7
:10D010002EFFDF409A99894000000C423333333FA2
:10D020005839343DF6281C3F0000484200FEFF46B8
:10D0300000FEFFC6237C012B41F20C8072B6E36830
:10D0400062B6032B40F39684237C012B41F22681A8
:10D0500072B6E36862B66F2B03DD72B66C23E360D1
:10D0600062B6237C012B41F2048072B6E36862B69B
:10D07000002BB8BF0333C3F3870307EE903AB8EE33
:10D08000677AF1EE0C7A27EE277AF3EE0B6AC7EE99
:10D09000267A4DF64059C2F2000989F8003077EE41
:10D0A000A87AF5EEC07AF1EE10FA00F15A841FED7D
:10D0B000287AF4EEC77AF1EE10FA00F3B783B0EEF7
:10D0C000677ABEEECA7A17EE103A41F68872C2F25B
:10D0D000010244F254301362C0F20200222111F026
:10D0E000B7FA99F8003007EE103AB8EE477AF1EE49
:10D0F0000C7A67EE277AF3EE0B6A87EEA67A77EE64
:10D10000287A17EE900A14F0B1FF41EC100B4EF2A2
:10D11000C0000221C2F200000EF066FD4EF2C00017
:10D12000C2F200000EF00EFDFFF76FBB237C012B57
:10D1300040F2A58772B6E36862B6032B40F314840D
:10D14000237C012B41F20F8172B6E36862B68F2B0C
:10D1500003DD72B68C23E36062B6237C012B40F2C0
:10D16000218772B6E36862B6002BB8BF0333C3F3FE
:10D17000870307EE903AB8EE677A5FED5A7A5FED73
:10D180005A6A5FED5A9A67EE277A41F6196987EE77
:10D19000A60AC2F2010989F8003030EE290A12F01D
:10D1A00083FB1FED617A5FED617AE0EE077AF4EEC2
:10D1B000E97AF1EE10FA00F1C182B1EE047AF4EEF0
:10D1C000C77AF1EE10FA00F38484F7EE006A86EE77
:10D1D000A77AF0EE477AFEEEC17A17EE902A41F672
:10D1E0008873C2F2010344F234305A621D21C0F246
:10D1F000020011F02DFA99F800301FED7A7A1FED38
:10D200007A6A5FED7A6A07EE903AF8EE677A67EE2F
:10D21000877A87EE860A30EE260A12F045FB1FED6C
:10D22000807A5FED807AE0EE077A6AE7237C012B53
:10D2300040F25E8772B6E36862B6032B40F3A083C8
:10D24000237C012B41F2308072B6E36862B6CB2BAF
:10D2500003DD72B6C823E36062B6237C012B40F283
:10D260004D8772B6E36862B6002BB8BF0333C3F3D1
:10D27000870307EE903A1FED947A5FED946AB8EE5B
:10D28000676A41F6D879C6EE077AC2F2010989F8D1
:10D290000030B7EE007A77EEA87A37EE677AB4EE10
:10D2A000E67AF1EE10FA00F353825FED9F6AB4EE76
:10D2B000E67AF1EE10FA00F11684F0EE476AFEEE1F
:10D2C000C86A16EE903A1FEDA77A41F21452C2F2E4
:10D2D0000102F4EEC77AF1EE10FA936100F33382A3
:10D2E0001FEDAD7AF4EEC77AF1EE10FA00F1F78394
:10D2F000B0EE677ABEEEC87A17EE103A1FEDB57A37
:10D30000D361F4EEC77AF1EE10FA01F301831FED59
:10D31000B87AF4EEC77AF1EE10FA00F13184B0EE8B
:10D32000677ABEEEC87A17EE103A44F2AC30192193
:10D33000C0F20200136211F08BF94EF2C00099F8AE
:10D34000001000230A22C2F200000EF00DFC4EF283
:10D35000C000C2F200000EF0F5FBFFF74BBB237CD0
:10D36000012B40F2D18672B6E36862B6032B40F31C
:10D370000C83237C012B41F2218072B6E36862B6F4
:10D380008F2B03DD72B68C23E36062B6237C012B06
:10D3900040F2968672B6E36862B6002BB8BF0333DC
:10D3A000C3F3870307EE903ADFEDC76A9FEDC77AB4
:10D3B000B8EE676A41F61869C6EE267AC2F201092C
:10D3C00089F8003077EEA87AF4EEC77AF1EE10FA19
:10D3D00000F3CE819FEDBE7AF4EEC77AF1EE10FA3B
:10D3E00000F18683B0EE677ABEEEC87A17EE103A87
:10D3F00041F6D852C2F2010244F290301B21C0F231
:10D400000200D36111F024F999F80030DFEDAE6A23
:10D4100007EE903AF8EE677A87EEA67A77EE287AEA
:10D4200017EE900A14F022FE41EC100B4EF2C000F1
:10D430000221C2F200000EF0D7FB4EF2C000C2F291
:10D4400000000EF07FFBFFF7D5BA40F2685BC2F236
:10D45000010B01999BF8003000220A7072B69B0004
:10D46000E36062B6237C012B3FF661AD72B658F8DB
:10D470000C2C636810781978637A227A194202EAD0
:10D48000000200F0B986A37A03F003030AB143F067
:10D49000040343F008039A10082BA27200F23087AD
:10D4A000072B81F0EC80032B01F0238141F21A81DC
:10D4B000042B00F03087062B7FF43AADE368023B83
:10D4C000E36036E5019A03231370FFF7B0B941F624
:10D4D000D8734DF64851C2F20001C2F2010309228D
:10D4E0001B780A7072B69B00E36062B6237C012B46
:10D4F00041F2A38072B6E36862B6002BB8BF033373
:10D500009B103360FDF7DAFA4FF0010BFEF7BABF5C
:10D5100072B6236861681A780878617A237A0842BB
:10D5200002EA030200F08581A37A03F003030AB143
:10D5300043F0040343F008039A10082BA27200F290
:10D54000AC81072B80F0F484032B00F0F68440F2CA
:10D550003386042B00F0AC81062B7FF432A8E368FD
:10D56000023BE360FFF72EB872B6236861681A7851
:10D570000878617A237A084202EA030200F06B819C
:10D58000A37A03F003030AB143F0040343F0080352
:10D590009A10082BA27200F29081072B80F0F88479
:10D5A000032B00F0FA8440F20F86042B00F09081E8
:10D5B000062B7FF4DEA8E368023BE360FFF7DAB8EE
:10D5C00072B6236861681A780878617A237A08420B
:10D5D00002EA030200F04881A37A03F00303002A61
:10D5E00041F0808143F008039A10082BA27200F2E8
:10D5F0004481072B80F0B784032B00F0B98440F2FC
:10D600001D86042B00F04481062B7FF4C9A8E36833
:10D61000023BE360FFF7C5B872B6236861681A7809
:10D620000878617A237A084202EA030200F00A814C
:10D63000A37A03F003030AB143F0040343F00803A1
:10D640009A10082BA27200F24881072B80F0808488
:10D65000032B00F0928440F2E985042B00F048810E
:10D66000062B7EF497AFE368023BE360FEF793BFBF
:10D6700072B6236861681A780878617A237A08425A
:10D6800002EA030200F09581A37A03F003030AB1D2
:10D6900043F0040343F008039A10082BA27200F22F
:10D6A0007482072B80F07086032B00F0628640F2B4
:10D6B000A286042B00F07482062B7EF475AFE3681B
:10D6C000023BE360FEF771BF00000C4200FEFF4624
:10D6D00000FEFFC60E74DA400000004F0000A042BA
:10D6E0004656153872B6236861681A780878617AE8
:10D6F000237A084202EA030200F05281A37A03F07F
:10D7000003030AB143F0040343F008039A10082B03
:10D71000A27200F24A82072B80F00E86032B00F0E3
:10D72000388640F26186042B00F04A82062B7FF493
:10D730002AA8E368023BE360FFF726B84FF43742BC
:10D74000C5F66D324BE50023C7F6FF73D361ECE5F8
:10D750000023C7F6FF73B6E5196A8E4540F2CC8107
:10D76000DA8BC3F820E0824238BFD883FFF70BBBC7
:10D770000023C7F6FF733BE6D3680233D360FEF79E
:10D7800066BF0D2B3FF434AC0E2B7EF45FAFD36835
:10D790000133D360FEF75BBF40F2685BC2F2010B5E
:10D7A0009BF80030002B40F0768472B6E36062B6DE
:10D7B000FFF75DB872B60023E36062B6FFF75FBAA9
:10D7C000012BE4D0022B3FF413ACFEF73FBF41F630
:10D7D00019634DF64851C2F20103C2F2000105225D
:10D7E0001B780A70FFF711BA41F61863C2F2010301
:10D7F0004DF6485108221B78C2F20001FFF73FB9ED
:10D800004DF63C534DF64851C2F20003C2F20001FE
:10D810001B780A70FFF7F9B945F27A5245F27B5B43
:10D82000C0F21702C0F2170BFFF735BB46F6FF73C5
:10D830004BE4A37A03F00303002A3FF47DAE43F0E8
:10D84000040379E6A37A03F00303002A3FF4F8AE59
:10D8500043F00403F4E6A37A03F00303002A3FF441
:10D8600097AE43F0040393E6A37A03F00303002A80
:10D870003FF4BAAE43F00403B6E60C2B00F0788315
:10D8800000F26B83092B3FF4C2AE0B2B7EF488AF02
:10D89000E368013BE360FEF784BF0C2B00F04D838F
:10D8A00000F24083092B3FF45AAE0B2B7EF489AE75
:10D8B000E368013BE360FEF785BE0C2B00F06D834F
:10D8C00000F26083092B3FF476AE0B2B7EF451AF50
:10D8D000E368013BE360FEF74DBF0C2B00F04D8386
:10D8E00000F23083092B3FF4BEAE0B2B7EF452AE18
:10D8F000E368013BE360FEF74EBE41F6D853C2F247
:10D9000001034FF480325A621FED8E0A5FED8E9A4A
:10D9100000229A6111F0C8FF1FED907A5FED907AB6
:10D92000F2EE046AA0EE267A27EE270A60EE297A44
:10D93000FDEEE77A17EE90BA11F046FD20EE290AC7
:10D94000FDEEC07A17EE902AFFF7A5BA01204FF03E
:10D95000000EFFF707BA72B60023E36062B6FFF766
:10D96000C7B90023FFF7B1BB72B60023E36062B60C
:10D97000FFF7F3BB72B60023E36062B6FFF771BB3B
:10D9800072B60023E36062B667E472B60023E36018
:10D9900062B6FBE472B60023E36062B6FFF72DBA0D
:10D9A000A37A03F00303002A3FF4B0AE43F004036C
:10D9B000ACE6A37A03F00303002A3FF46DAE43F014
:10D9C000040369E672B658F80C2C6368107819786D
:10D9D000637A227A194202EA000200F04183A37AB4
:10D9E00003F003030AB143F0040343F008039A1061
:10D9F000082BA27200F22A84072B80F0F685032BF5
:10DA000000F0FF8540F2F685042B00F02A84062BF7
:10DA10007FF4A9A8E368023BE360FFF7A5B872B6FC
:10DA200058F80C2C636810781978637A227A1942B6
:10DA300002EA000200F05383A37A03F003030AB161
:10DA400043F0040343F008039A10082BA27200F27B
:10DA5000C383072B80F0E085032B00F0E98540F2BB
:10DA6000E085042B00F0C383062B7FF463A8E368F2
:10DA7000023BE360FFF75FB872B658F80C2C63689E
:10DA800010781978637A227A194202EA000200F0CB
:10DA90001D83A37A03F00303002A40F0358743F087
:10DAA00008039A10082BA27200F2B083072B80F0B3
:10DAB000D085032B00F08E8540F28585042B00F085
:10DAC000B083062B7EF41BAFE368023BE360FEF7F6
:10DAD00017BF4CF6D042C0F6CC42FFF780BB002304
:10DAE000C8F201030AE40023C8F20103FFF7EBBB0D
:10DAF0000023C8F201037BE49107C3F820E006D5B8
:10DB0000596A7F31C9090131884238BF0846510737
:10DB100006D5996A7F31C9090131884238BF084664
:10DB2000110706D5D96A7F31C9090131884238BF4A
:10DB30000846D10606D5196B7F31C90901318842E3
:10DB400038BF0846910606D5596B7F31C9090131A6
:10DB5000884238BF0846510606D5996B7F31C909FE
:10DB60000131884238BF0846D20906D0DA6B7F32CD
:10DB7000D2090132904238BF1046D883FFF703B96B
:10DB80000023C8F20103FFF7D0BB0C2B00F0F18398
:10DB900000F2F483092B3FF492AD0B2B7EF404AD1D
:10DBA000E368013BE360FEF700BD0C2B00F0F1835E
:10DBB00000F2BC83092B3FF4BCAD0B2B7EF4E3AD2C
:10DBC000E368013BE360FEF7DFBD0EF17F00C009B3
:10DBD0000130FFF7C7B872B6236861681A78087811
:10DBE000617A237A084202EA030200F04E83A37AA4
:10DBF00003F003030AB143F0040343F008039A104F
:10DC0000082BA27200F25683072B80F07D85032B30
:10DC100000F0868540F27D85042B00F05683062BAC
:10DC20007FF410A8E368023BE360FFF70CB872B61C
:10DC3000236861681A780878617A237A084202EAD0
:10DC4000030200F01983A37A03F003030AB143F03F
:10DC5000040343F008039A10082BA27200F23A83DF
:10DC6000072B80F01785032B00F0378540F22E85B7
:10DC7000042B00F03A83062B7FF406A8E368023BEE
:10DC8000E360FFF702B872B6236861681A78087813
:10DC9000617A237A084202EA030200F05B83A37AE6
:10DCA00003F003030AB143F0040343F008039A109E
:10DCB000082BA27200F28883072B80F0D584032BF7
:10DCC00000F03A8540F23185042B00F08883062B62
:10DCD0007EF4B2ADE368023BE360FEF7AEBD72B620
:10DCE00094E80C0010781978637A227A194202EAD3
:10DCF000000200F02683A37A03F003030AB143F085
:10DD0000040343F008039A10082BA27200F2468322
:10DD1000072B80F0CA84032B00F0D38440F2CA841E
:10DD2000042B00F04683062B7EF4A6ADE368023B8D
:10DD3000E360FEF7A2BD72B60023E36062B69BF813
:10DD400000300133DBB218468BF8003002F0ACF93A
:10DD5000FEF78DBD72B658F80C2C636810781978F0
:10DD6000637A227A194202EA000200F05D83A37A04
:10DD700003F003030AB143F0040343F008039A10CD
:10DD8000082BA27200F26B83072B80F07A85032B9D
:10DD900000F06C8540F26385042B00F06B83062B4A
:10DDA0007FF4F4A8E368023BE360FFF7F0B872B6D3
:10DDB00058F80C2C636810781978637A227A194223
:10DDC00002EA000200F02783A37A03F003030AB1FA
:10DDD00043F0040343F008039A10082BA27200F2E8
:10DDE000A283072B80F0B384032B00F0BC8440F2A5
:10DDF000B384042B00F0A283062B7EF47BACE36893
:10DE0000023BE360FEF777BC72B658F80C2C6368EF
:10DE100010781978637A227A194202EA000200F037
:10DE2000F182A37A03F003030AB143F0040343F041
:10DE300008039A10082BA27200F22183072B80F0AE
:10DE40009D84032B00F0B68440F2AD84042B00F0D7
:10DE50002183062B7FF4B6A8E368023BE360FFF75B
:10DE6000B2B872B62046F6F70DF8FEF7D7BE72B616
:10DE700094E8090090F800C093F800E0637A207AF3
:10DE80001EEA030F0CEA000000F0E082A37A03F020
:10DE9000030308B143F0040343F008039810082B70
:10DEA000A07200F2FC82072B80F07384032B00F039
:10DEB000758440F20785042B00F0FC82062B7EF46B
:10DEC000D0AEE368023BE360FEF7CCBE72B62368D7
:10DED00061681A780878617A237A084202EA0302B4
:10DEE00000F0AB82A37A03F003030AB143F004030A
:10DEF00043F008039A10082BA27200F2FB82072B52
:10DF000080F08384032B00F0858440F2C684042BC8
:10DF100000F0FB82062B7EF499ACE368023BE360E1
:10DF2000FEF795BC0D2B3FF4C3AC0E2B7EF449AB32
:10DF3000E3680133E360FEF745BBE3680233E36067
:10DF4000FEF740BB0D2B3FF4D3AC0E2B7EF422AB7F
:10DF5000E3680133E360FEF71EBB0D2B3FF498AC82
:10DF60000E2B7EF41DACE3680133E360FEF719BCB1
:10DF7000E3680233E360FEF714BCE3680233E36056
:10DF8000FEF709BB0D2B3FF4A3AC0E2B7EF4F1ABD7
:10DF9000E3680133E360FEF7EDBBE3680233E3605F
:10DFA000FEF7E8BB72B6236861681A780878617A70
:10DFB000237A084202EA030200F08182A37A03F086
:10DFC00003030AB143F0040343F008039A10082B3B
:10DFD000A27200F2C882072B80F03784032B00F076
:10DFE000398440F25384042B00F0C882062B7FF45E
:10DFF000B9A8E368023BE360FFF7B5B872B62368DF
:10E0000061681A780878617A237A084202EA030282
:10E0100000F05E82A37A03F003030AB143F0040325
:10E0200043F008039A10082BA27200F2AC82072B6F
:10E0300080F00084032B00F0F28340F23584042B3F
:10E0400000F0AC82062B7EF4DDAEE368023BE360B9
:10E05000FEF7D9BE72B62046F5F714FFFEF7EFBF04
:10E06000A37A03F00303002A3FF4C1AC43F0040396
:10E07000BDE472B62046F5F705FFFEF7F7BF72B6AE
:10E080002046F5F7FFFEFFF756B872B62046F5F7C3
:10E09000F9FEFEF71BBE72B67C23E36062B69BF806
:10E0A0000030013BDBB218468BF8003001F0FCFF7A
:10E0B000FEF7DDBB72B62046F5F7E4FEFEF71DBEA7
:10E0C00072B62046F5F7DEFEFFF765B9A37A03F0D6
:10E0D0000303002A3FF4E5AC43F00403E1E4A37A30
:10E0E00003F00303002A3FF4AFAC43F00403ABE4B6
:10E0F00072B62046F5F7C6FEFFF79DB872B6204609
:10E10000F5F7C0FEFFF7AEB872B6236861681A78FB
:10E110000878617A237A084202EA030200F0FA8161
:10E12000A37A03F003030AB143F0040343F00803A6
:10E130009A10082BA27200F20682072B80F05583FA
:10E14000032B00F0578340F2B683042B00F00682C5
:10E15000062B7FF409A9E368023BE360FFF705B9EA
:10E1600072B6236861681A780878617A237A08425F
:10E1700002EA030200F0B581A37A03F003030AB1B7
:10E1800043F0040343F008039A10082BA27200F234
:10E190000A82072B80F01983032B00F01B8340F2C7
:10E1A0009983042B00F00A82062B7EF414AEE368F8
:10E1B000023BE360FEF710BE012B3FF4B9AE022B29
:10E1C0003FF476ABFEF7FDB9012B3FF4E1AE022B35
:10E1D0003FF47EABFEF7CDBA0C2B00F0298200F2A3
:10E1E0001582092B3FF443AC0B2B7EF4A3ACE36800
:10E1F000013BE360FEF79FBCA37A03F00303002A10
:10E200003FF449A943F00403FFF745B90C2B00F094
:10E21000E18100F21882092B3FF456AC0B2B7EF4FF
:10E220006EABE368013BE360FEF76ABB012B3FF492
:10E230008FAE022B3FF45CABFEF7ACB9012B3FF481
:10E2400092AE022B3FF424ABFEF7AABA0C2B00F0DF
:10E25000D88100F2C481092B3FF4DCAB0B2B7EF498
:10E2600082ACE368013BE360FEF77EBC72B62046F9
:10E27000F5F708FEFEF70DBCA37A03F00303002AAE
:10E280003FF4E9AC43F00403E5E4A37A03F00303AD
:10E29000002A3FF4B4AC43F00403B0E472B6204665
:10E2A000F5F7F0FDFEF7D5BE72B62046F5F7EAFDAC
:10E2B000FEF7CBBF0C2B00F0338200F21F82092B3C
:10E2C0003FF4B0AC0B2B7EF4BDACE368013BE360E4
:10E2D000FEF7B9BC0C2B00F0008200F2D581092BAF
:10E2E0003FF4CCAC0B2B7EF4CFACE368013BE36096
:10E2F000FEF7CBBC72B62046F5F7C4FDFEF775BD40
:10E300000C2B00F0F68100F2B481092B3FF4D6A863
:10E310000B2B7EF40DAEE368013BE360FEF709BE14
:10E3200072B62046F5F7AEFDFEF7DABC0D2B3FF4D2
:10E3300047AC0E2B7EF427AAE3680133E360FEF7B7
:10E3400023BAA37A03F00303002A3FF4DCAC43F0C2
:10E350000403D8E4A37A03F00303002A3FF4A7AC34
:10E3600043F00403A3E472B62046F5F78BFDFEF7F5
:10E37000ECBEE3680233E360FEF717B90D2B3FF400
:10E380000FAC0E2B7EF410A9E3680133E360FEF7B7
:10E390000CB9E3680233E360FEF7F6B90C2B00F02A
:10E3A000908100F27C81092B3FF4C0AC0B2B7EF4F2
:10E3B00063AAE368013BE360FEF75FBA72B62046EA
:10E3C000F5F760FDFEF7DABF0C2B00F0B58100F227
:10E3D0004581092B3FF47EAC0B2B7EF42DAAE3681C
:10E3E000013BE360FEF729BA012BA5D0022B3FF4D5
:10E3F000E7ABFEF7C8B9012BC6D0022B3FF4D0AB78
:10E40000FEF7D2B8A37A03F00303002A3FF411AD5C
:10E4100043F004030DE5A37A03F00303002A3FF45D
:10E42000DBAC43F00403D7E4A37A03F00303002A30
:10E430003FF4A5AC43F00403A1E4A37A03F0030383
:10E44000002A3FF457AD43F0040353E5A37A03F0E9
:10E45000030300283FF422AD43F004031EE50C2B18
:10E4600000F0048200F20782092B3FF49BAC0B2BD7
:10E470007EF48CADE368013BE360FEF788BD0C2BB6
:10E4800000F0988100F27481092B3FF4E5AC0B2B6E
:10E490007EF498ADE368013BE360FEF794BD0C2B7E
:10E4A00000F07C8100F26F81092B3FF40AAD0B2B49
:10E4B0007EF4D7ABE368013BE360FEF7D3BBA37AFE
:10E4C00003F00303002A3FF481AD43F004037DE52C
:10E4D000A37A03F00303002A3FF4A4AD43F004033E
:10E4E000A0E5A37A03F00303002A3FF44DAE43F006
:10E4F000040349E60C2B00F08D8100F28081092B8A
:10E500003FF40BAD0B2B7EF4A1A9E368013BE36064
:10E51000FEF79DB9A37A03F00303002A3FF408AE87
:10E5200043F0040304E60C2B00F01D8100F2098186
:10E53000092B3FF464AC0B2B7EF4DCA8E368013BB1
:10E54000E360FEF7D8B80C2B00F0548100F247814D
:10E55000092B3FF400AE0B2B7EF406AFE368013BC2
:10E56000E360FEF702BF0C2B00F0748100F26781BC
:10E57000092B3FF43EAD0B2B7EF4F4ADE368013B79
:10E58000E360FEF7F0BD0C2B00F0498100F24C81F6
:10E59000092B3FF45AAD0B2B7EF434ACE368013BFE
:10E5A000E360FEF730BC0C2B00F0148100F2078111
:10E5B000092B3FF4FCAD0B2B7EF40DACE368013B63
:10E5C000E360FEF709BC012B43D0022B3FF429AED8
:10E5D000FEF795B9E3680233E360FEF791B90D2BBE
:10E5E0003FF43FAE0E2B7EF4BEAAE3680133E36036
:10E5F000FEF7BABA012BF8D0022B3FF432AEFEF789
:10E60000B2BAE3680233E360FEF7AEBA0D2B3FF413
:10E61000EEAD0E2B7EF48EAAE3680133E360FEF7C5
:10E620008ABA012BF8D0022B3FF4E1ADFEF782BA93
:10E63000E3680233E360FEF77EBA72B62046F5F770
:10E6400021FCFEF758BF0D2B3FF4EBAD0E2B7EF4F3
:10E6500056A9E3680133E360FEF752B90D2B3FF48E
:10E66000BEAE0E2B7EF4E8A8E3680133E360FEF74C
:10E67000E4B80D2B3FF44FAE0E2B7EF459ACE3689B
:10E680000133E360FEF755BC0D2B3FF42EAE0E2B8D
:10E690007EF4FAAAE3680133E360FEF7F6BA0D2BC5
:10E6A0003FF487AE0E2B7EF4E7A8E3680133E36006
:10E6B000FEF7E3B8012BF8D0022B3FF47AAEFEF759
:10E6C000DBB8E3680233E360FEF7D7B8012BE1D093
:10E6D000022B3FF40AAEFEF7D7BAE3680233E360D9
:10E6E000FEF7D3BA012BCAD0022B3FF414AEFEF7CB
:10E6F0001FBCE3680233E360FEF71BBC0D2B3FF445
:10E70000E4AD0E2B7EF49EAAE3680133E360FEF7CE
:10E710009ABA012BF8D0022B3FF4D7ADFEF792BA8C
:10E72000E3680233E360FEF78EBA012B9CD0022B24
:10E730003FF455AEFEF780B8E3680233E360FEF7BE
:10E740007CB80D2B3FF4FAAE0E2B7DF4D3AFE3680B
:10E750000133E360FDF7CFBF012BF8D0022B3FF46C
:10E76000EDAEFDF7C7BFE3680233E360FDF7C3BF5B
:10E770000D2B3FF48FAE0E2B7EF424ACE3680133F7
:10E78000E360FEF720BC0D2B3FF494AE0E2B7EF41D
:10E7900068AAE3680133E360FEF764BAE368023312
:10E7A000E360FEF75FBA012BE8D0022B3FF472AEB4
:10E7B000FEF708BCE3680233E360FEF704BC0D2BF0
:10E7C0003FF4FCAE0E2B7EF406ABE3680133E3604E
:10E7D000FEF702BBE3680233E360FEF7FDBA0D2BE0
:10E7E0003FF4BCAE0E2B7EF4BFADE3680133E360B3
:10E7F000FEF7BBBDE3680233E360FEF7B6BD0D2B49
:10E800003FF483AE0E2B7EF421A8E3680133E3606E
:10E81000FEF71DB8E3680233E360FEF718B8E3685B
:10E820000233E360FEF7EFBA0D2B3FF4B7AE0E2BC9
:10E830007EF4E8AAE3680133E360FEF7E4BA0D2B47
:10E840003FF49CAE0E2B7EF48DACE3680133E360A5
:10E85000FEF789BCE3680233E360FEF784BC012B5A
:10E860000FD0022B3FF406AEFEF790BBE3680233F5
:10E87000E360FEF78CBB0D2B3FF4FCAD0E2B7EF45A
:10E8800085ABE3680133E360FEF781BB012BDCD08D
:10E89000022B3FF473AEFEF765BC012BB5D0022B03
:10E8A0003FF433AEFDF7D2BF012BC3D0022B3FF4B0
:10E8B00075AEFEF7A7BA012B97D0022B3FF44EAEF0
:10E8C000FEF752BD012B3FF464AF022B3FF4F2ADD3
:10E8D000FEF7C7B9012B3FF478AF022B3FF46EAEC1
:10E8E000FEF779BA43F00403FEF77CBE45F24663B7
:10E8F000C3F6150300EE103A4FF09E4309EE903A2E
:10E9000027EE800AFFF712B843F00403FFF7C7B8F9
:10E910000023C7F6FF73FEF708BD00BF2DE9F043E3
:10E920002DED028B002708EE101A44F2D43183B08B
:10E93000C0F20201AD22054680F8D97080F8DA7085
:10E9400080F8DB7080F8DC7080F8DD7080F8DE70B5
:10E9500080F8DF7080F8E07080F8E17080F8E27095
:10E9600080F8E37080F8E47080F8E57080F8E67075
:10E9700080F8E77080F8E87080F8CC7080F8CD708F
:10E9800080F8CE70F0300DF083FB102385F89D31B8
:10E9900002F09EFE02F0ECFE03F072FBB8EEC88AB5
:10E9A0002E46B0EE480A03F06FF9B0EE480A03F0C5
:10E9B000B7F9B0EE480A03F093FAB0EE480A02F055
:10E9C0008DFC4FF409700DF0F5FD0446F1F758FD8C
:10E9D000C5F8C0414FF409700DF0ECFD43F27873B7
:10E9E000C0F202030360C5F8C4014FF409700DF0D2
:10E9F000E1FD44F29473C0F20203C5F8BC01036068
:10EA000005F1C0092C464FF425700DF0D3FD80466A
:10EA10000C3401F02DFF44F8048C04F80A7C04F84F
:10EA2000097C04F8087CA1454FF00003EBD195F870
:10EA3000D9209FEDD16ADFEDCF6A85F89E3107EED0
:10EA4000902AB8EEE77A95F8DB20C5F8C43067EE77
:10EA5000067A102067EEA67A4FF40051FCEEE77AB2
:10EA6000C5F8C830CDED017A85F8D23085F8D130BF
:10EA700085F8D03085F8CF3085F8CE3085F8CD30A8
:10EA800085F8CC3085F89D019DF80430C5F8C0109C
:10EA90000AB185F8CC3095F8DA200AB185F8CD3086
:10EAA00095F8DC200AB185F8CE3095F8E1309FED7D
:10EAB000B26ADFEDB06A95F8E31007EE903AB8EE6F
:10EAC000E77A67EE067A67EEA67AFCEEE77ACDED96
:10EAD000017A9DF8043031B195F8CC10994238BFD5
:10EAE000194685F8CC1095F8E21031B195F8CD10A3
:10EAF000994238BF194685F8CD1095F8E40030B139
:10EB000095F8CE108B4238BF0B4685F8CE3095F87D
:10EB1000DD309FED996ADFED976A95F8DF1007EE1B
:10EB2000903AB8EEE77A67EE067A67EEA67AFCEEE0
:10EB3000E77ACDED017A9DF8043031B195F8CC102B
:10EB4000994238BF194685F8CC1095F8DE1031B1DE
:10EB500095F8CD10994238BF194685F8CD1095F833
:10EB6000E01031B195F8CE40A34238BF234685F876
:10EB7000CE3095F8E5309FED806ADFED7E6A95F83E
:10EB8000E74007EE903AB8EEE77A67EE067A67EE6E
:10EB9000A67AFCEEE77ACDED017A9DF8043034B127
:10EBA00095F8CC409C4238BF1C4685F8CC4095F87F
:10EBB000E64034B195F8CD409C4238BF1C4685F8FC
:10EBC000CD4095F8E84034B195F8CE70BB4238BFDF
:10EBD0003B4685F8CE302AB921B918B914B97F233C
:10EBE00085F8CE303F23002485F8D830C5F8D440CE
:10EBF00005F2791105F5D27003F0A8F895F8A03167
:10EC00000BB185F8A04195F8A231002485F89F4109
:10EC1000002B00F0F080D5F8BC3185F8A241C5F892
:10EC2000EC3033793BB1B368B47018463471F4708A
:10EC30000BB102F039FB0C36B145F2D195F8D93061
:10EC40009FED4D6A95F8DB1007EE903A95F8D230BB
:10EC5000B8EEE77A06EE903A67EE067AF8EEE66AE4
:10EC6000002267EEA67A85F8CE20FCEEE77A85F8DA
:10EC7000CD20CDED017A9DF8043085F8CC2009B186
:10EC800085F8CC3095F8DA200AB185F8CD3095F8C2
:10EC9000DC200AB185F8CE3095F8E1309FED366A78
:10ECA00095F8E31007EE903A95F8D030B8EEE77A91
:10ECB00006EE903A67EE067AF8EEE66A67EEA67A16
:10ECC000FCEEE77ACDED017A9DF8043031B195F88C
:10ECD000CC10994238BF194685F8CC1095F8E2104F
:10ECE00031B195F8CD10994238BF194685F8CD104D
:10ECF00095F8E40030B195F8CE108B4238BF0B4642
:10ED000085F8CE3095F8DD309FED1B6A95F8DF1061
:10ED100007EE903A95F8D130B8EEE77A06EE903AE1
:10ED200067EE067AF8EEE66A67EEA67AFCEEE77A18
:10ED3000CDED017A9DF8043031B195F8CC109942AF
:10ED400038BF194685F8CC1095F8DE1031B195F82A
:10ED5000CD10994238BF194685F8CD1095F8E010CE
:10ED600061B195F8CE40A34238BF234685F8CE3036
:10ED700004E000BF000000000AD7233C95F8E5300E
:10ED80001FED036A95F8E74007EE903A95F8CF300B
:10ED9000B8EEE77A06EE903A67EE067AF8EEE66AA3
:10EDA00067EEA67AFCEEE77ACDED017A9DF80430A5
:10EDB00034B195F8CC409C4238BF1C4685F8CC4015
:10EDC00095F8E64034B195F8CD409C4238BF1C46DA
:10EDD00085F8CD4095F8E84034B195F8CE60B3425F
:10EDE00038BF334685F8CE302AB921B918B914B9DD
:10EDF0007F2385F8CE30284603B0BDEC028BBDE8FA
:10EE0000F08300BF2DE9F04F90F8A131CDB0074657
:10EE1000069104923BB390F89D31DBB1002400F1E0
:10EE2000F00503E00134A4B2A34213D904EB440279
:10EE300007EB820108790028F4D04B78886817F82E
:10EE40002220294602F034F8013497F89D31A4B20B
:10EE5000A342EBD807F2791107F5D27002F076FFE2
:10EE6000002387F8A131069B002B00F086800DF16E
:10EE70002F0323F00F03039340F22006A3F1040BAA
:10EE800003F1FC0407F5D273C2F2010607934FF0B9
:10EE9000000A049B0AF10042013A03EB42020021FE
:10EEA0005B4643F8041F9C4222F8021FF9D1079DDC
:10EEB000284602F08DFF8046284602F0E3FF97F8CF
:10EEC0009D118146002951D0049BCDF814A003EB7D
:10EED0004A0307F1C002002502929A4603E0013579
:10EEE000EDB28D4240D205EB450307EB83031A795F
:10EEF000002AF4D09868029B0093424603994B463F
:10EF000001F08EFE51465A4600200BE0002B02DD38
:10EF1000BEF1000F34DB0FFA8EFE944221F802EBB3
:10EF200010601BD052F8043F1B1123F35723B1F993
:10EF300000C0BCF1000F0CEB630EE7DCEBD0002B44
:10EF4000E9DABEF1000FE6DD33684FF0000E013361
:10EF50009442336021F802EB1060E3D197F89D11E1
:10EF60000135EDB28D42BED3DDF814A0069B0AF147
:10EF7000400A1FFA8AFA53458BD84DB0BDE8F08F8E
:10EF80003368013333604FF0FF3EC6E72DE9F843A5
:10EF9000054690F8803190F89D61002A00F0D680F7
:10EFA000183BCF1890F89E81FFB2002E00F0C5806C
:10EFB0004FEA480909EB080300EB830341469C78BC
:10EFC000CE46002C00F09380002403E08378002BD1
:10EFD00000F08D800131013491FBF6F306FB131133
:10EFE000E4B24FEA410E0EEB0100B44205EB8000A3
:10EFF0005FFA81F8EAD195F8A031002B6ED095F830
:10F000009D31002B6AD02A79002A40F0CF81012B54
:10F0100064D92A7C002A40F0D781022B5ED02A7F57
:10F02000002A40F0CD81032B58D095F82820002AE3
:10F0300040F0C881042B51D095F83420002A40F0CC
:10F04000B781052B4AD095F84020002A40F0B281C4
:10F05000062B43D095F84C20002A40F0AD81072BB9
:10F060003CD095F85820002A40F0A881082B35D0D4
:10F0700095F86420002A40F0AB81092B2ED095F83A
:10F080007020002A40F0A6810A2B27D095F87C201A
:10F09000002A40F0A1810B2B20D095F88820002A6F
:10F0A00040F09C810C2B19D095F89420002A40F058
:10F0B00097810D2B12D095F8A020002A40F0928164
:10F0C0000E2B0BD095F8AC20002A40F07F810F2B3F
:10F0D00004D095F8B830002B40F032814FEA48094F
:10F0E000C84405EB880501232B71BDE8F8838E44E5
:10F0F0004FEA8E0E013105EB0E0991FBF6F306FB8C
:10F10000131685F89E6105F80E7089F8012095F8B0
:10F110009F3189F803300121134689F80210D9F88C
:10F1200008003A4605F1F00101F0BCFB95F8783192
:10F13000002B78D1002C7FF45EAF05F5D27002F081
:10F14000C7FE95F8A031002BC8D058E7183BCF1860
:10F15000FBB2002E65D00178994200F0BB80012EF1
:10F160005FD92A7B9A4200F0AF80022E59D02A7EC6
:10F170009A4200F0A380032E53D095F824209A429F
:10F1800000F09580042E4CD095F830209A4200F083
:10F190008780052E45D095F83C209A427AD0062EDD
:10F1A0003FD095F848209A426ED0072E39D095F876
:10F1B00054209A4262D0082E33D095F860209A42AB
:10F1C00056D0092E2DD095F86C209A424AD00A2E9E
:10F1D00027D095F878209A423ED00B2E21D095F872
:10F1E00084209A4232D00C2E1BD095F890209A425F
:10F1F00026D00D2E15D095F89C209A421AD00E2EAE
:10F200000FD095F8A8209A4200F093800F2E08D0D6
:10F2100095F8B4209A4204D195F8B630002B40F00E
:10F22000A780BDE8F883D9F8080002F03DF8002C6B
:10F2300083D0E0E695F89E20002AE0D00D2798E0E4
:10F2400095F89220002AD4D00C2792E095F88620D9
:10F25000002AC8D00B278CE095F87A20002ABCD071
:10F260000A2786E095F86E20002AB0D0092780E0B2
:10F2700095F86220002AA4D008277AE095F8562055
:10F28000002A98D0072774E095F84A20002A8CD0ED
:10F2900006276EE095F83E20002A80D0052768E01A
:10F2A00095F83220002A3FF474AF042761E095F806
:10F2B0002620002A3FF466AF03275AE0AA7E002AE0
:10F2C0003FF459AF022754E0AA7B002A3FF44DAF28
:10F2D00001274EE0817800293FF441AF8270174644
:10F2E000804695F8A031E3B14FF0000E73467146A9
:10F2F0004FF0FF3203EB430305EB8304481CA47873
:10F300002CB115F823309342C4BF5AB28E4641B295
:10F31000B1420B46EEDB013203D098F80430002BEB
:10F3200062D195F89F31C3B3012388F80330BDE85B
:10F33000F88395F8AA20002A3FF468AF0E2718E05A
:10F340000F2303EB43039B00EA189178C9B1EB5CF0
:10F35000BB42BFF466AF4FEA480909EB080305EB6F
:10F360008303002111719868916801F049FFB7E6A5
:10F370000F2707EB470805EB8808002388F80230C1
:10F38000AFE74FEA480909EB080305EB8303117166
:10F390009868916801F054FFA2E607EB470205EB7D
:10F3A0008205A868BDE8F84301F06EBD0023C8E7F8
:10F3B0000423C6E70523C4E70623C2E70723C0E703
:10F3C0000223BEE70323BCE70123BAE70E23B8E715
:10F3D0000823B6E70923B4E70A23B2E70B23B0E713
:10F3E0000C23AEE70D23ACE70EEB4E0E07EB470206
:10F3F00005EB8E03002105EB820288F80410012141
:10F4000019719868916801F0FBFE8AE7F8B590F8E9
:10F41000803190F89D71183B1944002F63D0037818
:10F42000C9B28B4260D0012F5DD9037B8B4200F0C3
:10F43000EA80022F57D0037E8B4200F0DE80032F3C
:10F4400051D090F824308B4200F0D080042F4AD065
:10F4500090F830308B4200F0C280052F43D090F8F6
:10F460003C308B4200F0B480062F3CD090F84830FE
:10F470008B4200F0A680072F35D090F854308B4295
:10F4800000F09880082F2ED090F860308B4200F06A
:10F490008A80092F27D090F86C308B427CD00A2FBD
:10F4A00021D090F878308B4270D00B2F1BD090F881
:10F4B00084308B4264D00C2F15D090F890308B4262
:10F4C00058D00D2F0FD090F89C308B424CD00E2F7F
:10F4D00009D090F8A8308B4240D00F2F03D090F87D
:10F4E000B4308B422ED0F8BD8378002B9BD0002502
:10F4F0008570064690F8A0310446E3B100231A4611
:10F500009C464FF0FF3E03EB430304EB8300511C8A
:10F51000807830B114F823307345C4BF4FFA83FEAE
:10F5200094464AB2BA421346EDDBBEF1FF3F02D029
:10F530003379002B76D194F89F31002B69D00123C9
:10F54000F370F8BD90F8B630002BCCD00F2505EB4A
:10F55000450600EB86060023B370CBE790F8AA308F
:10F56000002BBAD00E25F2E790F89E30002BAED0DB
:10F570000D25ECE790F89230002BA2D00C25E6E7A1
:10F5800090F88630002B96D00B25E0E790F87A3083
:10F59000002B8AD00A25DAE790F86E30002B3FF472
:10F5A0007EAF0925D3E790F86230002B3FF471AFAE
:10F5B0000825CCE790F85630002B3FF463AF0725C1
:10F5C000C5E790F84A30002B3FF455AF0625BEE75B
:10F5D00090F83E30002B3FF447AF0525B7E790F891
:10F5E0003230002B3FF439AF0425B0E790F82630D5
:10F5F000002B3FF42BAF0325A9E7837E002B3FF4BC
:10F600001EAF0225A3E7837B002B3FF412AF012539
:10F610009DE705EB450504EB8500BDE8F8408068F3
:10F6200001F032BC0CEB4C0C05EB450204EB8C03F7
:10F63000002104EB820231710121197198689168EF
:10F6400001F0DEFD77E700BF90F8A0318B4218BFD4
:10F6500080F8A011704700BF90F89F318B4218BF0F
:10F6600080F89F11704700BF90F89F01704700BF5E
:10F6700070B5044600F1C006002523793BB1A368AC
:10F68000A57018462571E5700BB101F00DFE0C3424
:10F69000B442F2D170BD00BF90F8D9309FED6C6AD2
:10F6A000DFED6C6A90F8DB1007EE903AB8EEE77A7F
:10F6B00070B467EE067A83B067EEA67A0023FCEE9C
:10F6C000E77A4FF40052CDED017AC0F8C020C0F8BF
:10F6D000C4309DF80420C0F8C83080F8D23080F8DB
:10F6E000D13080F8D03080F8CF3080F8CE3080F83C
:10F6F000CD3080F8CC3009B180F8CC2090F8DA30E9
:10F700000BB180F8CD2090F8DC1009B180F8CE2044
:10F7100090F8E1309FED4E6ADFED4E6A90F8E320FD
:10F7200007EE903AB8EEE77A67EE067A67EEA67AC9
:10F73000FCEEE77ACDED017A9DF8043032B190F815
:10F74000CC209A4238BF1A4680F8CC2090F8E220AC
:10F7500032B190F8CD209A4238BF1A4680F8CD20B9
:10F7600090F8E44034B190F8CE20934238BF13466D
:10F7700080F8CE3090F8DD309FED356ADFED356AE8
:10F7800090F8DF2007EE903AB8EEE77A67EE067A57
:10F7900067EEA67AFCEEE77ACDED017A9DF80430AB
:10F7A00032B190F8CC209A4238BF1A4680F8CC206B
:10F7B00090F8DE2032B190F8CD209A4238BF1A4638
:10F7C00080F8CD2090F8E02032B190F8CE50AB42D6
:10F7D00038BF2B4680F8CE3090F8E5309FED1C6A9C
:10F7E000DFED1C6A90F8E75007EE903AB8EEE77A42
:10F7F00067EE067A67EEA67AFCEEE77ACDED017A3F
:10F800009DF8043035B190F8CC509D4238BF1D466C
:10F8100080F8CC5090F8E65035B190F8CD509D422C
:10F8200038BF1D4680F8CD5090F8E85035B190F8BB
:10F83000CE60B34238BF334680F8CE3029B922B902
:10F840001CB915B97F2380F8CE3003B070BC704767
:10F850000AD7233C0000000003791BB18378002BFA
:10F8600040F09A80037C1BB1837B002B40F0918099
:10F87000037F1BB1837E002B40F0888090F82830F6
:10F880001BB190F82630002B7CD190F834301BB19E
:10F8900090F83230002B71D190F840301BB190F8C5
:10F8A0003E30002B66D190F84C301BB190F84A30B6
:10F8B000002B5BD190F858301BB190F85630002BDC
:10F8C00050D190F864301BB190F86230002B45D1D4
:10F8D00090F8703013B190F86E30DBBB90F87C304C
:10F8E00013B190F87A308BBB90F8883013B190F850
:10F8F00086303BBB90F8943013B190F89230EBB95E
:10F9000090F8A03013B190F89E309BB990F8AC30CD
:10F9100013B190F8AA304BB990F8B8302BB190F8E9
:10F92000B63013B1002380F8B6307047002380F85A
:10F93000AA30F1E7002380F89E30E7E7002380F843
:10F940009230DDE7002380F88630D3E7002380F88B
:10F950007A30C9E7002380F86E30BFE7002380F8D3
:10F960006230B5E7002380F85630AAE7002380F81C
:10F970004A309FE7002380F83E3094E7002380F868
:10F98000323089E7002380F826307EE70023837633
:10F9900074E7002383736BE70023837062E700BF83
:10F9A00090F89D01704700BF2DE9F04100F1F00390
:10F9B00084B004460A4600F5B775106856685E6064
:10F9C00018601089967A9E721881D07A00F003062A
:10F9D000C0F38100DE721873107BC0F3C30600F021
:10F9E00007001E755873507BC0F3820600F00300B9
:10F9F000DE739873907B1874D07BC0F3440600F0DC
:10FA000001009E745874107CD87415339D4202F125
:10FA10001102D2D10B460A4653F8660FDFEDD25AD7
:10FA20005B68C4F86E016B6091F86E3003F01F03E1
:10FA300084F8763191F86F30C3F3C00003F0070308
:10FA400084F8780184F877310B6FC4F8793191F834
:10FA50007430C3F30115C3F3420003F0010384F8CB
:10FA60007F5184F87E0184F87D3191F8753084F8F7
:10FA7000803152F8761F04F281175368C4F881115F
:10FA80007B6013893B8163220123072184F88B313A
:10FA900084F88C3184F88D2184F88F2184F89121A9
:10FAA00084F8932184F88E1184F8901184F89211CF
:10FAB00084F8941194F8D01084F8963106EE101A58
:10FAC00094F8D21084F8973106EE901A94F8D11079
:10FAD00084F89831B8EEC66AF8EEE66A07EE101AB6
:10FAE00026EE256A94F8CF1084F8993166EEA56A5F
:10FAF000B8EEC77A07EE901ABCEEC66AFCEEE66A6C
:10FB000027EE257A8DED016ACDED026AF8EEE77AEF
:10FB10009DF804009DF8081084F89A31BCEEC77A6D
:10FB200067EEA57A88428DED037A38BF0846FCEE71
:10FB3000E77A9DF80C10CDED017A884238BF08466F
:10FB40009DF8041084F89B318842C4F8C430C4F88E
:10FB5000C83084F8D92084F8DA3084F8DB3084F8AF
:10FB6000DC3084F8DD2084F8DE3084F8DF3084F87F
:10FB7000E03084F8E12084F8E23084F8E33084F85F
:10FB8000E43084F8E52084F8E63084F8E73084F83F
:10FB9000E830237938BF0846102500213F2284F839
:10FBA000CC0084F89511C4F8D41084F89C5184F8E2
:10FBB000CD0084F8CE0084F8D8201BB1A378002BA8
:10FBC00040F0A381237C1BB1A37B002B40F09A81E2
:10FBD000237F1BB1A37E002B40F0918194F8283045
:10FBE00023B194F82630002B40F0858194F834300E
:10FBF00023B194F83230002B40F0798194F84030F2
:10FC000023B194F83E30002B40F06D8194F84C30D5
:10FC100023B194F84A30002B40F0618194F85830B9
:10FC200023B194F85630002B40F0558194F864309D
:10FC300023B194F86230002B40F0758194F8703055
:10FC400023B194F86E30002B40F0698194F87C3039
:10FC500023B194F87A30002B40F05D8194F888301D
:10FC600023B194F88630002B40F0518194F8943001
:10FC700023B194F89230002B40F05D8194F8A030CD
:10FC800023B194F89E30002B40F0518194F8AC30B1
:10FC900023B194F8AA30002B40F0518194F8B83089
:10FCA00023B194F8B630002B40F01181102384F872
:10FCB0009D31254604F1C00800262B793BB1AB6885
:10FCC000AE7018462E71EE700BB101F0EDFA0C35E6
:10FCD0004545F2D194F8D9309FED246A94F8DB10B1
:10FCE00007EE903A94F8D230B8EEE77A06EE903A02
:10FCF00067EE067AF8EEE66A002267EEA67A84F8E6
:10FD0000CE20FCEEE77A84F8CD20CDED017A9DF887
:10FD1000043084F8CC2009B184F8CC3094F8DA208F
:10FD2000002A40F0288194F8DC200AB184F8CE3013
:10FD300094F8E1309FED0D6A94F8E31007EE903AE5
:10FD400094F8D030B8EEE77A06EE903A67EE067A8D
:10FD5000F8EEE66A67EEA67AFCEEE77ACDED017A78
:10FD60009DF8043004E000BFA3707D3F0AD7233C18
:10FD700031B194F8CC10994238BF194684F8CC10B0
:10FD800094F8E210002940F0EE8094F8E41031B1CC
:10FD900094F8CE00834238BF034684F8CE3094F8FE
:10FDA000DD301FED0E6A94F8DF0007EE903A94F80C
:10FDB000D130B8EEE77A06EE903A67EE067AF8EEC2
:10FDC000E66A67EEA67AFCEEE77ACDED017A9DF859
:10FDD000043030B194F8CC00984238BF184684F80B
:10FDE000CC0094F8DE00002840F0B58094F8E000E4
:10FDF00030B194F8CE50AB4238BF2B4684F8CE30A9
:10FE000094F8E5301FED276A94F8E75007EE903A32
:10FE100094F8CF30B8EEE77A06EE903A67EE067ABD
:10FE2000F8EEE66A67EEA67AFCEEE77ACDED017AA7
:10FE30009DF8043035B194F8CC509D4238BF1D4632
:10FE400084F8CC5094F8E650002D7CD194F8E8501A
:10FE500035B194F8CE60B34238BF334684F8CE3023
:10FE60002AB920B919B915B97F2384F8CE300125F4
:10FE700041F67C700A22394684F8A151C2F2010091
:10FE800013F08CF944F284400721C0F202000EF016
:10FE9000DFFB41F67C70C2F2010013F011F901465C
:10FEA00041F67C70C2F201000EF0D2FB44F28C40AD
:10FEB0000921C0F202000EF0CBFB4EF2C000C2F2EC
:10FEC00000000BF03FFE284604B0BDE8F08100239F
:10FED00084F8B630EAE6002384F85630A6E600231C
:10FEE00084F84A309AE6002384F83E308EE60023F8
:10FEF00084F8323082E6002384F8263076E6002348
:10FF0000A3766BE60023A37362E6A1705AE6002392
:10FF100084F88630AAE6002384F87A309EE600232F
:10FF200084F86E3092E6002384F8623086E600237F
:10FF300084F89E30AAE6002384F892309EE60023DF
:10FF400084F8AA30AAE694F8CD509D4238BF1D46E9
:10FF500084F8CD507AE794F8CD00984238BF18461F
:10FF600084F8CD0042E794F8CD10994238BF194685
:10FF700084F8CD1009E784F8CD30D4E610B50446F6
:10FF800013F09EF801462046BDE810400EF060BB1D
:10FF900010B5044613F094F8014620460EF058FBC5
:10FFA00004464EF2C000C2F200000BF0CBFD20442C
:10FFB00010BD00BF2DE9F04100262F270C468E60B2
:10FFC0000E604E60C1F80B600A2201F8017B80468A
:10FFD00012F034FC204613F073F808EB480540F2A9
:10FFE0003002C2F2010208EB85051544431C275478
:10FFF0002946E01812F0EAFF4EF2C00744F298409A
:020000021000EC
:10000000C2F200072121C0F202000EF021FB3346AC
:100010000A22414638460BF0A7FD44F2BC400A21B3
:10002000C0F202000EF014FB284613F049F8014616
:1000300028460EF00DFB44F278000321C0F20200C6
:100040000EF006FB204613F03BF8014620460EF06A
:10005000FFFA43F65440C0F2020001210EF0F8FA14
:100060003846BDE8F0410BF06DBD00BF10B584B05F
:100070000C460146684612F0A9FF44F294416846D6
:10008000C0F2020113F0BEF828B10146204612F07A
:100090009DFF04B010BD44F2C843C0F2020303CB7D
:1000A0002060616004B010BD2DE9F04194B00446B9
:1000B00004A804F06BFB41F61C60C2F201004FF48F
:1000C000B072002112F0B6FE41F2A463C2F2010345
:1000D0001B7833B904A804F067FB002014B0BDE816
:1000E000F08148F21F53C5F2EB13A3FB04235B0915
:1000F000642000FB1340C0B26946FFF75BFF44F287
:10010000D0401E21C0F202000EF0A2FA684612F0A2
:10011000D7FF014668460EF09BFA43F65440012192
:10012000C0F202000EF094FA4EF2C000C2F20000DB
:100130000BF008FD49F2741101236A460CA8C2F2C3
:10014000010104F0FFFB14AB9DF8344053F8131D7C
:10015000CDF81D105A689E681D7B0E99CDF82120A0
:10016000139B9DF83C20CDF825600CA88DF82950F4
:100170008DF8144006918DF81C200B9304F014FBAD
:1001800004A804F02BFB0028A4D004A804F022FB50
:1001900041F2080398420DD044F2F0401A21C0F217
:1001A00002000EF055FA4EF2C000C2F200000BF051
:1001B000C9FC8FE704A804F059FAF0280DD044F2E6
:1001C0000C501F21C0F202000EF042FA4EF2C000A5
:1001D000C2F200000BF0B6FC7CE704A804F046FA7B
:1001E00043280DD044F22C501C21C0F202000EF026
:1001F0002FFA4EF2C000C2F200000BF0A3FC69E738
:1002000041F2070104A804F0DBFA04A804F02EFA76
:10021000F72806D044F24C50C0F20200FFF7B8FEB7
:1002200058E7032104A804F0CBFA04A804F01EFA4E
:10023000092806D044F26C50C0F20200FFF7A8FE75
:1002400048E741F2060104A804F0BAFA04A804F051
:100250000DFA062146B204A804F0B2FA04A804F08C
:1002600005FA002741F61C6502463C46B846C2F234
:10027000010516E004F0FAF904F07F0108EB8803A9
:1002800008EB43030246A1F1760009282B449CBFEA
:100290005B1803F8762C7F2904BF08F101085FFA88
:1002A00088F80134A4B2D2B2B4F5805F04A8A7EBF9
:1002B0000207DFD144F28C50C0F20200FFF75EFE6D
:1002C00007F07F074EF2C000394600231022C2F229
:1002D00000000BF049FC44F2A050C0F20200FFF70E
:1002E0004DFE4EF2C000002310223146C2F2000043
:1002F0000BF03AFC43F65440C0F20200FFF748FE10
:10030000B7423FF4E7AE44F2A850C0F20200FFF754
:1003100035FE4EF2C000394600231022C2F2000022
:100320000BF022FC44F2C850C0F20200FFF726FE98
:100330004EF2C000314600231022C2F200000BF042
:1003400013FC4EF2C000C2F200000BF0FBFBC1E652
:100350002DE9F04192B002A804F018FA40F2300002
:10036000C2F2010040F21452002112F063FD41F28A
:10037000A463C2F201031C78002C00F09E8040F2BE
:100380003006C2F20106002408E00AA804F00CFAC4
:1003900002A804F023FA002800F08F802F23002504
:1003A0000A220DF10501204601958DF8043012F066
:1003B00045FA49F27411C2F20101012301AA0AA807
:1003C00004F0C0FA9DF82CE00C9D9DF834709DF867
:1003D00036009DF837109DF838209DF839309DF88B
:1003E0003AC09DF835808DF80CE004959DF83BE00F
:1003F0008DF814709DF83D509DF83C708DF81600F6
:100400008DF817109DF83E009DF83F108DF81820CC
:100410008DF819309DF840209DF841308DF81F105F
:100420008DF820208DF81AC08DF81BE08DF81E0085
:100430008DF815808DF81C708DF81D508DF82130C9
:100440000AA8119B099304F0AFF902A804F0C6F9B9
:10045000012202A988B30AA804F0ECFA0AA804F061
:10046000A7F9002891D10AA804F0A0F904EB4405EB
:1004700004EB850535440146284612F0A7FD44F2F9
:10048000D0500C21C0F202000EF0E2F8284612F023
:1004900017FE014628460EF0DBF843F654400121D2
:1004A000C0F202000EF0D4F84EF2C000C2F200001A
:1004B00001340BF047FBE4B267E702A804F074F9DB
:1004C000204612B0BDE8F0812DE9F0470E46904677
:1004D000054604F07FF941F2080398420FD044F238
:1004E000F040C0F202001A210EF0B2F84EF2C00045
:1004F000C2F200000BF026FB0020BDE8F087284682
:1005000004F0B4F8F02805D044F20C50C0F2020018
:100510001F21E9E7284604F0A9F8432805D044F252
:100520002C50C0F202001C21DEE741F207012846F0
:1005300004F046F9284604F099F8F72805D044F26B
:100540004C50C0F202001D21CEE70321284604F0E2
:1005500037F9284604F08AF8092804D044F26C5090
:10056000C0F20200EFE741F20601284604F028F944
:10057000284604F07BF806214FFA80F9284604F05B
:100580001FF906F1010A00244FEACA1AF6012746AC
:10059000284604F06BF8B442C3B2A7EB030704DBB0
:1005A000A31B5445B8BF08F803000134B4F5805FBD
:1005B000EED144F28C501221C0F202000EF048F845
:1005C00007F07F074EF2C000002310223946C2F226
:1005D00000000BF0C9FA44F2A0500421C0F202005E
:1005E0000EF036F84EF2C000002310224946C2F247
:1005F00000000BF0B9FA43F654400121C0F20200AA
:100600000EF026F84EF2C000C2F200000BF09AFA8B
:100610004F4508D140F22C03C2F2010300221A8098
:100620000120BDE8F08744F2A8501F21C0F202006B
:100630000EF00EF84EF2C000394600231022C2F22E
:1006400000000BF091FA44F2C8500621C0F20200FB
:100650000DF0FEFF4EF2C000494600231022C2F208
:1006600000000BF081FA4EF2C000C2F200000BF065
:1006700069FA0020BDE8F08730B541F2A462C2F209
:100680000102B5B01378002B00F09C80044604A84A
:100690000D4604F07BF848F21F53C5F2EB13A3FBA1
:1006A00004235B09642000FB1340C0B26946FFF7D6
:1006B00081FC49F2741101236A4614A8C2F20101B7
:1006C00004F040F934AB9DF8544053F8732DCDF845
:1006D0001D2059689A681B7BCDF82110CDF8252084
:1006E00016999DF85C208DF8293014A81B9B8DF875
:1006F000144006918DF81C200B9304F055F804A8C3
:1007000004F06CF8044600BB44F2E0501021C0F243
:1007100002000DF09DFF684612F0D2FC01466846CB
:100720000DF096FF44F2F450C0F2020008210DF0E3
:100730008FFF4EF2C000C2F200000BF003FA04A8D3
:1007400004F032F8204635B030BDDDF82130DDF858
:100750001D20CDF84130DDF82530CDF84530CDF8FD
:100760003D209DF82930069A8DF849300E929DF86B
:1007700014308DF8343044F674429DF81C308DF8F6
:100780003C30C0F2020205F01F050B9B0C9229467B
:100790000CA814AA1393FFF797FE04460CA804F0C4
:1007A00003F804BB44F210601A21C0F202000DF0FD
:1007B0004FFF4EF2C000C2F200000BF0C3F904A8D4
:1007C00003F0F2FF44F22C601321C0F202000DF09E
:1007D0003FFF4EF2C000C2F200000BF0B3F900245C
:1007E000204635B030BD0A220DF1C6010CA812F02A
:1007F000D5FC44F200600E21C0F202000DF028FF8B
:10080000684612F05DFC014668460DF021FF44F297
:1008100088100221C0F202000DF01AFF05EB8503DB
:1008200041F61C6005EB4305C2F201000544284671
:1008300012F046FC014628460DF00AFF43F65440EC
:100840000121C0F202000DF003FF4EF2C000C2F21F
:1008500000000BF077F941F2E463C2F2010314A93E
:100860001868FFF7A1F8044669E700BF0BF06CBBFE
:100870000022C0F8A421C0F89C21C0F8B421C0F81F
:10088000AC21C0F8C421C0F8BC21C0F8D421C0F804
:10089000CC21C0F8E421C0F8DC21C0F8F421C0F874
:1008A000EC2170472DE9F04F45F255541646C0F241
:1008B000150404FB06F49A4604F142732DED088BEF
:1008C00008EE903A4FF04E530AEE103A4CF2830382
:1008D000CBF6CA6309EE903A43F27A63C3F6AB43B0
:1008E00009EE103A4DF20A73C3F623430BEE103AA9
:1008F0004AF63B23C4F6B83345F256550AEE903A11
:1009000018EE903AC5F2555593B085FB022703F2D5
:1009100031733246A7EBE67744F2886B08EE903AE3
:100920004FEA6A0303958146073F08930C46054644
:10093000C0F2020B0026099190464EE0BAF1000F7A
:1009400000F30F816FF0EE0101FB02F20732D210CB
:1009500000EB0213002F23EAE373627B40F3FF8076
:100960001F2FCCBFC2EB42127A43D21000920AA9C9
:100970000EAA09EB060000F0C9FC627CA37CE17CB6
:10098000207D002A7AD003F0030C4FF0640E40F66D
:1009900078031EFB0C11C0F2440303FB01F307288C
:1009A0004FEAE301C3BF073843F2914343430023B7
:1009B0000B44C5F86C22C5F83032A37B03F0030367
:1009C00044365BF82330C5F85432B6F5CC7F04F1D9
:1009D000150405F1040500F0D480207821796278AF
:1009E00063790A90A0780E910B92A179E2780F9327
:1009F0000C90E379207C0D921193109100F0E0FDB2
:100A0000237AC3EB0803B3F1110200F18680039A45
:100A1000217B94F80AE0103B82FB03C2A2EBE37354
:100A200001B303291ED01F2BDBBF44F21872C0F2A2
:100A30000202FA23D35C03FB0EFE40F2491303FBD0
:100A40000EF301294FEAE33316DD18447F28A8BFCF
:100A50007F20BAF17F0F4FEA4010E27B7FF76EAF45
:100A60000F2171E703FB0EF340F2491202FB03F37F
:100A700001294FEA2333E8DC5B42E6E7B8EEE88A77
:100A8000079028EE0A0A069120EE290A059304929F
:100A90000EF00AFF20EE090AF1EE0C7A80EE277ABA
:100AA0000798059B0699073844F2986E03F01F03D8
:100AB000C0F2020E5EF8233007EE900A27EE087AA5
:100AC000F8EEE77AA7EE278ABDEEC88A18EE102A5C
:100AD0001A441346049A00293FF46BAF07EE901AAC
:100AE000F8EEE77AB7EE000AA7EE8B0A05930EF050
:100AF0005DFFF6EE007AE0EE2A7A17EE900A11F02A
:100B0000B5FA41EC100B0EF01BFB51EC100B11F081
:100B1000B1FD059B049A03444BE7039B94F809C07D
:100B2000C2F10101E27A83FB013EAEEBE17102B357
:100B3000032A1ED01F29DBBF44F2187EC0F2020E2A
:100B4000FA211EF8011040F2491301FB0CF103FBDE
:100B500001F3DB13012A3FF778AF5B4275E7002210
:100B600004E744F24063C0F202030899595CEF398C
:100B7000EAE601FB0CF140F2491303FB01F31B13FE
:100B8000E8E7DDF8248098F87E5098F8824098F8DD
:100B90007F3098F8830098F880600A950E9498F852
:100BA000845098F881400B930F9098F885301193FA
:100BB0000EAA0AA909F5FC700C9610950D9401F087
:100BC000ABF998F88630C9F8883298F887302BB39B
:100BD000C3F10803C9F8503298F88B3003EB830354
:100BE00003EB43139B11C9F88C3298F88F3044F211
:100BF0008062C0F2020203F00703D35CC9F89032AE
:100C000098F88C3003EB830303EB43139B11C9F873
:100C1000843213B0BDEC088BBDE8F08F1023D9E708
:100C20002DE9F04F2DED048B89B0D0F89052DDF80E
:100C3000588007918146D0F88C0298F80DE09B46C9
:100C4000A2F5000305FB03F500FB0BF0A0FB056715
:100C5000EB1700FB037714468EFB0523900B40EA4D
:100C60008340FE1186EAE67380EAE072A2EBE0724E
:100C7000A3EBE6739342B8BF134609F5FC701E461A
:100C800001F082F9D8F80030002DB4BF4FF0FF32E8
:100C90000122B3F5005A06FB02001AD0D8F808204A
:100CA000002A40F0D980D8F804304FEACA2A07EE6B
:100CB00090AA07EE103AF8EEE77AB8EEC77AF2EEAD
:100CC000086A67EE877A87EEA67AFDEEC77A17EE96
:100CD00090AA4FF05A5309EE103A45F62943C3F64D
:100CE0008F53D9F8842298F80C1008EE903A43F20A
:100CF0003333C4F2431308EE103A82FB0B23C4F1E2
:100D000080744FEA122B4BEA036BE3170BFB03F2E1
:100D100098F80E30002704FB07225B04ABFB046746
:100D200081FB0445C3F57E0BE30943EA45635B455C
:100D300017444FEA166138BF5B4641EA0721D8F8ED
:100D400014208B4238BF0B4692449B4600EB0A03AB
:100D500005934E4609F50C744F46002514E05044A7
:100D600000F0C2FFC6F8A001384600F027FB626A17
:100D700002BBC6F898010135062D07F1440706F1BC
:100D8000100604F1040452D098F818302B4113F0E7
:100D9000010344D0E36B2068002BE0D1059B18448D
:100DA00000F0A2FFC6F8A001384600F007FB626A17
:100DB000002ADED0D117ABFB0223CDE90223039A30
:100DC00006900BFB01230393DDE90201020E42EAC8
:100DD000012207EE902AF8EE677AB0EE480A67EE35
:100DE000897AA7EEA80A0EF05FFDFCEEC07A06989D
:100DF00017EE901AC3174FEA011E0EFB03F3090FFB
:100E000000FB0131AEFB0023CDE902230B44039329
:100E1000029B1A0F039B42EA0312801AA9E7384685
:100E2000029300F0CBFA029BC6F89831A3E7D8F8FA
:100E30002C00D9F850120268D9F88832019109F5CE
:100E4000127100919468079909F5CC72A04709B016
:100E5000BDEC048BBDE8F08F21230C21C8F2040304
:100E600091FBF2F202FB0AFA83FB0A1353444FEAA6
:100E7000EA7ACAEB233A41F6FF7393FBF2F303FBE2
:100E80000AFA4FEACA2A24E770B50646044600F576
:100E9000CC7520460021443400F042FBAC42F8D12E
:100EA00006F5FC700021BDE8704001F0BBB800BF42
:100EB0002DE9F04F45F255549246C0F2150404FB5B
:100EC0000AF4994604F142732DED088B08EE903A2E
:100ED0004FF04E530AEE103A4CF28303CBF6CA633E
:100EE00009EE903A43F27A63C3F6AB4309EE103A47
:100EF0004DF20A73C3F623430BEE103A4AF63B2336
:100F0000C4F6B83345F256550AEE903A18EE903AC8
:100F1000C5F2555593B085FB0A2803F23173A8EB4F
:100F2000EA7844F2886B08EE903A4FEA690302953A
:100F3000074607900891A8F1070809930C46054653
:100F4000C0F2020B00262AE0B9F1000F00F3128173
:100F50006FF0EE0101FB02F20732D21000EB021338
:100F6000B8F1000F23EAE373627B40F30181B8F12B
:100F70001F0FCCBFC2EB421208FB02F2D21000924C
:100F8000384601360EAA0AA900F024FB062E04F109
:100F9000150405F1040507F1440700F0FB80627CAD
:100FA000A37CE17C207D002A71D003F0030C4FF07C
:100FB000640E40F678031EFB0C11C0F2440303FBE1
:100FC00001F307284FEAE301C3BF073843F2914317
:100FD000434300230B44C5F83032A37BC5F86C2291
:100FE00003F003035BF82330C5F8543220782179ED
:100FF000627863790A90A0780E910B92A179E278D9
:101000000F930C90E379207C0D921193109100F0D6
:10101000D7FA237AC3EB0A03B3F1110200F18680F9
:10102000029A217B94F80AE0103B82FB03C2A2EBF8
:10103000E37301B303291ED01F2BDBBF44F21872E8
:10104000C0F20202FA23D35C03FB0EFE40F2491306
:1010500003FB0EF301294FEAE33316DD18447F2822
:10106000A8BF7F20B9F17F0F4FEA4010E27B7FF7E6
:101070006BAF0F216EE703FB0EF340F2491202FB48
:1010800003F301294FEA2333E8DC5B42E6E7B8EEDD
:10109000E88A069028EE0A0A059120EE290A0493B0
:1010A00003920EF001FC20EE090AF1EE0C7A80EEBC
:1010B000277A0698049B0599073844F2986E03F046
:1010C0001F03C0F2020E5EF8233007EE900A27EEEF
:1010D000087AF8EEE77AA7EE278ABDEEC88A18EEFE
:1010E000102A1A441346039A00293FF474AF07EEFE
:1010F000901AF8EEE77AB7EE000AA7EE8B0A04938F
:101100000EF054FCF6EE007AE0EE2A7A17EE900A22
:1011100010F0ACFF41EC100B0EF012F851EC100B7C
:1011200011F0A8FA049B039A034454E7029B94F835
:1011300009C0C2F10101E27A83FB013EAEEBE1712D
:1011400002B3032A1ED01F29DBBF44F2187EC0F26F
:10115000020EFA211EF8011040F2491301FB0CF1B6
:1011600003FB01F3DB13012A3FF778AF5B4275E71E
:10117000002204E744F24063C0F202030999595C7B
:10118000EF39E7E601FB0CF140F2491303FB01F3F1
:101190001B13E8E7089A079992F88630C1F888325D
:1011A00092F887303BB3C3F1080308461446C0F8F1
:1011B000503294F88B3003EB830303EB43139B1102
:1011C000C0F88C3294F88F3044F28062C0F2020290
:1011D00003F00703D35CC0F8903294F88C3003EB33
:1011E000830303EB43139B11C0F8843213B0BDECAF
:1011F000088BBDE8F08F102308461446D7E700BFE0
:101200002DE9F04104460F4600F5CC7806460D4620
:101210003946204600F036FAD5F89C31C6F89C31A4
:101220004434D5F8A431C6F8A431444507F1440745
:1012300005F1100506F11006EAD1BDE8F08100BF06
:10124000D1F8AC31D1F8A42110B4D1F89C41C0F848
:101250009C41C0F8A421C0F8AC31D1F8B431C0F839
:10126000B431D1F8BC31C0F8BC31D1F8C431C0F8C8
:10127000C431D1F8CC31C0F8CC31D1F8D431C0F878
:10128000D431D1F8DC31C0F8DC31D1F8E431C0F828
:10129000E431D1F8EC31C0F8EC31D1F8F431C0F8D8
:1012A000F4315DF8044B70470023C0F89C31C0F85E
:1012B000A431C0F8AC31C0F8B431C0F8BC31C0F8CA
:1012C000C431C0F8CC31C0F8D431C0F8DC31C0F83A
:1012D000E431C0F8EC31C0F8F43170474FF4884382
:1012E000C4F22C7307EE103A87EE000A4FF09743D2
:1012F00007EE903A20EE270A4DF64C53BCEEC00A9A
:10130000C2F2000383ED000A704700BF30B40C68DE
:101310000460146804614D684560556845618D68D6
:10132000856095688561C968C160D268C261132C07
:101330004FF0000282624263DBBF44F23C72C0F2B3
:1013400002021C3452F824400362641003EB84133D
:10135000A3F58553026802994162102B02EB8204C7
:10136000B8BF102302EBC4021B04002B01EBA21236
:10137000D4BF0024012401253E2A80F84050C362D6
:1013800080F8304016DC02F0030392100433083278
:1013900003FA02F2D3174DF64C51C2F2000109686C
:1013A000A1FB024501FB0355230E43EA052383639A
:1013B00030BC70474FF060720023ECE7426B022AAA
:1013C000F0B4034605DD032A66D190F840100029E9
:1013D00062D193F8301071B9986A996BDC6A401A3F
:1013E000A042986259DC511C03299C6259635BDD61
:1013F0002046F0BC70474FF6FF70996AC0F2B360A8
:1014000081424CDDC1F1885000169D6BDC6A05FB02
:101410000010A042986240DB511C03299C62596372
:10142000E6DC03EB820251691329DBBF44F23C7016
:10143000C0F2020001F11C0550F82150196A586AE7
:101440006D1001EB8511A1F585511029B8BF102150
:1014500009048C42ACBF00250125D96283F83050C5
:10146000526802EB820102EBC10200EBA2123E2A9B
:101470004CDD4FF0607600274DF64C52C2F2000270
:1014800020461268A2FB064502FB0755220E42EADF
:1014900005229A63F0BC7047986AF0BC704700213F
:1014A000C0F2B4610A20B0E703EB8202516913294C
:1014B000DBBF44F23C70C0F2020001F11C0550F8A1
:1014C0002150196A586A6D1001EB8511A1F58551FB
:1014D0001029B8BF102109048C42ACBF002501259A
:1014E000D96283F83050526802EB820102EBC102EC
:1014F00000EBA2103E28BCDC00F00306801004368E
:10150000083006FA00F00646C717B5E702F00306F2
:1015100092100436083206FA02F21646D717ABE7E5
:1015200090F840308B4241D000290CBF03230023A8
:1015300030B49D00421980F8401043631369816AFA
:10154000132BDBBF44F23C72C0F2020203F11C0415
:1015500052F82340036A426A641003EB8413A3F534
:101560008553102BB8BF10231B048B42D4BF00211E
:10157000012180F83010C362435903EB830103EB70
:10158000C10302EBA3123E2A11DD4FF0607200236B
:101590004DF64C51C2F200010968A1FB024501FB66
:1015A0000355230E43EA052330BC8363704702F0E2
:1015B000030392100433083203FA02F2D317E7E769
:1015C0001328DBBF44F23C73C0F202031C3053F813
:1015D0002000704730B40C680460146804614C68E3
:1015E0004460546844618C68846094688461C9680C
:1015F000C16090F84010D568029AC56103624262EA
:10160000002934D0132CDBBF44F23C71C0F202013C
:101610001C3451F824408568816A641003EB8413FC
:10162000A3F58553102BB8BF102305EB85041B04CD
:1016300005EBC4058B4202EBA512D4BF00210121AA
:1016400002243E2AC36280F83010446311DD4FF05B
:10165000607200234DF64C51C2F200010968A1FBF3
:10166000024501FB0355230E43EA0523836330BC87
:10167000704702F0030322410433083203FA02F2F6
:10168000D317E7E70A680B69036102604B684360A0
:101690004B6943618B6883608B698361CB68C360EE
:1016A000F0B5CB69C3610B6A4F6A8E6ACD6A91F857
:1016B00030E04C6B8A6B036291F84030476286627F
:1016C000C56280F830E04463826380F84030F0BD4A
:1016D00070B54FF09D432DED048B08EE103A41F2AA
:1016E0003063002144F2CC04C3F680730020C4F2BE
:1016F000D01108EE903AC2F201040025B6EE009A2D
:101700000BE078EE097A17EE900A10F0AFFC41EC8E
:10171000100B0DF015FD51EC100B6E0010F0AAFF30
:1017200001360135B5F5806F28EE288A44F8260089
:10173000E7D1002340F2FF355A00D11C501C54F869
:10174000211054F820000133091AAB4244F2CC00B6
:1017500044F82210C2F20100EED141F6FC73BDEC58
:10176000048BC35841F6F872C3F10043835070BD37
:10177000002207EE902A4FF0974202EE102A4FF017
:101780006C5204EE902A4FF06E5202EE902A4AF606
:10179000AB22C3F62A2242F2CC0303EE102AC2F295
:1017A00001030022F6EE003AB7EE006AB0EE004AFE
:1017B000F0EE465AE7EEE75A03EBC2010132B0EE13
:1017C000677AA5EEA47AB2F5806FB0EE465AA7EE1E
:1017D000475AF0EE636AE7EE826AB0EE677AA5EEEA
:1017E000247AFDEEE66AC1ED016AF0EE466AE7EEA4
:1017F000476AB0EE677AA6EEA27A76EE856AB0EE18
:10180000465AA7EE475A35EE257AA6EE847AE7EED9
:10181000037ACDD130B4002240F2FF355100C81C0C
:101820004C1C53F8200053F824400132001BAA42FC
:1018300042F2CC0443F82100C2F20104EED14FF091
:10184000974306EE903AB6EE007AA7EEA67A41F6F6
:10185000FC7341F6F872E358FDEEC77A17EE901A62
:10186000CB1AA35030BC7047704700BF2DE9F04F32
:1018700044F2A07491B003EB4303C0F2020404EB02
:10188000C3041546069007910FCC0AAE0FC694E824
:101890000300002386E803004FF0010844F2CC0661
:1018A0000AAF05F160098DF824808DF825308DF898
:1018B0002630C2F2010605973BE00AF1FF30069B95
:1018C00000EB001003EB0010133020F00F0095E840
:1018D000084003F1724B4FEA6B3340F2FE721A403C
:1018E000531C56F8222056F82340CBF30D0382FBFD
:1018F0000323920B4FEA2B6B42EA8342CBF1060B98
:10190000144444FA0BF4BEF58C6F6C601CDAB4F529
:101910008C6F19DABCF1000F03D110AB9A440AF8AE
:101920001CCCEB68AA6803EB8213EB601035A94569
:101930002FD0059B53F8041B059311F0030A01F007
:10194000040CBAD10798C2E710AB9A441AF81C3CB1
:101950001BB11CF1000318BF0123C1F301123AB1FE
:1019600010AF07EB020C1CF81CCCBCF1000F13D11C
:1019700001F0C001C02902D11B9A0F2A20DDAA68FC
:10198000E96801930094734600F09AF80AF81C8CF9
:10199000C7E711B0BDE8F08F0699D5F808C0013A45
:1019A00002EB021201EB02111331EA68029321F0FB
:1019B0000F0163460194CDF800E000F015F8E5E76B
:1019C0001746E968AA6802971A9F03938DE890006A
:1019D000734600F0D3F8D9E710B54FF40971044607
:1019E0000AF0EAFD204610BD2DE9F04F099E0A9C41
:1019F0009DF82C50C6EB040C0CF1200C9E464FEACF
:101A0000AC1C47F2D80785B3C2F201074FF0400B78
:101A10004FF0000A51F82A4014444FEA643840F26B
:101A2000FE7508EA0505C4F30D0457F825300135A5
:101A300083FB048957F8255050F82A304FEA983430
:101A400044EA89442C44664484FB06894FEA1864BE
:101A500044EA09242344BBF1010B40F82A307244C4
:101A60000AF1010AD6D1BDE8F08FAA46C2F20107F9
:101A70004FF0400B51F82A3013445D1340F2FE74CE
:101A80002C40C3F30D0357F82450013485FB038920
:101A900057F824404FEA983343EA89431C4466448C
:101AA00084FB0645230E43EA0523BBF1010B40F8F6
:101AB0002A3072440AF1010ADCD1BDE8F08F00BF80
:101AC0002DE9F043079C9DF82050C3EB040C0CF16A
:101AD000200C4FEAAC1C47F2D80E4DB3C2F2010EF7
:101AE0004FF040094FF000084D1340F2FE742C40B7
:101AF000651C5EF824605EF82550C1F30D0486FB7A
:101B00000467B40B44EA87442C44634484FB0356C3
:101B10002C0E50F8285044EA06242C44B9F101094F
:101B200040F82840114408F10108DDD1BDE8F083F8
:101B3000A846C2F2010E4FF040094D1340F2FE7468
:101B40002C40651C5EF824605EF82550C1F30D043E
:101B500086FB0467B40B44EA87442C44634484FB4B
:101B600003562C0E44EA0624B9F1010940F8284036
:101B7000114408F10108E0D1BDE8F0832DE9F04FF0
:101B8000099F0A9C9DF83080D4F800C065680B9EC0
:101B9000C3EB070A0AF1200A1C4696464FEAAA1A26
:101BA00047F2D807B8F1000F39D0C2F201076246F8
:101BB00006F1010BD4464FF040094FF00008BA4639
:101BC00000E03546561946FA0BF60E44721340F201
:101BD000FE731340C6F30D025AF82360013386FBEF
:101BE00002675AF82330B20B42EA874264441A442F
:101BF00082FB0423160E46EA032650F82830B9F17A
:101C00000109334440F828307144334608F1010893
:101C10002A46D6D10A9A15605360BDE8F08F8646F1
:101C200001366046C2F201074FF040098B469446E8
:101C300000E00D46284430415844421340F2FE7300
:101C40001340C0F30D0057F82320013382FB00013D
:101C500057F82320830B43EA814354441A4482FB00
:101C60000423110E41EA0321B9F101094EF82810AD
:101C7000E3440B4608F101082846DAD10A9A1560B8
:101C80005360BDE8F08F00BF38B54FF0AB4307EEAF
:101C9000903A2DED048B87EE808A41F23063C3F6D3
:101CA000807346F2C80447F2CC05C2F20104C2F2C6
:101CB000010509EE103AF6EE008A78EE287A28EE51
:101CC000098A17EE900A10F0D1F941EC100B0DF0D3
:101CD00037FA51EC100B10F0CDFC44F8040FA5427C
:101CE000EBD1BDEC048B38BD10B446F2CC01C0F38F
:101CF0008934631CC2F20101C0F30D0251F8233094
:101D000051F824105DF8044B5B1A83FB0223920BFD
:101D1000001642EA8342C0F1140388181841704744
:101D200043F20C03C4F6C06307EE903A87EE800AD4
:101D300047F2D003C2F20103F6EE007A30EE270A32
:101D4000BDEEC00A83ED000A704700BF0B7810B4E7
:101D5000002B35D003EB830303EB43139A119F2A27
:101D6000C5BFA2F1A0031B110B230B3302FB03F32E
:101D700047F2D002C2F20102146803FB04F343608D
:101D80004A78C2F16303EAB103F00F021B11013379
:101D900010329A404FF680731340802BB8BF8023D7
:101DA00004FB03F304FB02F2436102614B7903720B
:101DB0000B795DF8044B003318BF01238372704721
:101DC0000B23D5E74FF0FF3303614361EEE700BF1C
:101DD00003684168027A0B44022A03603BD00CD9A5
:101DE000042A14D032D3052A2DD199423DD8407A05
:101DF00080F0800001300004704782B3012A22D1B4
:101E00004FF6FF701A0AC0F27F00504070471B0A5D
:101E1000581340F2FE7247F2D8010240C2F20101AB
:101E200030B451F82240C3F30D03013284FB034563
